:0800000C32322E342E302E3565
:1000000ADCF7FDDF2318FED91E2A2E0DE80D13EBAF
:1000000A2B161AEFFBF5F8F7FEF9FEFFFA41352732
:1000000AF2473A4429011F220444312023091816D1
:1000000A13171B16161A1E1916222425212621211A
:1000000A25292426222E30312D322D2D3135302D21
:1000000A37363D383D38383C403B38414148434813
:1000000A4343474B464366486A3B716063496367AB
:1000000A4C8C6A4F988C7E497F6E715781855A7FD6
:0100000A7F76
:020000040800F2
:40800000C0D90120E1BD0008F3BD000855FC0308F7BD0008F9BD0008FBBD00080000000000000000000000000000000021830008FFBD000800000000E583000859840008CD
:4080400005BE000805BE000805BE000805BE000805BE000805BE000805BE000805BE000805BE000805BE000805BE000805BE000805BE000805BE000805BE000805BE000850
:4080800005BE000805BE000829630308876803089B69030805BE000805BE000805BE00082FCC03083BCC030847CC0308BFCB0308E1CB0308EFCB0308FBCB0308C5930308AE
:4080C000D5930308E5930308EF93030805BE0008F99C0308C5730308CF730308D973030805BE000805BE000805BE000853CC03085FCC03086BCC030823CC030805BE0008E3
:4081000005BE000805BE000805CC030805BE000805BE000805BE000811CC03081BCC030805BE000805BE000805BE000805BE000805BE000805BE000805BE00084169030850
:408140000F6A0308856A030805BE000805BE000805BE000805BE000805BE0008F7730308F99303080994030805BE000805BE000805BE000805BE000805BE000800000000DF
:4081800005BE000805BE0008017403080B74030805BE000805BE0008039D030805BE0008000000000000000005BE000800F002F800F073F80AA090E8000C82448344AAF1AD
:4081C0000107DA4501D100F068F8AFF2090EBAE80F0013F0010F18BFFB1A43F00103184748080400680804000A444FF0000C10F8013B13F0070408BF10F8014B1D1108BF75
:4082000010F8015B641E05D010F8016B641E01F8016BF9D113F0080F1EBF10F8014BAD1C0C1B09D16D1E58BF01F801CBFAD505E014F8016B01F8016B6D1EF9D59142D6D37C
:40824000704700000023002400250026103A28BF78C1FBD8520728BF30C148BF0B607047632937F07683732937F07B83002070471FB53CF09CF89DE8030037F000FB37F075
:40828000AAF937F06FFC0400002000213BF0C0F9401C60601FBD10B510BD37F03EFC1146FFF7E6FF12F00BFF37F06FFC03B4FFF7F2FF03BC37F0A0FC80F309887047EFF3E8
:4082C00009807047684680F3098804480078C00714BF0220032080F31488704770790408DFF818C0EFF305831B0618BF6047EFF31483DB0708BF604700DF7047972704084D
:40830000DFF818C0EFF305831B0618BF6047EFF31483DB0708BF604700DF70479D290408EFF30980816911F8021C01B142E010B590E80F10E047BDE81040EFF3098C254BA5
:4083400093E80600914232D041B91EF0100F16D12149086820F00100086010E00CB41EF0100F06BF2CED108A0323012381F826302CE9F00FC1F82CC03AF0A6FE0CBC1A600F
:40838000D2F82CC0BCE8F00F92F8263013F0020F1ABFBCEC108A6FF0120E6FF0020E8CF3098813F0010F08BF704792F82500CCF80000704710B5094A1268914209D8084C02
:4083C00054F8214090E80F10A047EFF3098C8CE80F0010BD1408002034EF00E044FC030844FC030810B53AF023FDBDE81040194B93E80600914208BF70470CB4EFF3098C45
:408400001EF0100F06BF2CED108A0223002381F826302CE9F00FC1F82CC03AF055FE0CBC1A60D2F82CC0BCE8F00F92F8263013F0020F1ABFBCEC108A6FF0120E6FF0020EB2
:408440008CF3098813F0010F1CBF92F82530CCF8003070471408002010B53AF005FFC4E710B53AF097F93AF0FFFEBEE70B49D1F800C04A685CF8043B1068184442F8040B10
:408480008C4528BFA1F1DC0C8A4228BFA1F1DC02C1F800C04A6020F0004070471CFC00200146FB48B0F8AA0000EE100AB8EE400A81ED080AF64890ED800A81ED010A90ED76
:4084C000810A81ED020A90ED820A81ED030A90F8AF0000EE100AB8EE400A81ED050AEC4890F8AE000877EA4890ED7D0A81ED000A90F8B00000EE100AB8EE400A81ED060A02
:40850000B7EE000A81ED040A012070474FF6FF76DFF880C300DF074639460120DFF878C300DF0421DD4880F8D0110021DC4880F8441000BF002231460120DFF868C300DF99
:408540000446012C17D100BFD44890F8D10140F00101D24880F8D111B0F8DC014FF6FF71884207DACD48B0F8DC01401C81B2CB48A0F8DC11DEE7022CDCD1DFF82CC300DFD6
:40858000054605F001000028D4D0C548FFF788FFD0E7C34880ED0C0ADFEDC40AC0ED0D0ADFEDC20AC0ED0F0ADFEDC00AC0ED0E0A80ED0A0A704710B52DED0C8BB0EE409AA2
:4085C000B0EE608AF0EE419A9FEDB80AF0EE408A2422B349243101F1240037F092F89FEDB40AC9EE000AAE48C0ED090AB5EEC08AF1EE10FA04D1B0EE480AFFF7CAFF10E1DA
:40860000B5EEC08AF1EE10FA07DDA54890ED130AB5EEC00AF1EE10FA0CD9B5EEC08AF1EE10FA0FD29E4890ED130AB5EEC00AF1EE10FA07DBB0EE480AFFF7ABFF31F024FC7E
:4086400097490867964A92ED080ABCEEC00A10EE101A106F31F01EFC50BBB5EEC08AF1EE10FA0ADD9FED930A8D4880ED0A0A9FED8F0A914880ED000A11E09FED900A884841
:4086800080ED0A0AD0ED050AB7EE001A81EE200AF0EE000A80EE201A874880ED001A804890ED0A0A80ED0C0A012085490870B8E09FED800AB4EEC08AF1EE10FA07DB9FEDFB
:4086C000810A774880ED0A0AF0EE488A80E09FED7B0AB4EEC08AF1EE10FA07D89FED7A0A6F4880ED0A0AF0EE488A71E0724890ED000A30EE290A80ED000A694890ED050A4B
:40870000DFED720A20EE200A6B48D0ED000A20EE200A10EE101A08463BF0D8FD41EC1D0BB0EE4D0AF0EE6D0A39F06AF8B0EE40BAF0EE60BA5A4890ED060A10EE101A084632
:408740003BF0C4FD41EC1C0B53EC1B2B3BF0C8FA41EC1A0B3AF07EFF08EE900AF5EEC08AF1EE10FA05DD4E4890ED060AF0EE408A06E04B4890ED060AB1EE400AF0EE408A64
:4087800038EE880AF0EE408AB5EEC08AF1EE10FA09DDF5EEC08AF1EE10FA04D89FED4C0AF0EE408A0DE0B5EEC08AF1EE10FA08D2F5EEC08AF1EE10FA03DB9FED460AF0EED6
:4087C000408A374890ED000A20EE280A80ED0A0A3B48007870B13248C0ED0C8A90ED0A0AD0ED090A30EE600A80ED0D0A00203449087016E09FED2D0A2949243101F12400F7
:4088000016F02FFB26493431A1F1300015F048FFF0EE408A224890ED0C0A30EE280A80ED0C0A1F4890ED0A0AB5EEC00AF1EE10FA0BDD90ED0C0AB5EEC00AF1EE10FA04D2B9
:408840009FED1A0A80ED0C0A54E0154890ED0A0AB5EEC00AF1EE10FA0BD290ED0C0AB5EEC00AF1EE10FA04DD9FED100A80ED0C0A40E00B4890ED0C0ADFED0E0AB4EEE00A07
:40888000F1EE10FA28DD9FED0B0A80ED0C0A31E030210020413504080129040878520020DC16002061290408A92804080000000000007A440000C842A00300200000C8C2E8
:4088C0009C03002066662640666626C0DB0FC9400AD7233C0AD723BCF74890ED0C0A5FED090AB4EEE00AF1EE10FA03D21FED0D0A80ED0C0AF04890ED0C0ABDEC0C8B10BDE9
:4089000001B500BF01226946EC480068B03012F091FE20B99DF80000E94981F8B00000BFE848D0F8CC110120DFF89CC300DF08BD10B52DED020B00BF04226946DF4800687C
:4089400000F5FA7012F076FE20B99DED000ADC4880ED7D0A00BFDB48D0F8CC110120DFF868C300DF1CBD01B500BF01226946D3480068AE3012F05EFE20B99DF80000D049AE
:4089800081F8AE0000BFCF48D0F8CC110120DFF838C300DF08BD01B500BF01226946C7480068AF3012F046FE20B99DF80000C44981F8AF0000BFC348D0F8CC110120DFF891
:4089C00008C300DF08BD10B52DED020B00BF04226946BA48006800F5027012F02BFE20B99DED000AB64880ED820A00BFB548D0F8CC110120DFF8D0C200DF1CBD10B52DEDA6
:408A0000020B00BF04226946AC48006800F5017012F010FE20B99DED000AA94880ED810A00BFA848D0F8CC110120DFF89CC200DF1CBD10B52DED020B00BF042269469F48A4
:408A4000006800F5007012F0F5FD20B99DED000A9B4880ED800A00BF9A48D0F8CC110120DFF864C200DF1CBD01B500BF0222694692480068AA3012F0DDFD20B9BDF8000004
:408A80008F49A1F8AA0000BF8E48D0F8CC110120DFF834C200DF302004F062FD08BD10B58AB00446022C1FD1B2EE040A8DED090A9FED860A8DED020A1FED840A8DED030AC7
:408AC0009FED820A8DED040A9FED810A8DED060A01208DF820009FED7F0A8DED010AB1EE080A8DED070AA8E0042C1FD1B3EE080A8DED090A1FED910A8DED020A1FED950AD9
:408B00008DED030A1FED950A8DED040A1FED970A8DED060A01208DF820009FED6F0A8DED010AB1EE040A8DED070A86E0052C01D01A2C1FD1B2EE060A8DED090A9FED670AE4
:408B40008DED020A1FEDA70A8DED030A9FED630A8DED040A1FEDA90A8DED060A01208DF820009FED5F0A8DED010AB2EE020A8DED070A62E00E2C1FD1B2EE040A8DED090A43
:408B80009FED520A8DED020A1FEDB80A8DED030A9FED520A8DED040A9FED4D0A8DED060A01208DF820009FED4E0A8DED010AB2EE040A8DED070A40E0152C1FD1B2EE040AAE
:408BC0008DED090A9FED470A8DED020A1FEDC90A8DED030A9FED430A8DED040A9FED3C0A8DED060A01208DF820009FED3A0A8DED010AB1EE080A8DED070A1EE01FEDD50A22
:408C00008DED090A1FEDD70A8DED020A1FEDD90A8DED030A1FEDDB0A8DED040A1FEDDD0A8DED060A00208DF820001FEDE00A8DED010A1FEDE20A8DED070A9DED090ABDEEBD
:408C4000C00A10EE101A08B2FFF70EFFDDED020AB0EE600AFFF7EDFEDDED030AB0EE600AFFF7CCFEDDED040AB0EE600AFFF7ABFE9DED060ABCEEC00A10EE101AC8B2FFF7C2
:408C80008AFE9DF82000FFF76EFEDDED010AB0EE600AFFF74DFE9DED070ABCEEC00A10EE101AC8B2FFF72CFE302004F059FC552004F056FC0AB010BDDC160020FC0300201A
:408CC000302100207852002001290408000048420000A042F3FDD43CA69B443C0000484396438B3C0000F042204890ED0A0ABDEEC00A10EE100A00B270471C4890ED090A76
:408D0000BDEEC00A10EE100A00B2704780220270164A92ED010ADFED160A20EE200ABCEEC00A10EE102A91B241700A0A82700F4A92ED020ADFED0E0A20EE200ABCEEC00A01
:408D400010EE102A91B2C1700A0A0271074A92ED030ADFED070A20EE200ABCEEC00A10EE102A91B241710A0A82717047DC1600200000C84270B5054601249148DFF844C208
:408D800000DF204670BD9049097801708F49416001218160002181764176704700B5A1B06846FFF7F0FF01208DF8180006219DF81920501CC0B28DF819000DF14B0081548E
:408DC00000208DF819006846019930F029FD002021B000BD00B5A1B06846FFF7D4FF02208DF8180005219DF81920501CC0B28DF819000DF14B00815400208DF81900684643
:408E0000019930F00DFD9DF81800401E0DF11B01085C21B000BD2DE9F74F814615464FF000081FFA89F7E8191FFA80FBBBF5005F02DD4FF0080855E02D2D02DD4FF0400832
:408E400050E04FF47A615E48DFF884C100DF012802D14FF0100845E0842036F057FA0446002C3FD0FFF79AFFFFF7B4FF82462046FFF789FFE81C20760221627E501C607628
:408E800004F14B008154390A627E501C607604F14B008154627E501C607604F14B008754627E014650182A46019936F0E5FB002060762046616830F0B3FC94F8800001281E
:408EC0000BD1FFF787FF06460AF0020010B106F0020020B14FF0800801E04FF02008204636F04FFA3648DFF8ECC000DFB8F1000F05D03948007840EA08003749087040464E
:408F0000BDE8FE8F2DE9F043A1B080460F4614460026BDB260191FFA80F9B9F5005F01DD082642E02D2C01DD40263EE06846FFF72AFFE01CC0B28DF8180003219DF8192090
:408F4000501CC0B28DF819000DF14B008154290A9DF81920501CC0B28DF819000DF14B0081549DF81920501CC0B28DF819000DF14B0085549DF819200146501855222146F5
:408F800036F0F1FB00208DF819006846019930F047FC9DF88000012806D122460DF11E01404636F069FB00E0202626B10A480078304309490870304621B0BDE8F083000029
:408FC000E8560020D52C04084A07002000380040C92D0408E52C0408F903002000487047E0FA0020401ECAB210F8011F8A4202D00029F9D100207047FFFFFFFFFFFFFFFF87
:40900000FE4890ED0A0A704710B52DED048BB0EE408A0446F94890ED720ADFEDF90A80EE201AB0EE419AF74890F8AE0058B1FFF7E7FFF0EE409A9FEDF41AF0EE480AFFF786
:40904000BAFAB0EE408AEF4890F89C00012803D1B1EE480AB0EE408A9FEDEC0AB4EEC08AF1EE10FA04D29FEDE90AB0EE408A0AE09FEDE70AB4EEC08AF1EE10FA03DD9FED67
:40908000E40AB0EE408A0E2C14D008DCA4F10200052866D2DFE800F0111410124B00A4F1120009285DD2DFE800F0430C5C065C5C0D5C0A0000BF00BF00BF00BF00BF00BFFF
:4090C00000BF00BFB5EEC08AF1EE10FA0ED2B1EE480AB0EE408A0021CE4800782EF03CFB0121CD4800782EF037FB19E0B5EEC08AF1EE10FA0ADD0121C64800782EF02CFB3D
:409100000021C54800782EF027FB09E00021C14800782EF021FB0021BF4800782EF01CFBB0EE480ABD48007832F01AFF1AE000BFF0EE000A89EE200A9FEDB51AC8EE010AA9
:4091400060EE890AB1EE001AC0EE811A70EE218ADFEDB30AB0EE680AB24800782EF076FB00E000BF00BFBDEC048B10BDAE480078704710B50446AD480078A04205D0AB48BB
:4091800004700C2028F0F8F80DE0A948006830F0A3FEB0F5FA7F06D930F076FEA44908600C2028F0E9F810BD10B50446954991F830000FF089FF90B12046FFF7DAFF21461E
:4091C0009C4800782EF0C8FA21469B4800782EF0C3FA2146994800782EF0BEFA1CE02FF0E4F850B12146934800782EF0B5FA2146914800782EF0B0FA0EE021468D4800785F
:409200002EF0AAFA21468C4800782EF0A5FA21468A4800782EF0A0FA10BD10B52FF0C5F8C8B127F053FBDFED860AB4EEE00AF1EE10FA10D24FF47A718248006830F02AFEEC
:40924000E0B101217D4800782EF086FA30F01CFE7D49086012E02FF0A8F878B140F6B8317948006830F016FE40B10021734800782EF072FA30F008FE7249086010BD6A490A
:409280000870704770B52DED048B04460D466F48007848B10120207001216D4880F8291030F0F2FD6A490862207830B1012845D0022857D003287ED168E0654890F829005F
:4092C00001280ED16248016A284630F014FEFA2807D2012020705E4890ED090A84ED010A2BE05B4890F8350001280ED15848C16A284630F000FEFA2807D202202070544840
:4093000090ED0C0A84ED010A17E0514890F8410001280ED14E48816B284630F0ECFDFA2807D2032020704A4890ED0F0A84ED010A03E09FED480A84ED010A3FE0444890F802
:40934000290030B14248016A284630F0D4FDFA2802D90020207004E03D4890ED090A84ED010A2BE03A4890F8350030B13848C16A284630F0C0FDFA2802D90020207004E0BB
:40938000334890ED0C0A84ED010A17E0304890F8410030B12E48816B284630F0ACFDFA2803D90020207005E005E0294890ED0F0A84ED010A02E00020207000BF00BF94EDE5
:4093C000020A84ED030A2078B0B194ED050AB5EEC00AF1EE10FA6ED094ED010A10EE101A08463AF073FF41EC190BB0EE490AF0EE690A37F045FB2FE086E00000F808002099
:4094000000007A44302100206F12833A0000C8C20000C8423D0700203E0700209B070020030058416307002038000020400000203C0000207C070020940700209C07002045
:409440003D0A0F4030000020340000202D0000204C08002000000000B0EE408AF0EE608A9FEDFA0B53EC102B51EC180B3AF0FCFB3DD894ED010AB5EEC00AF1EE10FA04D169
:409480001FED0C0A84ED020A35E094ED010AD4ED050A30EE600AD4ED020AB4EEE00AF1EE10FA09DD94ED020AD4ED050A30EE200A84ED020A1FE01AE094ED010AD4ED050A75
:4094C00030EE200AD4ED020AB4EEE00AF1EE10FA08D294ED020AD4ED050A30EE600A84ED020A08E094ED010A84ED020A03E094ED010A84ED020A94ED020A84ED040A01209C
:40950000D44981F8480013E01FED2E0A84ED020A1FED300A84ED010A1FED320A84ED030A1FED340A84ED040A0020CA4981F8480094ED040AC74880ED110ABDEC048B70BDC9
:4095400070B52DED088B044603F066FFB0EE408A94ED090AD4ED0B0A30EE200AF0EE000A80EE201AF0EE418A94ED080AD4ED0A0A30EE200AF0EE000A80EE201AB0EE419A6B
:4095800094ED020AB4EEE80AF1EE10FA33DD94F84400022825D1B2EE040A03F000F8E0B994ED120A38EE400AF0EE040AB4EEE00AF1EE10FA11D20FF0AFFD10B141F28830C7
:4095C00001E04FF47A7005462946E06C30F062FC30B101215020015502E000215020015508E0022084F8440084ED128A30F04CFCE06400BF5EE094ED020AB4EEC90AF1EEE6
:4096000010FA33D294F84400012825D1B2EE040A02F081FFE0B994ED120A38EE400AF8EE040AB4EEE00AF1EE10FA11DD0FF074FD10B141F2883001E04FF47A70054629462B
:40964000E06C30F027FC30B101215020015502E000215020015508E0012084F8440084ED128A30F011FCE06400BF23E0002084F8440094ED120A30EE480A10EE101A08465D
:409680003AF024FE41EC1B0BB0EE4B0AF0EE6B0A37F0F6F9B0EE40AAF0EE60AA9FED6E0B53EC102B51EC1A0B3AF018FC02D2002150200155BDEC088B70BD70B52DED0C8B26
:4096C00004460D4694ED0A0AF2EE040AB4EEE00AF1EE10FA0CD294ED0A0AFAEE040AB4EEE00AF1EE10FA03DD1FEDA60A84ED0A0A94ED0A0A5FEDBE0AC0EE208A95ED020A47
:40970000D5ED080AB4EEE00AF1EE10FA18D895ED0C0AD5ED020A20EE200A1FEDC31AC0EE010A94ED780A20EE800A1FEDCB1AC0EE010A95ED0D0A30EEC00A84ED620A25E008
:4097400095ED020AD5ED090AB4EEE00AF1EE10FA18DB95ED0C0AD5ED020A60EE200A1FEDD41A80EE810AD4ED780A60EE200A1FEDDC1A80EE810AD5ED0D0A30EE200A84ED05
:40978000620A03E01FEDCD0A84ED620A95ED020AB5EEC00AF1EE10FA02D11FEDE78A18E094ED620A10EE101A08463AF08FFD41EC1B0BB0EE4B0AF0EE6B0A37F061F9B0EE9D
:4097C00040AAF0EE60AA51EC1A0B39F043FF08EE100A94ED620A10EE101A08463AF076FD41EC1D0BB0EE4D0AF0EE6D0A37F048F9B0EE40BAF0EE60BA18EE900A3AF066FDF6
:4098000041EC1D0BB0EE4D0AF0EE6D0A37F038F9B0EE40CAF0EE60CA53EC1B2B51EC1C0B3AF06AFC41EC1A0B39F014FF09EE100A89EE080AB0EE409A1E210948B0EE490AE7
:409840001EF011F8BDEC0C8B70BD000000000000000059404C080020000000000000F83F380800202DE9F0412DED028B04460D46FA4890F8BD010A287DD14FF432700159EE
:40988000001D0151001FD4F8C4120151F448007832F0C1FAC4F8C4024FF432700059D4F8C412081A00EE100AB8EEC00ADFEDED0A80EE201A84EDB41A94EDB40AB2EE041AF2
:4098C000C0EE010A9FEDE80A20EE800A84EDC40A95ED020AD5ED080AB4EEE00AF1EE10FA23D895ED0E0AD5ED020A20EE200A9FEDDF1AC0EE010A94ED780A20EE800A9FED83
:40990000DC1AC0EE010A95ED0F0A30EEC00A84EDDA0A94EDDA0AB5EEC00AF1EE10FA37DD9FEDD40A84EDDA0A32E095ED020AD5ED090AB4EEE00AF1EE10FA25DB95ED0E0A8E
:40994000D5ED020A20EE200A9FEDC81AC0EE010A94ED780A20EE800A9FEDC51AC0EE010A95ED0F0A30EE800A84EDDA0A94EDDA0AB5EEC00A00E08CE0F1EE10FA08D29FEDF6
:40998000BD0A84EDDA0A03E09FEDBA0A84EDDA0AB24890F8300091280ED0B04890F83000922809D0AD4890F83000712804D0AB4890F83000B82803D132274FF0480802E034
:4099C00032274FF04108D4EDC40AB0EE600A394604F53E701DF047FFD4EDDA0AB0EE600A414604F554701DF03EFF94EDD40AD4EDBE0A30EE600AF2EE040A20EE208A9FED99
:409A00009C0AB4EEC08AF1EE10FA04DD9FED980AB0EE408A0AE09FED980AB4EEC08AF1EE10FA03D29FED940AB0EE408A012104F53970B0EE480A1DF016FF94EDD40A84ED3A
:409A4000DD0A94EDBE0A84EDC70A04261AE0711E04F55D7000EB810090ED000A04F55D7000EB860080ED000A04F5477000EB810090ED000A04F5477000EB860080ED000A1F
:409A8000701EC6B2002EE2DC94EDB90A7B4880ED150ABDEC028BBDE8F081704991F84A10062904D06D4991F84A10122901D1012000E00020704710B52DED020B00BF0422E7
:409AC00069466F48006800F5587011F0B3FD20B99DED000A614880EDD80A00BF1CBD10B52DED020B00BF042269466548006800F5577011F09FFD20B99DED000A574880EDC6
:409B0000D70A00BF1CBD10B52DED020B00BF042269465B48006800F5567011F08BFD20B99DED000A4D4880EDD60A00BF1CBD10B52DED020B00BF042269465148006800F580
:409B4000557011F077FD20B99DED000A434880EDD50A00BF1CBD414991F84A10032901D1012000E00020704710B52DED020B00BF042269464248006800F55C7011F05AFD01
:409B800020B99DED000A354880EDDC0A00BF1CBD10B52DED020B00BF042269463848006800F55B7011F046FD20B99DED000A2B4880EDDB0A00BF1CBD10B52DED020B00BFEF
:409BC000042269462E48006800F55A7011F032FD20B99DED000A214880EDDA0A00BF1CBD10B52DED020B00BF042269462448006800F5597011F01EFD20B99DED000A17480A
:409C000080EDD90A00BF1CBD144991F84A10042922D0124991F84A1002291DD00F4991F84A10052918D00D4991F84A100E2913D00A4991F84A1015290ED0084991F84A105D
:409C4000132909D0054991F84A10182904D0034991F84A101A2915D1012014E030210020600700208DED244800606A470000C84200007A440000000000007AC44C080020B3
:409C8000FC0300200020704710B52DED028B84B00446FFF760FF10B1B2EE048A01E0B7EE008AFE4890ED280A20EE080A84ED000AB0F8A80000EE100AB8EE400A84ED020A1B
:409CC0001FED140A84ED010AF44890F89C0084F82C00F24890F842106C3000EB810090ED000A84ED030AED4890F84210743000EB810090ED000A84ED040AE84890F8421066
:409D00007C3000EB810090ED000A84ED050AE34890F84210843000EB810090ED000A84ED060ADE4890ED700A84ED070A90ED710A84ED080A90ED720A84ED090A90ED730A46
:409D400084ED0A0A2DF0DEFC002876D0FFF7A5FE78B30121D24800782DF0FEFC0021D14800782DF0F9FC0021CF4800782DF0F4FCB2EE040AFFF7DBFE9FEDCC0AFFF7C3FE53
:409D8000B7EE000AFFF7ABFE1FED460AFFF793FE9FEDC70AFFF724FF9FEDC60AFFF70CFF9FEDC50AFFF7F4FE1FED4F0AFFF7DCFE95E0FFE7FFF728FFF0B3C048009094EDF3
:409DC000020AF0EE400A9FEDBE0A01231A46BD49BD48007831F026FD0021B14800782DF0BBFC0121AF4800782DF0B6FC0121AE4800782DF0B1FC9FEDB50AFFF798FE9FED0D
:409E0000AD0AFFF780FE9FEDAC0AFFF768FE1FED680AFFF750FE9FEDAE0AFFF7E1FE9FEDA50AFFF7C9FE9FEDA40AFFF7B1FE1FED700AFFF799FE52E000E041E0FFF78BFEE2
:409E400070B39E48009094ED020AF0EE400A9FED9C0A01231A469B499B48007831F0E2FC00218F4800782DF077FC01218D4800782DF072FC01218C4800782DF06DFC9FED26
:409E8000930AFFF754FE9FED8B0AFFF73CFE9FED8A0AFFF724FE1FED8A0AFFF70CFE1EE000217F4800782DF057FC01217D4800782DF052FC01217C4800782DF04DFC0EE04A
:409EC0007E48009094ED020AF0EE400A9FED7C0A012300227F497C48007831F0A3FC94F82C00B0B90020009001900290034603227949039055202DF006FD002000900190AE
:409F00000290034603227549039056202DF0FBFC15E00020009001900290034603226F49039055202DF0EFFC0020009001900290034603226849039056202DF0E4FC01202F
:409F400004B0BDEC028B10BD2DED028B5421644835F011FC4FF46771624835F00CFC5821614835F008FC5E48604908605E4848305F4908605B485F49086000F5F0705E495F
:409F80000860A0F5DC705D49086000F5B0705C49086000F59E705B4908604C305A490860514854305949086059485A4908604C481430594908601FEDD30A143880ED030A2E
:409FC0001FEDD60A484880ED130A9FED540A80ED140AFFF7C0FD40B1DFF844C100DF06460A22022130F05AF80AE02DF08BFB38B1DFF82CC100DF06460122022130F04EF869
:40A00000DFF81CC100DF0646022130F08DF8DFF810C100DF064631460120DFF808C100DF0321414880F8541000BF00224FF6FF710320DFF8F8C000DF044604F00100002878
:40A04000F3D104F002000028EFD0DFF8E4C000DF054605F0010030B121481430FFF714FE1D2027F089F905F002000028DDD03148007818F085FB1B4880ED780AD0ED780A62
:40A08000B0EE600A142100F5E4701DF0ECFB2DF021FB08B1284851E05FE00000302100207807002099070020980700206F12833A00401C45000048420000FA4380EC002093
:40A0C000A037A04B001800409B070020000048450080544500000140AD070020AE070020A4080020F80800204C0800200000002004000020080000200C00002010000020CC
:40A100001400002018000020200000201C000020600C002024000020280000200000C8C241350408012904087852002061290408A92804081B0700206C070020007818F02B
:40A14000DCFCFE4880ED0A0AD0ED0A0AB0EE600A1E2110301DF087FB87E02DF0D3FA002823D0FFF79AFC08B3F548007818F0C5FCF24880ED8E0AF348007818F001FBEF48FB
:40A1800080EDA40AD0EDA40AB0EE600A142100F51E701DF068FBE948D0ED8E0AB0EE600A142100F508701DF05EFB5EE0E648007818F0A3FCE14880ED0A0AD0ED0A0AB0EEAF
:40A1C000600A1E2110301DF04EFBDC4890ED0A0AD0ED040A30EE600A20EE000AB0EE408A1E212030B0EE480A1DF03DFBD748007818F083FCD14880ED200AD0ED200AB0EE81
:40A20000600A1E2168301DF02EFBCC4890ED200AD0ED1A0A30EE600A20EE000AB0EE408A1E217830B0EE480A1DF01DFBC848007818F063FCC14880ED360AD0ED360AB0EEC7
:40A24000600A1E21C0301DF00EFBC248007818F054FCBA4880ED4C0AD0ED4C0AB0EE600A1E2100F58C701DF0FEFABB49B348FFF7F9FAB949B148FFF720FAB748FFF760F9FF
:40A280002FF002FE06463146B348FEF7FBFFB248007818B1B14890F84800A0BB2DF01AFA90B19FEDAF0AAC4880ED020A0020A34908700021AB4800782DF04EFA0021AA48C7
:40A2C00000782DF049FA50E02DF01CFA00284CD09FEDA30AA04880ED020A0020974908700021A14800782DF037FA00219D4800782DF032FA00219D4800782DF02DFA002054
:40A30000FEF7BDFF31E0FFE7944890F8480001282BD18A48007840BB2DF0DCF968B10120864908700121904800782DF015FA01218C4800782DF010FA17E02DF0E3F9A0B178
:40A3400001207E4908700121874800782DF004FA0121844800782DF0FFF90121834800782DF0FAF90120FEF78AFFFEF756FFFEF7FDFE0646FEF718FF7D4991F84A00764980
:40A38000D1ED020AB0EE600AFEF73EFE4DE601B50DF076FB70B900BF01226946754800689C3011F047F920B99DF80000704981F89C0000BF7048016D0120DFF8C0C100DFDE
:40A3C000142003F0CDF808BD10B52DED020B00249DED000AF2EE040AB4EEE00AF1EE10FA05DDB2EE040A8DED000A02240BE09DED000AB5EEC00AF1EE10FA04D29FED580AD2
:40A400008DED000A032400BF0422694659480068A03011F00FF920B99DED000A544880ED280A00BF5448016D0120DFF850C100DF192003F095F820461CBD01B500BF022211
:40A4400069464C480068A83011F0F4F820B9BDF800004749A1F8A80000BF4748016D0120DFF818C100DF08BD10B5FFF774FB58B144F62060FFF7E1FFB6EE000AFFF7A4FFD2
:40A480000020FFF784FF1BE0FFF707FB50B12820FFF7D3FF9FED320AFFF796FF0020FFF776FF0DE0FFF7B0FB50B144F62060FFF7C4FF9FED2B0AFFF787FF0020FFF767FF66
:40A4C0002B4991F84A00FEF7EAFA012010BD70B52DED028BB0EE408A04460D460026012C04D0022C03D0032C6DD101E000BF00BF1A4890ED140AB4EEC80AF1EE10FA05DD4D
:40A5000090ED140AB0EE408A03260CE0134890ED130AB4EEC80AF1EE10FA04D290ED130AB0EE408A022610210C48DFF854C000DF012846D004EB4401084823E0F80800207C
:40A5400064070020690700206C0700206F070020AD070020AE070020A40800204C080020000000007D0700207E0700207F07002030210020FC03002078520020012904080F
:40A58000C92D0408143000EB810080ED018A2FF07BFC04EB4402F84941F82200012104EB4402F54800EB8200017204EB4401F24800EB81004572F0481438DFF8C0C300DFC8
:40A5C00000E0062601E0062600BF00BF3046BDEC028B70BDE848143890ED110A7047E84890F85000012800D170470020FCE7E248143890ED150A70470020DF49143991F87D
:40A600004810012904D1DF490978012900D10120704701B500BF01226946DB4800684A3011F008F820B99DF80000D84981F84A0000BFFFF719FFD648016D0120DFF854C340
:40A6400000DF272002F08CFF08BDCE4890ED780A7047CC4890ED8E0A7047CA4890ED040A7047C84890ED1A0A7047C64890ED080A7047C44890ED300A7047C24890ED460A65
:40A68000704700B5FFF767FA30B1C348007808B1012000BD0020FCE70020FAE700207047BD480078022804D1BC48007D012800D170470020FCE710B5FFF7EFF930B1B848CC
:40A6C00000782DF04BFC08B1012010BD0020FCE7AE4890F84A00182801D1012070470020FCE700B50121FFF7F3FF00B900E00021084600BD70B52DED068B0024FFF77CFF36
:40A7000080B32DF01BF868B3FFF7EBFF50B3FFF77BFA38B39D4890EDD50A10EE101A084639F0D4FD41EC180BFEF76AFC10EE105A284639F0CBFD41EC1A0BB0EE4A0AF0EE1D
:40A740006A0A36F09DF9B0EE409AF0EE609A53EC182B51EC190B39F0C1FB01D2012000E0002004462046BDEC068B70BD0020844991ED020A854991F84220743101EB820142
:40A78000D1ED000AB4EEE00AF1EE10FA10DB7C4991ED020A7D4991F84220843101EB8201D1ED000AB4EEE00AF1EE10FA00D8012070470020724991ED020A744991F8422053
:40A7C0006C3101EB8201D1ED000AB4EEE00AF1EE10FA10D86A4991ED020A6C4991F842207C3101EB8201D1ED000AB4EEE00AF1EE10FA00DB0120704700B50023FFF7D9FF99
:40A8000010B9FFF7B3FF00B10123184600BD70B52DED068B0024FFF7EFFE88B32CF08EFF70B3FFF7E9FF58B3FFF75BFF40B3FFF7EBF928B3554890EDD60A10EE101A084688
:40A8400039F044FD41EC180BFEF7DAFB10EE105A284639F03BFD41EC1A0BB0EE4A0AF0EE6A0A36F00DF9B0EE409AF0EE609A53EC182B51EC190B39F0F7F902D2012001E039
:40A8800001E0002004462046BDEC068B70BD70B52DED068B0024FFF7AFFE70BB2CF04EFF58B3FFF71EFF40B3FFF7AEF928B3374890EDD70A10EE101A084639F007FD41EC1F
:40A8C000180BFEF79DFB10EE105A284639F0FEFC41EC1A0BB0EE4A0AF0EE6A0A36F0D0F8B0EE409AF0EE609A53EC182B51EC190B39F0F4FA02D2012001E001E000200446C0
:40A900002046BDEC068B70BD70B52DED068B0024FFF77AF970B3FFF76FFE58B32CF00EFF40B3FFF7DEFE28B3184890EDD50A10EE101A084639F0CAFC41EC180BFFF799FE95
:40A9400010EE105A284639F0C1FC41EC1A0BB0EE4A0AF0EE6A0A36F093F8B0EE409AF0EE609A53EC182B51EC190B39F0B7FA19D2012018E018E0000060080020E52C040826
:40A98000A4080020F8080020FC0300203021002078520020012904082C000020002C0020A0070020002004462046BDEC068B70BD70B52DED068B0024FFF726F988B3FFF72B
:40A9C0001BFE70B3FFF7F5FE58B32CF0B7FE40B3FFF787FE28B3F74890EDD60A10EE101A084639F073FC41EC180BFFF742FE10EE105A284639F06AFC41EC1A0BB0EE4A0A34
:40AA0000F0EE6A0A36F03CF8B0EE409AF0EE609A53EC182B51EC190B39F026F902D2012001E001E0002004462046BDEC068B70BD70B52DED068B0024FFF7E6F880B3FFF710
:40AA4000DBFD68BB2CF07AFE50B3FFF74AFE38B3D84890EDD70A10EE101A084639F036FC41EC180BFFF705FE10EE105A284639F02DFC41EC1A0BB0EE4A0AF0EE6A0A35F0A0
:40AA8000FFFFB0EE409AF0EE609A53EC182B51EC190B39F023FA01D2012000E0002004462046BDEC068B70BD70B52DED068B0024FFF7AAF880B3FFF79FFD68B32CF03EFE50
:40AAC00050B3FFF70EFE38B3BA4890EDD50A10EE101A084639F0FAFB41EC180BFFF7CDFD10EE105A284639F0F1FB41EC1A0BB0EE4A0AF0EE6A0A35F0C3FFB0EE409AF0EEA6
:40AB0000609A53EC182B51EC190B39F0E7F901D2012000E0002004462046BDEC068B70BD70B52DED068B0024FFF76EF888B3FFF763FD70B3FFF71AFE58B32CF0FFFD40B3FC
:40AB4000FFF7CFFD28B39B4890EDD60A10EE101A084639F0BBFB41EC180BFFF78EFD10EE105A284639F0B2FB41EC1A0BB0EE4A0AF0EE6A0A35F084FFB0EE409AF0EE609A98
:40AB800053EC182B51EC190B39F06EF802D2012001E001E0002004462046BDEC068B70BD70B52DED068B0024FFF72EF880B3FFF723FD68BB2CF0C2FD50B3FFF792FD38B36B
:40ABC0007C4890EDD70A10EE101A084639F07EFB41EC180BFFF751FD10EE105A284639F075FB41EC1A0BB0EE4A0AF0EE6A0A35F047FFB0EE409AF0EE609A53EC182B51EC08
:40AC0000190B39F06BF901D2012000E0002004462046BDEC068B70BD70B52DED088B0024FEF7F2FFB8B32CF089FDA0B3FFF759FD88B3FFF71EFDF0EE400AFFF71EFD30EE2D
:40AC4000800AB0EE408A5B4890EDD80A10EE101A084639F03BFB41EC190BFFF7FEFC30EE480A10EE105A284639F030FB41EC1B0BB0EE4B0AF0EE6B0A35F002FFB0EE40AAE9
:40AC8000F0EE60AA53EC192B51EC1A0B39F026F902D2012001E002E00020044600BF2046BDEC088B70BD444890ED030A704710B50124404890F84A000E281BD03D4890F890
:40ACC0004A00022816D03B4890F84A00152811D0384890F84A001A280CD0364890F84A00032802D12CF00EFD20B9324890F84A00182800D100240CB1012010BD0020FCE79A
:40AD000010B50024FFF778FCB0B12CF017FD98B1FFF7CDFF80B1FFF7E4FC68B1FFF7C3FF2448D0EDD90AB4EEE00AF1EE10FA01DD012000E000200446204610BD10B5002466
:40AD4000FFF75AFCB0B12CF0F9FC98B1FFF7AFFF80B1FFF7A8FF1748D0EDDA0AB4EEE00AF1EE10FA04D2FFF7BCFC08B1012000E000200446204610BD10B50024FFF73CFCF3
:40AD8000B0B92CF0DBFC98B1FFF791FF80B1FFF78AFF0848D0EDDB0AB4EEE00AF1EE10FA04DDFFF79EFC08B1012000E000200446204610BD30210020940C00209B4890EDF8
:40ADC000030A704710B50024FFF716FCB0B12CF0B5FC98B1FFF76BFF80B1FFF782FC68B1FFF7ECFF9248D0EDD90AB4EEE00AF1EE10FA01DD012000E000200446204610BDBD
:40AE000010B50024FFF7F8FBB0B12CF097FC98B1FFF74DFF80B1FFF764FC68B1FFF7CEFF8348D0EDDA0AB4EEE00AF1EE10FA01D2012000E000200446204610BD10B5002407
:40AE4000FFF7DAFBB0B92CF079FC98B1FFF72FFF80B1FFF746FC68B1FFF7B0FF7448D0EDDB0AB4EEE00AF1EE10FA01DD012000E000200446204610BD70B52DED068B002436
:40AE80002CF05CFC88B3FFF712FF70B3FFF729FC58B3674890EDDC0A10EE101A084639F015FA41EC180BFFF7FEFEF0EE400AFFF785FF30EEC00A10EE105A284639F006FA08
:40AEC00041EC1A0BB0EE4A0AF0EE6A0A35F0D8FDB0EE409AF0EE609A53EC182B51EC190B38F0FCFF02D2012001E001E0002004462046BDEC068B70BD10B52DED028B9FED86
:40AF00004D0AB0EE408A2CF0E5FB28B14A4890ED030AB0EE408A11E02CF0F4FB70B1FFF7C2FEB0EE408AB3EE040AB4EEC08AF1EE10FA03D89FED3F0AB0EE408AB0EE480A32
:40AF4000BDEC028B10BD3D4890EDA40A704710B52DED068BFEF7A1FD20B1FFF7A4FEB0EE408A0CE0324890F84A00032803D1344890ED038A03E0FFF770FBB0EE408A18EE24
:40AF8000100A39F0A3F941EC1A0BB0EE4A0AF0EE6A0A35F075FDB0EE409AF0EE609A9FED290B53EC102B51EC190B38F05DFE03D89FED200AB0EE408AB0EE480ABDEC068BF4
:40AFC00010BD00B50022FFF717FB90B1FEF765FD78B1FFF7B8FFF0EE400AFFF736FB9FED1B1A20EE010AF4EEC00AF1EE10FA00DD0122104600BD00B50022FFF7FDFA90B161
:40B00000FEF74BFD78B1FFF79EFFF0EE400AFFF71CFB9FED0F1A20EE010AF4EEC00AF1EE10FA00D20122104600BD0000EC0C00203021002000000000440D0020F80800205D
:40B040009C0D002000000000000034406666663FCDCCCC3D10B501F004FF292002F080FA2A2002F07DFA0EF022F970B1DFF8F0C300DF044604212FF057F8DFF8E4C300DF82
:40B08000044602212FF050F80DE0DFF8D4C300DF044604212FF065F8DFF8C4C300DF044602212FF05EF810BD10B5EE48C16B01202FF074F8EB48C16B0120DFF8ACC300DF33
:40B0C00010BD10B52DED0C8BB0EE408AE74890ED630AB0EE409AB4EEC98AF1EE10FA02DD01F0A9FE38B9B4EEC98AF1EE10FA2CD201F0A1FE48BBDD4890ED6A0A10EE101A21
:40B10000084639F0E3F841EC1B0B38EE490A10EE101A084639F0DAF841EC1D0BB0EE4D0AF0EE6D0A35F0ACFCB0EE40CAF0EE60CA53EC1B2B51EC1C0B38F0D2FD41EC1A0B32
:40B1400038F088FA08EE900A3BE0B4EEC98AF1EE10FA02DD01F06FFE38B1B4EEC98AF1EE10FA2CD201F067FE48B3C04890ED6B0A10EE101A084639F0A9F841EC1B0B38EE96
:40B18000490A10EE101A084639F0A0F841EC1D0BB0EE4D0AF0EE6D0A35F072FCB0EE40CAF0EE60CA53EC1B2B51EC1C0B38F098FD41EC1A0B38F04EFA08EE900A01E0DFED7E
:40B1C000AC8A9FEDAC0AF4EEC08AF1EE10FA03DD9FEDA80AF0EE408A9FEDA70AF4EEC08AF1EE10FA03D29FEDA40AF0EE408AB0EE680ABDEC0C8B10BD10B52DED028B2EF04C
:40B2000043FE9E490860002001F072F9B0EE408AFFF757FF994880ED030A01F03BFBBDEC028B10BD2821954834F0A5FA01218D4880F82012DFF828C200DF0646012204210B
:40B240002EF02CFFDFF818C200DF0646192202212EF024FFDFF808C200DF064631460120DFF804C200DF03217E4880F8201200BF00224FF6FF710720DFF804C200DF85B226
:40B28000012DF5D0022DF3D1DFF8F8C100DF044604F0040008B101F0D9FB04F0020018B1FFF7AAFFFFF700FF04F001000028DFD0FFF7D0FEDCE710B504466A48D0F81C121C
:40B2C0002046DFF8A4C100DF10BD10B52DED088B664890ED630AD0ED610A30EE600ADFED660A80EE801A11EE104A204638F0EEFF41EC1B0BB0EE4B0AF0EE6B0A35F0C0FBB5
:40B30000B0EE40AAF0EE60AA51EC1A0B38F096F941EC190B38F09EF908EE900A534890ED620AD0ED630A30EE600ADFED520A80EE801A11EE104A204638F0C8FF41EC1A0B7E
:40B34000B0EE4A0AF0EE6A0A35F09AFBB0EE409AF0EE609A51EC190B38F07CF908EE100A002001F066FA414890F8300091280ED03E4890F83000922809D03C4890F830001B
:40B38000712804D0394890F83000B8280CD1374890F8B201032807D19FED3B0AB0EE408AB1EE480AF0EE408AB0EE680A01F0B9FAB0EE480A01F0C9FABDEC088B10BD70B515
:40B3C00005460C4601F0F0F9284600F019FE204600F02EFEFFF779FF64201BF0DCFB0120FFF769FF70BD2548D0ED030AB0EE600A7047224890F82400042801D0012070477E
:40B400000020FCE70220704710B52DED088BB0EE408A18EE100A38F059FF41EC190BFFF7E2FF10EE104A204638F050FF41EC1B0BB0EE4B0AF0EE6B0A35F022FBB0EE40AAF6
:40B44000F0EE60AA53EC192B51EC1A0B38F00CFC03D20120BDEC088B10BD0020FAE7000041350408785200200129040830210020000000000000C8420000C8C2E01C00200C
:40B4800061290408A9280408D051863910B501F0E8FC292002F064F82A2002F061F80DF03FFF70B1DFF828C400DF044604212EF03BFEDFF81CC400DF044602212EF034FE5C
:40B4C0000DE0DFF80CC400DF044604212EF049FEDFF8FCC300DF044602212EF042FE10BD10B5FC48C16B01202EF058FEF948C16B0120DFF8E4C300DF10BDF0EE400AF7480F
:40B50000D0ED631AB0EE611AD0ED611AF4EEC11AF1EE10FA1FD2F4EEC10AF1EE10FA08D2D0ED671A90ED6A2AB0EE610A02EE200A31E0F4EEC10AF1EE10FA09DBE748D0ED90
:40B54000691A90ED6B2AB0EE610A02EE200A22E09FEDE30A1FE0F4EEC10AF1EE10FA09D2DE48D0ED691A90ED6B2AB0EE610A02EE200A10E0F4EEC10AF1EE10FA09DBD74804
:40B58000D0ED671A90ED6A2AB0EE610A02EE200A01E09FEDD30A7047D048B0F9A0037047CE48B0F9A2037047CE49097D31B1012906D0022906D0032906D106E0002006E073
:40B5C000012004E0022002E000BF032000BF00BF704710B52DED028BFFF7E6FF10B9FFF7DFFF01E0FFF7D8FF08EE100A2EF04CFCBD490860002000F07BFFF0EE408AFFF78D
:40B600007CFFB94880ED030A90ED030AF8EEC80A30EE600A80ED030A01F03CF9BDEC028B10BD2C21B04834F0A6F80121A94880F83412DFF89CC200DF0646012204212EF009
:40B640002DFDDFF88CC200DF0646192202212EF025FDDFF87CC200DF064631460120DFF878C200DF03219B4880F8341200BF00224FF6FF710720DFF874C200DF85B2012D17
:40B68000F5D0022DF3D1DFF868C200DF044604F0040008B101F0DAF904F0020018B1FFF798FFFFF71DFF04F001000028DFD0FFF7EDFEDCE710B504468648D0F83012204618
:40B6C000DFF814C200DF10BD8448B0F8900370478248B0F88E0370478048B0F88C03704710B52DED048BFFF7EFFF0146FFF7F4FF081A00EE100AB8EEC00A7848D0ED630ABD
:40B7000090ED611A70EEC10A80EE201AB0EE418AFFF7DEFF0146FFF7D7FF081A00EE100AB8EEC00A6D48D0ED620A90ED631A70EEC10A80EE201AF0EE418AFFF7C5FF00EE5D
:40B74000100AB8EE400A6548D0ED630A08EE600AB0EE409AFFF7B8FF00EE100AB8EE400A5E48D0ED630A08EEE00AF0EE409A002001F05FF8B0EE480A01F0D3F8B0EE680ADF
:40B7800001F0E3F8B0EE490A01F0F3F8B0EE690A01F003F9BDEC048B10BD70B505460C4601F002F8284600F02BFC204600F040FCFFF796FF0120FFF77DFF70BD4A48D0ED8F
:40B7C000030AB0EE600A7047474890F82400042801D0012070470020FCE70220704773B50D46002400BF022269464248006800F563700FF01FFF20B9BDF800003749A1F8E2
:40B800008C0300BF5C2001F0ABFE20467CBD73B50D46002400BF022269463648006800F28E300FF007FF20B9BDF800002B49A1F88E0300BF5D2001F093FE20467CBD31B5CA
:40B84000002400BF022269462A48006800F564700FF0F0FE20B9BDF800002049A1F8900300BF5E2001F07CFE204638BD31B5002400BF022269461F48006800F292300FF03E
:40B88000D9FE20B9BDF800001449A1F8920300BF622001F065FE204638BD1048B0F89203704731B5002400BF022269461148006800F565700FF0BEFE20B9BDF8000007499C
:40B8C000A1F8940300BF682001F04AFE204638BD4135040878520020012904083021002000000000482C0020382A002061290408A9280408FC0300205648B0F894037047EE
:40B9000031B5002400BF012269465348006800F567700FF08FFE20B9BDF800004D4981F89C0300BF692001F01BFE204638BD494890F89C03704731B5002400BF012269461E
:40B940004548006800F29E300FF074FE20B9BDF80000404981F89E0300BF632001F000FE204638BD3B4890F89E03704731B5002400BF022269463848006800F568700FF031
:40B9800059FE20B9BDF900003249A1F8A00300BF6D2001F0E5FD204638BD31B5002400BF022269462C48006800F2A2300FF042FE20B9BDF900002749A1F8A20300BF6C206D
:40B9C00001F0CEFD204638BD10B52DED0C8BB0EE408AFFF779FE044638F032F941EC1A0BFFF772FE00EE100AB8EE401AFFF7E6FE31EE400A10EE104A204638F067FC41ECCF
:40BA00001D0BB0EE4D0AF0EE6D0A35F039F8B0EE40CAF0EE60CA9FED110B53EC102B51EC1C0B38F05DF941EC1B0B53EC1A2B37F0FFFE41EC190B37F00DFE08EE900AF4EE9A
:40BA4000C88AF1EE10FA03D20120BDEC0C8B10BD0020FAE730210020FC030020000000000000594010B52DED028BB0EE408ABE4880ED008A2EF008FABC490860BDEC028BCA
:40BA800010BD10B52DED088BB0EE408A9FEDB80AF0EE408AB3EE040AB0EE40BA18EE100A38F014FC41EC1A0BB0EE4A0AF0EE6A0A34F0E6FFB0EE409AF0EE609A9FEDAD0B17
:40BAC00053EC102B51EC190B38F008FA0ED2B3EE040A38EE400ADFEDA90A80EE201AB3EE040A21EE000AF0EE408A03E09FEDA00AF0EE408AB0EE680ABDEC088B10BD10B50C
:40BB00002DED048B04469FED9A0AB0EE408A9FED980AF0EE408A9A4890F83000922804D0974890F83000932875D1954890F8FF0102280ED0924890F8FF01032809D0904839
:40BB400090F8300092280BD08D4890F83000932806D0864800682EF0BFF9B0F57A7F03D300208849087001E086480470864800682EF0B2F9C8284ED3814890F830001D2878
:40BB80004AD18048007828B1774890ED000AB0EE408A15E07D4800782BF0A4FF00EE100AB8EE400ADFED7A0A30EE600ADFED790A80EE201AB2EE0E0A21EE000AB0EE408AB3
:40BBC000754890ED000A78EE400A744890ED000A9FED731A01EE200A80ED000A062025F0CBFB44B114F07CFBB0EE409AFFF749FFF0EE408A03E001F088FCF0EE408A6948E5
:40BC000090ED000A30EE280A674880ED000A052025F0B2FB2CE049E05A48007828B1524890ED000AB0EE408A15E0584800782BF059FF00EE100AB8EE400AF3EE040A70EEAA
:40BC4000600A9FED541A80EE810AF2EE0E0A20EE200AB0EE408A504890ED000A78EE400A90ED000A9FED4E1A01EE200A80ED000A2EF00AF944490860414890F8FF010228A4
:40BC800004D03F4890F8FF0103280CD13C4890F83000922804D03A4890F83000932802D1042025F069FB072025F066FBBDEC048B10BD394890ED000A704701B500BF012271
:40BCC00069463A48006800F2FF100FF0B3FC20B99DF800002A4981F8FF0100BF08BD224890ED000A70472D4890ED000A70472E4890ED000A70472B4890ED000A7047F0B5B9
:40BD00000546059C0E78022E02D0042E28D113E08F78487867F31F2000EE100AB8EE400ADFED230A30EE600ADFED220A80EE201A1C4E86ED001A14E08F78487867F31F20AD
:40BD400000EE100AB8EE400ADFED190A30EE600ADFED180A80EE201A0F4E86ED001A00E000BF00BFF0BD00000C040020240400200000000000000000000034400000A042FB
:40BD800030210020200400202804002061070020000048420000804518040020100400209A99993E1C04002014040020FC0300200000FB4600007A4488B0016807914168B9
:40BDC000069181680591C1680491016903914169029181690191C169009108B0704700000C48016841F4700101600B4880470B480047FEE7FEE7FEE7FEE7FEE7FEE7FEE7D3
:40BE0000FEE7FEE7FEE7000005480649064A074B7047000088ED00E009E90308AD81000828FC0020C0D9012028FE0020C0D501207047704770471EF0CDB97047000000006C
:40BE40000000000000000000000000000000000000000000000000000000000000000000000000000000000000000000526176656E20496E647573747269657320496E6342
:40BE80000000000000000000000000004175672D31382D32303138000000000032322E342E302E3500000000000000005374656572696E6720436F6E74726F6C20556E69C2
:40BEC0007400000000000000000000003037373031373135323100000000000000000000000000000000000000000000FFFFFFFFFFFFFFFFFFFFFFFFFFFFFFFFFFFFFFFFE3
:40BF0000FFFFFFFFFFFFFFFFFFFFFFFFFFFFFFFFFFFFFFFFFFFFFFFFFFFFFFFFFFFFFFFFFFFFFFFFFFFFFFFFFFFFFFFFFFFFFFFFFFFFFFFFFFFFFFFFFFFFFFFFFFFFFFFF41
:40BF4000FFFFFFFFFFFFFFFFFFFFFFFFFFFFFFFFFFFFFFFFFFFFFFFFFFFFFFFFFFFFFFFFFFFFFFFFFFFFFFFFFFFFFFFFFFFFFFFFFFFFFFFFFFFFFFFFFFFFFFFFFFFFFFFF01
:40BF8000FFFFFFFFFFFFFFFFFFFFFFFFFFFFFFFFFFFFFFFFFFFFFFFFFFFFFFFFFFFFFFFFFFFFFFFFFFFFFFFFFFFFFFFFFFFFFFFFFFFFFFFFFFFFFFFFFFFFFFFFFFFFFFFFC1
:40BFC000FFFFFFFFFFFFFFFFFFFFFFFFFFFFFFFFFFFFFFFFFFFFFFFFFFFFFFFFFFFFFFFFFFFFFFFFFFFFFFFFFFFFFFFF00C00008FFFF030800800008FBBF0008A8C83C8F17
:40C0000001B500BF01226946FE48006800F5D9700FF010FB20B99DF80000FB4981F8B20100BF02201AF0E3FB0120FFF744F908BD01B500BF01226946F248006800F2B31065
:40C040000FF0F8FA20B99DF80000EF4981F8B30100BF02201AF0CBFB0120FFF72CF908BD70B52DED068BB0EE408AF0EE608A04460425E54890F8B201E4490978884206D120
:40C08000E14890F8B301E249097888427ED0DE4890F8B2010C287CD2DFE800F05D213E06595A5B5C073C3D5E00BF9FEDDA0ADA4880ED000A9FEDD70AD84880ED000A9FED5B
:40C0C000D50AD74880ED000A9FEDD20AD54880ED000A0120D4490870D449087059E0B6EE000ACD4880ED000A9FEDD10ACB4880ED000A9FEDC80ACA4880ED000A9FEDC50ADE
:40C10000C84880ED000A0120C74908700020C74908703EE000BF00BF9FEDC60ABE4880ED000A9FEDC50ABD4880ED000A9FEDB90ABB4880ED000A9FEDB70ABA4880ED000A4C
:40C140000120B94908700020B849087021E000BF00BF00BF00BF00BF9FEDAE0AAE4880ED000A9FEDAC0AAD4880ED000A9FEDA90AAB4880ED000A9FEDA70AAA4880ED000A21
:40C180000120A94908700020A84900E002E0087000BF00BFA448007808B900254CE0A3480078012804D1FEF76CFA50B3002543E03CB99A4890ED000AB4EEC08AF1EE10FA7B
:40C1C00009DC012C09D1974890ED000AB4EEC08AF1EE10FA01DD01252EE03CB98E4890ED000AB4EEC08AF1EE10FA09D3012C09D18B4890ED000AB4EEC08AF1EE10FA01D2FA
:40C20000002519E018EE900A38F060F841EC1A0BB0EE4A0AF0EE6A0A34F032FCB0EE409AF0EE609A9FED850B53EC102B51EC190B37F054FE00D203252846BDEC068B70BD49
:40C2400031B52DED020B044600BF042269466D48006800F5C2700FF0EDF920B99DED000A694880ED610A00BF0DF021F810B1FFF72CF808E00DF054F810B1FFF731FA02E00F
:40C2800001201AF0ADFB212025F076F801203EBD31B52DED020B2DED088B044694B300209FED680A19F04CF910EE105A284638F00DF841EC1B0BB0EE4B0AF0EE6B0A34F054
:40C2C000DFFBB0EE40AAF0EE60AA51EC1A0B37F0C1F908EE100A4C4890EDE20A30EE480AF0EE408A90EDE20A30EE080AB0EE409A9DED080AB4EEC90AF1EE10FA03DD8DED27
:40C30000089A09E009E09DED080AB4EEE80AF1EE10FA01D2CDED088A0FE000BF042208A93848006800F562700FF084F920B99DED080A354880EDE20A00BF00BF042208A901
:40C340003048006800F5C6700FF074F920B99DED080A2D4880ED630A00BF0CF0A8FF10B1FEF7B3FF08E00CF0DBFF10B1FFF7B8F902E002201AF034FB212024F0FDFF0120E3
:40C38000BDEC088B3EBD31B52DED020B044600BF042269461B48006800F5C4700FF04AF920B99DED000A184880ED620A00BF0CF07EFF10B1FEF789FF08E00CF0B1FF10B1B4
:40C3C000FFF78EF902E003201AF00AFB212024F0D3FF01203EBD014600200B2955D2DFE801F054494A06474854543B4546009FED161AC0EE010A9FED151A70EE810AFCEE02
:40C40000E00A25E0FC030020302100205800002059000020000000005C0000206000002064000020680000206C0000206D00002066664640CDCCCC3C33339F400000000033
:40C4400000406F4035FA0E3D0000AF4300401C4510EE902A90B21AE05FED040A70EE200AFCEEE00A10EE902A90B210E000BF00BF00BF00BF00BFDFEDFC0A60EE200AFCEE3D
:40C48000E00A10EE902A90B201E0002000BF00BF7047014600200B2926D2DFE801F0251A1B0618192525101617005FED190A80EE201AFDEEC10A10EE902A10B216E0FCEED8
:40C4C000C00A10EE902A10B210E000BF00BF00BF00BF00BFDFEDE40A60EE200AFDEEE00A10EE902A10B201E0002000BF00BF70475FED380AB0EE600A28B9DC49D1ED560ADC
:40C50000B0EE600A06E0012804D1D849D1ED990AB0EE600A704770B52DED0A8BB0EE408A9FEDD30AC8EE000A10EE905AD14890ED610AF0EE408A90ED630AB0EE409A002056
:40C54000FFF7D6FFF0EE409A284637F0BFFE41EC1A0B38EEE90A78EEC90A80EE201A11EE106A304637F0B2FE41EC1C0BB0EE4C0AF0EE6C0A34F084FAB0EE40BAF0EE60BA06
:40C5800053EC1A2B51EC1B0B37F06EFB01D2012000E0002004462046BDEC0A8B70BD70B52DED0A8BB0EE408A9FEDB10AC8EE000A10EE905AAF4890ED620AF0EE408A90EDC5
:40C5C000630AB0EE409A0020FFF792FFF0EE409A284637F07BFE41EC1A0B38EEE90A78EEC90A80EE201A11EE106A304637F06EFE41EC1C0BB0EE4C0AF0EE6C0A34F040FA21
:40C60000B0EE40BAF0EE60BA53EC1A2B51EC1B0B37F02AFB01D2012000E0002004462046BDEC0A8B70BD70B52DED0C8BF0EE408A9FED8F0AC8EE800A10EE904A8D4890ED1B
:40C64000620AF0EE409A90ED610AB0EE40AA90ED630AB0EE408A0020FFF74AFFB0EE409A204637F033FE41EC1B0B39EE480A7AEE480A80EE201A11EE106A304637F026FED7
:40C6800041EC1D0BB0EE4D0AF0EE6D0A34F0F8F9B0EE40CAF0EE60CA53EC1B2B51EC1C0B37F0E2FA24D2204637F010FE41EC1B0B39EE480A79EEC80A80EE201A11EE106A73
:40C6C000304637F003FE41EC1D0BB0EE4D0AF0EE6D0A34F0D5F9B0EE40CAF0EE60CA53EC1B2B51EC1C0B37F0BFFA01D2012000E0002005462846BDEC0C8B70BD5B4890F84D
:40C700005000042801D0012070470020FCE710B50124FFF7F3FF28B95449C86A64212DF0B9FB00B10024204610BD504890F82800042801D0012070470020FCE710B50124E7
:40C74000FFF7F3FF28B94949486864212DF0A2FB00B10024204610BD10B5FFF7EFFF10B1FFF7D5FF08B9022411E0424890ED6A0AB5EEC00AF1EE10FA08D090ED6B0AB5EE1D
:40C78000C00AF1EE10FA01D0012400E00024204610BD18B9354991ED080A04E0012802D1324991ED120A704710B50021324800782FF0C4FB0021314800782FF0BFFB2D48F8
:40C7C00090F8B201032802D0082820D10FE000209FED2B0AFFF734FD00201FEDF20AFFF757FD00209FED270AFFF7CDFD1FE000209FED250AFFF724FD00201FEDFA0AFFF7C3
:40C8000047FD00209FED210AFFF7BDFD0FE00020B6EE000AFFF714FD0020B0EE040AFFF737FD0020B1EE020AFFF7ADFD00BF00BF10BD01B50F4890F8410001280FD000BF20
:40C84000012269461248006800F2B5100EF0F2FE20B99DF80000074981F8B50100BF212024F08AFD08BD000000007A44F40D00200000C84230210020600700205F070020CB
:40C8800090ED24C990ED244900803BC500803B45FC03002010B52DED028B044694ED030AD4ED040A30EE600A84ED060A94ED030A84ED040A2DF0E8FA2060D4E90001401AC5
:40C8C000A06094ED020AB8EE400A5FED190A80EE201AB0EE418A20686060B5EEC08AF1EE10FA1BDD94ED060AC0EE080AC4ED050A0CF012FC48B1D4ED050AB0EE600AC82150
:40C9000004F11C001AF0AFFF08E0D4ED050AB0EE600A042104F11C001AF0A5FFBDEC028B10BD10B52DED020B00BF04226946FA48006800F5D4700EF07DFE20B99DED000A3E
:40C94000F64880ED6A0A00BF1CBD10B52DED020B00BF04226946F048006800F5D6700EF069FE20B99DED000AEC4880ED6B0A00BF1CBD10B52DED020B00BF04226946E64877
:40C98000006800F5CE700EF055FE20B99DED000AE24880ED670A00BF1CBD10B52DED020B00BF04226946DC48006800F5D2700EF041FE20B99DED000AD84880ED690A00BFD2
:40C9C0001CBD19B9D64A82F8280004E0012902D1D34A82F85000704710B52DED088BB0EE408A9FEDD00AF0EE408AB3EE040AB0EE40BA18EE100A37F069FC41EC1A0BB0EE80
:40CA00004A0AF0EE6A0A34F03BF8B0EE409AF0EE609A9FEDC50B53EC102B51EC190B37F05DFA0AD21FED6E0AC8EE000A9FEDC00A20EE800AF0EE408A03E09FEDBA0AF0EE2D
:40CA4000408AB0EE680ABDEC088B10BD10B52DED028BB34890F86D02012816D0AF4890F84B00AF4981F86C02084690F86C1254301AF0E8FEAA4890F86C1200F5B0701AF0DE
:40CA8000E1FE0120A64981F86D02A44890F8B2010B287DD2DFE800F0FE06162AFDFCFBFA2B3BB400A34800782BF01CF800EE100AB8EE400ADFEDA00A20EE200A984880ED6E
:40CAC000040A03E19B4800782BF00CF800EE100AB8EE400ADFED980A20EE200ADFED970A80EE201A8E4880ED041AEFE000BF914800782FF090F900EE100AB8EEC00A8848E7
:40CB0000D0ED000A30EE200A80ED040ADEE00AF0B7FF10B90AF069FE18B3FDF75BFDB0EE408AFFF759FF864880ED000A854800682DF0D2F900EE100AB8EE400A5FEDB60AA0
:40CB400080EE201A804880ED001A7D4890ED000A7D48D0ED000A20EE200A7C4880ED000A20E0744800782FF056F900EE100AB8EEC00A7748D0ED000A30EE600A5FEDC60A2F
:40CB800080EE201A714880ED001A6A48007800E094E02FF040F900EE100AB8EEC00A6C4880ED000A2DF070F9664908605C4890ED040A6648D0ED000A30EE200AF6EE000A9D
:40CBC000B4EEE00AF1EE10FA19DD554890ED040A5E48D0ED000A30EE200AF1EE020AB4EEE00AF1EE10FA0AD24D4890ED040A5748D0ED000A30EE200A494880ED040A65E092
:40CC0000FFF779F8B2EE041AC0EE010AB0EE040A30EE800A424880ED040A464800782FF0FAF800EE100AB8EEC00A4948D0ED000A30EE600A5FEDF40A80EE201A404880ED67
:40CC4000001A3C4800782FF0E6F800EE100AB8EEC00A3F4880ED000A3A4800682DF03CF900EE100AB8EE400ADFED3A0A80EE201A354880ED001A324890ED000A3248D0ED03
:40CC8000000A20EE200AF1EE040A04E018E00FE008E006E013E020EE200A2F4880ED000A14E000BF9FED1F0A1D4880ED040A0DE09FED1C0A1A4880ED040A07E000BF00BF6A
:40CCC0009FED180A164880ED040A00BF00BF144890F86C12D0ED040AB0EE600A54301AF05DFD0F48001DFFF7D5FD0D4890ED081AF0EE410A90ED041AB0EE410A0020FFF71F
:40CD0000AFF904460021FFF75CFE044890F8B3010B2866D222E00000FC03002030210020F40D0020000000000000000000003440713DAA3F600700203333533A0CAC233F4B
:40CD400070000020800000207C000020780000207400002000007A4454000020DFE800F0420616312A2B3B3532333400FE4800782AF0B8FE00EE100AB8EE400A5FED120AF7
:40CD800020EE200AF94880ED0E0A31E0F64800782AF0A8FE00EE100AB8EE400A5FED1A0A20EE200A5FED1B0A80EE201AEF4880ED0E1A1DE000BF1FED250AEC4880ED0E0AB9
:40CDC00016E000BF00BF00BF00BF1FED2A0AE74880ED0E0A0CE01FED2D0AE44880ED0E0A06E000BF1FED310AE04880ED0E0A00BF00BFDE4890F86C12D0ED0E0AB0EE600A4D
:40CE000000F5B0701AF0CAFCD8482C30FFF742FDD64890ED121AF0EE410A90ED0E1AB0EE410A0120FFF71CF904460121FFF7C9FDBDEC028B10BDCE4890ED610AD0ED630A5F
:40CE400030EE600AB5EEC00AF1EE10FA01DD012070470020FCE7B0EE040AC44880ED040A704730B589B02AF060FC40B10021084619F0A3FD0121002019F09FFD2AE0BC489F
:40CE800090F8B201032804D0B94890F8B201082808D10021032019F090FD0121032019F08CFD17E0B24890F8B20109280AD10021032019F082FD0121032019F07EFDFFF77F
:40CEC000CAFF07E00021032019F077FD0121002019F073FDA64890F8B25190F8B3410B2D7ED2DFE805F08C06182A8E8F608D2B2C2D000020009001900290034603229D4944
:40CF00000390084600782AF0FEFC0321994800782BF0A7F888E000200090019002900346032294490390084600782AF0ECFC0021904800782BF095F876E000BF00BF00BFC0
:40CF400000200090019002900346022289490390084600782AF0D7FC0221864800782BF080F82AF0B7FB68B183485FED920A9FED830A04230022824900907E4800782EF0AC
:40CF800051FC0FE02AF0BEFB60B17B485FED9B0A9FED7A0A0423002219070090754800782EF040FC40E000200090019002900346022270490390084600782AF0A4FC0621B2
:40CFC0006C4800782BF04DF8002000900190022314220121029004A82EF03CFD04A800E00DE05FEDB00A9FED670A032300224FF0804100905F4800782EF014FC14E000BFFE
:40D0000000BF00BF00200090019002900346032258490390084600782AF075FC0121554800782BF01EF800BF00BF0B2C7ED2DFE804F08B06182A8D8E608C2B2C2D00002006
:40D040000090019002900346032247490390084600782AF058FC0321434800782BF001F89AE00020009001900290034603223E490390084600782AF046FC00213A480078EB
:40D080002AF0EFFF88E000BF00BF00BF00200090019002900346022233490390084600782AF031FC0221304800782AF0DAFF2AF011FB68B130485FEDE50A9FED300A042382
:40D0C00001222F490090284800782EF0ABFB0FE02AF018FB60B128485FEDEE0A9FED270A04230122910700901F4800782EF09AFB52E00020009001900290034602221A49E2
:40D100000390084600782AF0FEFB0621164800782AF0A7FF002000900190034614220121029004A82EF096FC04A800E00CE0DFED160A9FED120A02230122910700900A4828
:40D1400000782EF06FFB27E000BF00BF00BF00200090019002900346032203490390084600782AF0D0FB11E05F070020F40D0020302100206007002080EC0020809FD54A46
:40D1800000040140A037A04C000000000121E14800782AF066FF00BF00BF09B030BD10B5DD4988684FF496712CF074FE10BDDB4890ED000A704710B52DED048B19F0B0FBFE
:40D1C00010EE104A204637F081F841EC190BB0EE490AF0EE690A33F053FCB0EE408AF0EE608A9FEDCF0B53EC102B51EC180B36F03BFD03D20120BDEC048B10BD0020FAE702
:40D20000C94991F84110012901D1012007E0C64991F8B51109B1012100E000210846704710B52DED068BB0EE408AC048007838B91FED2B0ABE4880ED000A0120BB4908701A
:40D24000FFF7DEFF00287ED0FFF7B5FF18B90AF017FC002877D0FFF7AAFF10EE104A204637F034F841EC1A0BB0EE4A0AF0EE6A0A33F006FCB0EE409AF0EE609A9FEDAD0B6F
:40D2800053EC102B51EC190B36F0EEFC5BD2FFF786FF002857D123F01DFBDFEDA80AB4EEE00AF1EE10FA4EDBFFF756FA01284AD19D4890F83000912845D09B4890F83000B4
:40D2C000922840D0984890F8300071283BD0964890F83000B82836D0934890F8B2010B282AD2DFE800F029121306141529290708160000BF00BF8E4890ED000ADFED900A7B
:40D3000008EE200A80ED000A1CE000BF00BF00BF00BF8548D0ED630A9FED891A48EE410AB0EE600A0120FEF7B3FF1FED690A804880ED000A06E006E01FED6D0A7C4880EDA9
:40D34000000A00BF00BFBDEC068B10BD784890F8280008B9012070470020FCE7744890F82800012800D170470020FCE7704890F82800032801D1012070470020FCE76C48FE
:40D3800090F8500008B9012070470020FCE7684890F85000012800D170470020FCE7644890F85000032801D1012070470020FCE700B50021FFF7CAFF08B13D2103E0FFF7DC
:40D3C000CDFF00B13C21084600BD00B50021FFF7CDFF08B1082117E0FFF7B8FF08B1072112E0FFF7BBFF08B106210DE0FFF7D7FF08B10B2108E0FFF7A9FF08B10A2103E0DC
:40D40000FFF7ACFF00B10921084600BD10B519F0AAFB0446204610BD10B52DED028B0BF046FF20B1FDF7DFFFB0EE408A16E019F073FA3D48D0ED640A30EE600ADFED410A03
:40D4400020EE200AD0ED650A90ED641A70EEC10A80EE201A9FED3C0A31EE008AB0EE480ABDEC028B10BD01B59DF80000202801DD2020009000BF01226946344800684B30DD
:40D480000EF0D8F820B99DF80000274981F84B0000BF0020264981F86D0208BD10B54FF41C71234832F067F910BD29490870704727480078704710B52DED028BB0EE408A9F
:40D4C0002448007830B9154800210160416001202049087023F0FAF9F0EE408AF0EE680AB0EE480A19F00FF91B4880ED000A28210A48194A92ED000A1AF0B5F9BDEC028B8F
:40D5000010BD154890ED000A7047144890ED000A704700005F070020AC5500204C000020000000A046DF913F3021002084000020F40D0020000000A046DF813F2FDDE43E58
:40D540000AD7A33B000048430000C8C2FC0300204400002085000020480000205400002010B50446204625F0BBFA10BD07B586B000200490002108980170069800786F2842
:40D5800081F0AF82DFE810F06F007100ED000D013B01AD0AB10050075B0766076901CF01E1014702BC0211036603B303080470045D048200BD042F059D05E3053206B00637
:40D5C0000D09CA0671079B097D07C307D20710081E082C0872087E088E089808A808AD0AAD0AAD0AB808C908E308890795079F07B707AB07AD0AAD0AAD0AAD0AAD0AAD0A7D
:40D60000AD0AAD0AAD0AAD0AAD0AD404AD0AAD0AAD0A1109390956097E09AD0AAD0AAD0AAD0AAD0AAD0AAD0AAD0AAD0AAD0AAD0AAD0AAD0AAD0AAD0AAD0AAD0AAD0AAD0A83
:40D64000AB09DC090D0AAD0AAD0AAD0A1F0A670AAD0AAD0AAD0AAD0A310A430AAD0A550A790A8B0A9D0A01F040BAF94890F841000390069890ED010ABCEEC00A10EE100AC8
:40D68000C0B20290039919F098F9ECE70698007A032803D006210898017025E0069890ED010AF7EE000AB4EE600AF1EE10FA02D117F08BFA18E0069890ED010AF0EE000A9B
:40D6C000B4EE600AF1EE10FA02D117F066FA0BE0069890ED010AF0EE080AB4EE600AF1EE10FA01D117F05DF8BDE70698007A032809D1069890ED010A8DED030A9DED030AD2
:40D7000010F006F92AE00698007A012811D1D048B0F8BE110A22079802FB001000EE100AB8EEC00A8DED030A9DED030A10F0F0F814E00698007A022810D1C548B0F8BE113D
:40D740000A22079802FB101000EE100AB8EEC00A8DED030A9DED030A10F0DAF80120049081E70AF08DF9C0B90698007A032811D1069890ED010A8DED030A9DED030A0BF0DF
:40D78000AAF9B448D0F81801014603908020DFF8C8C200DF0120049002E001210898017061E716F071FB30BB0698007A03281ED1069890ED010ABCEEC00A10EE100A80B2AA
:40D7C00003900BF066F90BF0E4F880B90821A348DFF88CC200DF012809D0A248406840F00100A04948609D48DFF87CC200DF182023F0C2FD02E001210898017033E716F0A6
:40D8000043FB30BB0BF0C5F818B30698007A03281BD1069890ED010ABCEEC00A10EE100AC0B203900BF00FF908218C48DFF830C200DF012809D08B48406840F0010089492E
:40D8400048608648DFF820C200DF182023F094FD02E001210898017005E70698007A032817D17B4890F842000390794890F841000290069890ED010ABCEEC00A10EE100AA4
:40D88000C0B20190DDE9021212F088FD0899087046E00698007A01281FD16D4890F841105C3000EB41006A4991F84210415C0122079802FB0010C0B20190654890F84200DA
:40D8C0000390634890F8410002900146039A019812F064FD0899087022E00698007A02281ED15B4890F841105C3000EB4100584991F84210415C0122079802FB1010C0B2C5
:40D900000190534890F842000390514890F8410002900146039A019812F040FD08990870012004909FE60698007A03280CD1069890ED010ABCEEC00A10EE100AC0B2039084
:40D9400012F068FD089908708DE60698007A032817D13F4890F8420003903D4890F841000290069890ED010ABCEEC00A10EE100AC0B20190DDE9021212F08CFD0899087092
:40D9800046E00698007A01281FD1314890F84110603000EB41002E4991F84210415C0122079802FB0010C0B20190294890F842000390274890F8410002900146039A01982C
:40D9C00012F068FD0899087022E00698007A02281ED11F4890F84110603000EB41001C4991F84210415C0122079802FB1010C0B20190174890F842000390154890F84100D7
:40DA000002900146039A019812F044FD089908700120049027E60698007A032826D10C4890F8420003900A4890F841000290069890ED010ABCEEC00A10EE100AC0B201906C
:40DA4000DDE9021212F063FD0899087055E0000030210020785200200129040858320020C92D040868320020E52C04080698007A01281FD1FB4890F84110643000EB4100FB
:40DA8000F84991F84210415C0122079802FB0010C0B20190F34890F842000390F14890F8410002900146039A019812F030FD0899087022E00698007A02281ED1E94890F8FE
:40DAC0004110643000EB4100E64991F84210415C0122079802FB1010C0B20190E14890F842000390DF4890F8410002900146039A019812F00CFD0899087001200490B2E597
:40DB00000698007A032810D1D64890F842000390069890ED010A8DED020A03989DED020A12F053FE089908703CE00698007A01281AD1CC4890F842107C3000EB8100D0EDF2
:40DB4000000A9DED070AB8EEC00A30EEC00A8DED020AC44890F8420003909DED020A12F034FE089908701DE00698007A022819D1BC4890F842107C3000EB8100D0ED000AF0
:40DB80009DED070AB8EEC00A30EE800A8DED020AB44890F8420003909DED020A12F015FE08990870012004905DE50698007A032810D1AC4890F842000390069890ED010A7D
:40DBC0008DED020A03989DED020A12F044FD089908703CE00698007A01281AD1A14890F842106C3000EB8100D0ED000A9DED070AB8EEC00A30EEC00A8DED020A994890F856
:40DC0000420003909DED020A12F025FD089908701DE00698007A022819D1924890F842106C3000EB8100D0ED000A9DED070AB8EEC00A30EE800A8DED020A8A4890F84200BB
:40DC400003909DED020A12F006FD089908700120049008E50698007A032812D1814890F842000390069890ED010ABCEEC00A10EE100AC0B20290039912F087FC089908707F
:40DC800032E00698007A012815D1764890F842106830415C0122079802FB0010C0B20290704890F8420001460390029812F06DFC0899087018E00698007A022814D1694841
:40DCC00090F842106830415C0122079802FB1010C0B20290634890F8420001460390029812F053FC0899087001200490BBE40698007A032810D15B4890F8420003900698C9
:40DD000090ED010A8DED020A03989DED020A12F0BAFD089908703CE00698007A01281AD1504890F84210843000EB8100D0ED000A9DED070AB8EEC00A30EE800A8DED020AF8
:40DD4000484890F8420003909DED020A12F09BFD089908701DE00698007A022819D1414890F84210843000EB8100D0ED000A9DED070AB8EEC00A30EEC00A8DED020A394800
:40DD800090F8420003909DED020A12F07CFD089908700120049066E40698007A032810D1304890F842000390069890ED010A8DED020A03989DED020A12F0ABFC0899087045
:40DDC0003CE00698007A01281AD1264890F84210743000EB8100D0ED000A9DED070AB8EEC00A30EE800A8DED020A1E4890F8420003909DED020A12F08CFC089908701DE08A
:40DE00000698007A022819D1164890F84210743000EB8100D0ED000A9DED070AB8EEC00A30EEC00A8DED020A0E4890F8420003909DED020A12F06DFC0899087001200490AC
:40DE400011E40698007A03280AD1069890ED010ABCEEC00A10EE100AC0B20390FCF797FA13E40000302100200698007A032812D1F74890F842000390069890ED010ABCEE5A
:40DE8000C00A10EE100AC0B20290039912F0B0FB0899087032E00698007A012815D1EC4890F842106A30415C0122079802FB0010C0B20290E64890F842000146039002985D
:40DEC00012F096FB0899087018E00698007A022814D1DF4890F842106A30415C0122079802FB1010C0B20290D94890F8420001460390029812F07CFB089908700120049096
:40DF00002EE40698007A032803D00621089801700DE0069890ED010A8DED030A9DED030A0A2009F02BFC10B901210898017017E40698007A032814D1069890ED010ABCEE17
:40DF4000C00A10EE100A80B200EE100AB8EE400A8DED030A9DED030A0FF0DAFC089908703EE00698007A01281BD110F092FAF0EE400AB748B0F8BE0100EE100AB8EE401A1C
:40DF80009DED070AF8EE401AB0EE410A00EEA10A8DED030A9DED030A0FF0BAFC089908701EE00698007A02281AD110F072FAF0EE400AA748B0F8BE0100EE100AB8EE401AFB
:40DFC0009DED070AF8EE401AB0EE410A00EEE10A8DED030A9DED030A0FF09AFC08990870012004900AE40698007A032815D1984890F842000390964890F8410002900698D8
:40E0000090ED010A8DED010ADDE902019DED010A12F073F90899087050E00698007A012824D18B4890F842000290894890F841000190029910F01AFBDDED070AF8EE600A53
:40E040009FED841A01EE200A8DED030A804890F8420002907E4890F84100019002999DED030A12F04AF90899087027E00698007A022823D1764890F842000290744890F867
:40E0800041000190029910F0F1FADDED070AF8EE600A9FED701A01EE600A8DED030A6C4890F8420002906A4890F84100019002999DED030A12F021F90899087001200490AF
:40E0C00030E40698007A03280BD1069890ED010A8DED030A9DED030A12F06FFC0899087032E00698007A012815D15948D0ED7E0A9DED070AB8EE401ADFED571AB0EE600A24
:40E1000001EE810A8DED030A9DED030A12F055FC0899087018E00698007A022814D14C48D0ED7E0A9DED070AB8EE401ADFED4A1AB0EE600A01EEC10A8DED030A9DED030A38
:40E1400012F03BFC089908700120049062E40698007A032814D1069890ED010ABCEEC00A10EE100A80B200EE100AB8EE400A8DED030A9DED030AFCF727F90899087032E0F2
:40E180000698007A012815D13148D0ED280A079800EB8000400000EE100AB8EEC00A30EE800A8DED030A9DED030AFCF70DF90899087018E00698007A022814D12448D0EDEE
:40E1C000280A079800EB8000400000EE100AB8EEC00A30EEC00A8DED030A9DED030AFCF7F3F8089908700120049039E20698007A032835D1069890ED010ADFED180AB4EE5F
:40E20000E00AF1EE10FA06DD022108980170642006F07CFB62E0069890ED010AF2EE040AB4EEE00AF1EE10FA06D20321089801700A2006F06BFB51E0069890ED010ABCEEA4
:40E24000C00A10EE100AC0B2039006F05FFB45E0302100200AD7233CCDCCCC3D0000C8420698007A01281BD1FE4890F8401007984000C0F1650081420BDAFA4890F84010E3
:40E280000222079802FB0010C0B2039006F03EFB24E0022108980170642006F037FB1DE00698007A022819D1EE4890F8401007984000093081420BDDEA4890F8401002224E
:40E2C000079802FB1010C0B2039006F01FFB05E00321089801700A2006F018FB1A20FFF73FF901200490BBE10698007A032803D006210898017010E0069890ED010ABCEE39
:40E30000C00A10EE100AC0B21FED2C0A039009F035FA10B9012108980170E6E30698007A032803D00621089801707CE0069890ED010AF8EE000AB4EE600AF1EE10FA13D12E
:40E34000C84890F842107C3000EB810090ED000A8DED030A9DED030A082009F00FFA00BB0121089801705EE0069890ED010AFFEE000AB4EE600AF1EE10FA13D1B94890F821
:40E3800042106C3000EB810090ED000A8DED030A9DED030A082009F0F1F910B901210898017040E0069890ED010AF7EE000AB4EE600AF1EE10FA13D1AA4890F842107430D9
:40E3C00000EB810090ED000A8DED030A9DED030A082009F0D3F900BB01210898017022E0069890ED010AF0EE000AB4EE600AF1EE10FA13D19B4890F84210843000EB81006B
:40E4000090ED000A8DED030A9DED030A082009F0B5F910B901210898017004E09FED920A002009F0ABF960E30020FEF761F88DED030A00209DED030AFDF702FF55E3002067
:40E44000FEF756F88DED030A00209DED030AFDF71FFF4AE30020FEF74BF88DED030A00209DED030AFDF78FFF3FE3069890ED010ABCEEC00A10EE100AC0B203900FF05FFE8F
:40E4800033E3069890ED010ABCEEC00A10EE100AC0B20390FEF7CDF927E3069890ED010ABCEEC00A10EE100AC0B2039012F0E2FB1BE3069890ED010A8DED030A9DED030AF2
:40E4C00012F0EDFB11E3069890ED010ABCEEC00A10EE100AC0B2039013F026F905E3069890ED010ABCEEC00A10EE100A80B2039012F0FEFEF9E2069890ED010ABCEEC00A93
:40E5000010EE100A80B2039012F007FFEDE2069890ED010ABCEEC00A10EE100AC0B2039011F0B5F82120FFF71BF8DEE20698007A032803D006210898017034E0069890ED3B
:40E54000010AF7EE000AB4EE600AF1EE10FA0ED10AF0E2FD28B1B7EE000A112009F00EF921E0B7EE000A072009F008F91BE0069890ED010AF0EE000AB4EE600AF1EE10FA6C
:40E5800005D19FED390A002009F0F8F80BE0069890ED010AF0EE080AB4EE600AF1EE10FA01D100F08BFCA0E2069890ED010ABCEEC00A10EE100A80B201460390022018F004
:40E5C00025F892E2069890ED010ABCEEC00A10EE100A80B201460390012018F017F884E20698007A03283BD1069890ED010AB5EEC00AF1EE10FA0BD11A4890F842000390C8
:40E60000184890F84100029003990AF03BFC27E0069890ED010AF7EE000AB4EE600AF1EE10FA07D10F4890F84200012103900AF092FB15E0069890ED010AF0EE080AB4EE5F
:40E64000600AF1EE10FA0BD1064890F842000390044890F841000122029003990AF0FAFA43E200003021002000000000069890ED010ABCEEC00A10EE100AC0B203900AF025
:40E68000BBFA32E20698007A03280AD1069890ED010ABCEEC00A10EE100AC0B20390FBF7B8FF22E215F0F0FB28B90698007A032801D10AF042FA18E20698007A03280AD1DB
:40E6C000069890ED010ABCEEC00A10EE100AC0B20390FDF795FC08E20698007A03280AD1069890ED010ABCEEC00A10EE100AC0B20390FDF79DFCF8E10698007A03280BD19A
:40E70000069890ED010ABCEEC00A10EE100AC0B20121039012F016FEE7E10698007A032814D1069890ED010ADFEDFE0AB4EE600AF1EE10FA0AD10EF096F801200DF038FF4F
:40E740000021F94801720020F8490870CDE10698007A03280BD1069890ED010ABDEEC00A10EE100A00B20390FAF77EF918E00698007A012808D1EE48B0F8AA00401C00B216
:40E780000390FAF771F90BE00698007A022807D1E748B0F8AA00401E00B20390FAF764F9A3E11C20FEF7DCFE9FE10698007A03281AD1DF4890F842106C3000EB810090ED31
:40E7C000000A8DED050A9DED050AB5EEC00AF1EE10FA03D19FEDD70A8DED050A9DED050A082008F0CBFF07E00698007A20B91FED620A082008F0C2FF77E10698007A03287E
:40E800000FD1CB4890F842107C3000EB810090ED000A8DED030A9DED030A082008F0AEFF07E00698007A20B91FED710A082008F0A5FF5AE10698007A03281AD1BC4890F869
:40E840004210743000EB810090ED000A8DED050A9DED050AB5EEC00AF1EE10FA03D19FEDB60A8DED050A9DED050A082008F086FF07E00698007A20B91FED850A082008F0BD
:40E880007DFF32E10698007A03280FD1A84890F84210843000EB810090ED000A8DED030A9DED030A082008F069FF07E00698007A20B91FED930A082008F060FF15E10698FB
:40E8C000007A03280AD1069890ED010ABCEEC00A10EE100AC0B203900AF06FF905E10698007A03280ED1069890ED010ABCEEC00A10EE100A80B201210390FCF770FF0899DB
:40E9000008701CE00698007A01280AD1FCF7E4FE401C80B201210390FCF761FF089908700DE00698007A022809D1FCF7D5FE401E80B201210390FCF752FF08990870D4E09E
:40E940000698007A03280ED1069890ED010ABCEEC00A10EE100A80B201210390FCF757FF089908701CE00698007A01280AD1FCF7AFFE401C80B201210390FCF748FF0899A4
:40E9800008700DE00698007A022809D1FCF7A0FE401E80B201210390FCF739FF08990870A3E00698007A03280CD1069890ED010ABCEEC00A10EE100A80B20390FCF73FFF71
:40E9C0000899087091E00698007A03280CD1069890ED010ABCEEC00A10EE100A80B20390FCF744FF089908707FE00698007A03280CD1069890ED010ABCEEC00A10EE100A76
:40EA000080B20390FCF74DFF089908706DE00698007A03280CD1069890ED010ABCEEC00A10EE100A80B20390FCF76AFF089908705BE00698007A03280CD1069890ED010ADF
:40EA4000BCEEC00A10EE100AC0B2039018F0A3F80899087049E00698007A03280CD1069890ED010ABCEEC00A10EE100A80B20390FCF761FF0899087037E00698007A0328C3
:40EA80000CD1069890ED010ABDEEC00A10EE100A00B20390FCF781FF0899087025E00698007A03280CD1069890ED010ABDEEC00A10EE100A00B20390FCF758FF0899087075
:40EAC00013E00698007A03280AD1069890ED010ABCEEC00A10EE100AC0B20390FDF7EDF803E007210898017000BF00BF049809B000BD86B04FF6FF7438211048DFF840C053
:40EB000000DF02210F4880F808110C2284210E4833F0A0FD002879D103210A4880F8081100BF13E000007E43683200204805002030210020CDCCCCBDCDCCCC3DFC1000208E
:40EB4000892A04087852002078100020224605A98748DFF820C200DF012858D000208DF800008DF80D0001208DF80C0000208DF80E0005980078002839D004AA0121059827
:40EB8000FEF7F4FC05469DF8100068B100250599087824F013FB06460598837A427A9DF81010304624F010FB08F06AFF08B1002504E00598007A032800D100250DB39DF866
:40EBC0000D00F0B90598007AD8B1059A07CA8DE8070001208DF80D008DF80C004FF47A649DF80E00401CC0B28DF80E0009E008F0FCFD30B16048D0F890110120DFF87CC169
:40EC000000DF5F480599F9F77BFB8AE747E09DF80000002885DD9DF80E0000283CDD9DF80E00032803D102208DF80C000EE09DF80E00052803D106208DF80C0006E09DF896
:40EC40000E00072802D110208DF80C009DF80E00FF2805DA9DF80E00401CC0B28DF80E009DF80C1004AA6846FEF780FC9DF8100078B100208DF80E000599087824F09EFA4D
:40EC800006460598837A427A9DF81010304624F09BFA4FF4FA6444E74FF6FF7441E70521354880F808110020DFF8D8C000DF00BFFEE72DE9F0472DED028B0546B0EE408A45
:40ECC0000E46174698464FF001092948DFF8B8C000DFD0B900BF284890F8090140F00201254880F80911B0F814014FF6FF71884207DA2148B0F81401401C81B21E48A0F851
:40ED0000141100BF4FF000092CE01D48F9F7E8FA04466CB1257084ED018A2672677284F80A800A2221461248DFF860C000DF19E000BF114890F8090140F004010E4880F88C
:40ED40000911B0F814014FF6FF71884207DA0A48B0F81401401C81B20748A0F8141100BF4FF000094846BDEC028BBDE8F0870000FC100020192C040878520020012904082E
:40ED80007810002085330408812A0408752B040831B52DED020B0446FE4890EDD40ADDED000AB4EEE00AF1EE10FA00D3ACB100BF04226946F848006800F554700CF03AFCEC
:40EDC00020B99DED000AF34880EDD40A00BFF348C16B0220DFF8C8C300DF3EBD31B52DED020B0446EB4890EDD30ADDED000AB4EEE00AF1EE10FA00DCACB100BF04226946A2
:40EE0000E548006800F553700CF014FC20B99DED000AE04880EDD30A00BFE048C16B0220DFF87CC300DF3EBD31B52DED020B0446D84890ED2F0ADDED000AB4EEE00AF1EE09
:40EE400010FA00D3A4B100BF04226946D2480068BC300CF0EFFB20B99DED000ACD4880ED2F0A00BFCD48C16B0220DFF834C300DF3EBD31B52DED020B0446C64890ED2E0A6C
:40EE8000DDED000AB4EEE00AF1EE10FA00DCA4B100BF04226946C0480068B8300CF0CAFB20B99DED000ABB4880ED2E0A00BFBB48C16B0220DFF8E8C200DF3EBD10B54FF4A3
:40EEC000F671B84830F057FCB24890F82800B54981F8E0012AF0D8FFB2498860012081F8DC01002081F8DD019FEDAF0A084680ED500A002007F07DF901209FEDAB0AFFF735
:40EF0000B8FF01209FEDA80AFFF78EFF01209FEDA60AFFF763FF01209FEDA30AFFF738FF10BD10B517F055FEA04880ED000A90ED000AF2EE000A20EE200ADFED9D0A80EE27
:40EF4000201A9C4880ED001A984890ED000AF0EE080A20EE200ADFED960A80EE201A964880ED001A914890ED000AF3EE010A20EE200ADFED8F0A80EE201A904880ED001AF4
:40EF800010BD10B5002428F0A5FB40B38C4800680078012800D128E0894800680078022801D1142421E0864800680078052801D128241AE0824800680078032801D13C245A
:40EFC00013E07F4800680078062801D150240CE07B4800680078082807D1642405E028F091FB10B16F4890F8E141204610BD10B56C4890F8DD0173490978884203D0FFF757
:40F00000C0FF7149087010BD70B52DED028B044614F03AFF00287DD1002596E05D48C03000EB8400D0ED000AB0EE600A284611F000FD5848C03000EB8400D0ED000AB0EE0B
:40F04000600A284611F007FB5248C83000EB8400D0ED000AB0EE600A284611F00EFD4D48C83000EB8400D0ED000AB0EE600A284611F04FFB4748D03000EB8400D0ED000A22
:40F08000B0EE600A284611F01CFD4248D03000EB8400D0ED000AB0EE600A284611F095FB3C48D83000EB8400D0ED000AB0EE600A284611F02AFD3748D83000EB8400D0EDE6
:40F0C000000AB0EE600A284611F0DDFB3149E031085D294611F03DFD2E49E231085D294611F055FD28F0F6FA08B32A49E0310A5D891C095D501800EBD071491000EE101AAE
:40F10000B8EEC00AB0EE408ABCEEC80A10EE101AC8B200E01DE0214611F037FABCEEC80A10EE101AC8B2214611F062FA0BE01949E031085D214611F028FA1649E231085D5D
:40F14000214611F055FA681CC5B2022DFFF666AFAFE01048C03000EB8400D0ED000AB0EE600A204611F065FC0A48C03000EB8400D0ED000AB0EE600A204611F06CFA05482D
:40F18000C83000EB8400D0ED000AB0EE600A20461CE0000030210020FC03002078520020012904083811002000000000700300200000C84274030020780300207C03002030
:40F1C00048030020800300206E03002011F055FCFE4800EB8400D0ED000AB0EE600A204611F097FAF948083000EB8400D0ED000AB0EE600A204611F064FCF448083000EBC5
:40F200008400D0ED000AB0EE600A204611F0DDFAEE48103000EB8400D0ED000AB0EE600A204611F072FCE948103000EB8400D0ED000AB0EE600A204611F025FBE349183109
:40F24000085D214611F085FCE0491A31085D214611F09DFC28F03EFAF8B1DC4918310A5D891C095D501800EBD071491000EE101AB8EEC00AB0EE408ABCEEC80A10EE101A0C
:40F28000C8B2214611F081F9BCEEC80A10EE101AC8B2214611F0ACF90BE0CC491831085D214611F072F9C9491A31085D214611F09FF9BDEC028B70BD01B500BF01226946DA
:40F2C000C348006800F5E9700CF0B4F928B99DF80000BE49C83981F8D20100BF08BD10B5032006F086FF1FED500A002008F046FA0120FFF7E1FFB549C83991F84200FFF77E
:40F3000083FE1C2022F038F810BD01B5B8B000203590349033903290319030902F902E901FED5F0A389880ED530A1FED610A389880ED560A1FED640A389880ED540A1FED73
:40F34000660A389880ED580A1FED690A389880ED550A1FED6B0A389880ED590A01203790FEE3379834F06CFC9FED9A0B53EC102BCDE926019DED260B51EC100B34F058FA0D
:40F38000CDE92C0137983690389890ED6A0B8DED200B9DED2C0B53EC102B9DED200B51EC100B34F09DFCCDE92401389890ED680B8DED1A0B9DED2C0B53EC102B9DED1A0B45
:40F3C00051EC100B34F08CFCCDE91C019DED2C0B53EC102B9DED1C0B51EC100B34F080FCCDE92001389890ED660B8DED140B9DED2C0B53EC102B9DED140B51EC100B34F0C4
:40F400006FFCCDE916019DED2C0B53EC102B9DED160B51EC100B34F063FCCDE918019DED2C0B53EC102B9DED180B51EC100B34F057FCCDE91C01389890ED640B8DED0E0B2B
:40F440009DED2C0B53EC102B9DED0E0B51EC100B34F046FCCDE910019DED2C0B53EC102B9DED100B51EC100B34F03AFCCDE912019DED2C0B53EC102B9DED120B51EC100B94
:40F4800034F02EFCCDE914019DED2C0B53EC102B9DED140B51EC100B34F022FCCDE91801389890ED620B8DED080B9DED2C0B53EC102B9DED080B51EC100B34F011FCCDE988
:40F4C0000A019DED2C0B53EC102B9DED0A0B51EC100B34F005FCCDE90C019DED2C0B53EC102B9DED0C0B51EC100B34F0F9FBCDE90E019DED2C0B53EC102B9DED0E0B51ECBB
:40F50000100B34F0EDFBCDE910019DED2C0B53EC102B9DED100B51EC100B34F0E1FBCDE91401389890ED600B8DED020B9DED2C0B53EC102B9DED020B51EC100B34F0D0FB82
:40F54000CDE904019DED2C0B53EC102B9DED040B51EC100B34F0C4FBCDE906019DED2C0B53EC102B9DED060B51EC100B34F0B8FBCDE908019DED2C0B53EC102B9DED080B68
:40F5800051EC100B34F0ACFBCDE90A019DED2C0B53EC102B9DED0A0B51EC100B34F0A0FBCDE90C019DED2C0B53EC102B9DED0C0B51EC100B34F094FBCDE91001389890EDB8
:40F5C0005E0B8DED000B9DED2C0B07E0F8210020FC030020000000000000244053EC102B9DED000B51EC100B34F07AFBCDE902019DED2C0B53EC102B9DED020B51EC100BD6
:40F6000034F06EFBCDE904019DED2C0B53EC102B9DED040B51EC100B34F062FBCDE906019DED2C0B53EC102B9DED060B51EC100B34F056FBCDE908019DED2C0B53EC102B7B
:40F640009DED080B51EC100B34F04AFBCDE90A019DED2C0B53EC102B9DED0A0B51EC100B34F03EFBCDE90C019DED2C0B53EC102B9DED0C0B51EC100B34F032FBCDE90E01CF
:40F680009DED100B53EC102B9DED0E0B51EC100B34F012F8CDE912019DED140B53EC102B9DED120B51EC100B34F006F8CDE916019DED180B53EC102B9DED160B51EC100BFE
:40F6C00033F0FAFFCDE91A019DED1C0B53EC102B9DED1A0B51EC100B33F0EEFFCDE91E019DED200B53EC102B9DED1E0B51EC100B33F0E2FFCDE922019DED240B53EC102BBC
:40F700009DED220B51EC100B33F0D6FFCDE92601389890ED6C0B8DED240B9DED240B53EC102B9DED260B51EC100B33F0C5FFCDE92A01389890ED7A0B8DED200B9DED2C0B32
:40F7400053EC102B9DED200B51EC100B34F0C8FACDE92401389890ED780B8DED1A0B9DED2C0B53EC102B9DED1A0B51EC100B34F0B7FACDE91C019DED2C0B53EC102B9DED23
:40F780001C0B51EC100B34F0ABFACDE92001389890ED760B8DED140B9DED2C0B53EC102B9DED140B51EC100B34F09AFACDE916019DED2C0B53EC102B9DED160B51EC100BC4
:40F7C00034F08EFACDE918019DED2C0B53EC102B9DED180B51EC100B34F082FACDE91C01389890ED740B8DED0E0B9DED2C0B53EC102B9DED0E0B51EC100B34F071FACDE901
:40F8000010019DED2C0B53EC102B9DED100B51EC100B34F065FACDE912019DED2C0B53EC102B9DED120B51EC100B34F059FACDE914019DED2C0B53EC102B9DED140B51EC96
:40F84000100B34F04DFACDE91801389890ED720B8DED080B9DED2C0B53EC102B9DED080B51EC100B34F03CFACDE90A019DED2C0B53EC102B9DED0A0B51EC100B34F030FA11
:40F88000CDE90C019DED2C0B53EC102B9DED0C0B51EC100B34F024FACDE90E019DED2C0B53EC102B9DED0E0B51EC100B34F018FACDE910019DED2C0B53EC102B9DED100B37
:40F8C00051EC100B34F00CFACDE91401389890ED700B8DED020B9DED2C0B53EC102B9DED020B51EC100B34F0FBF9CDE904019DED2C0B53EC102B9DED040B51EC100B34F01F
:40F90000EFF9CDE906019DED2C0B53EC102B9DED060B51EC100B34F0E3F9CDE908019DED2C0B53EC102B9DED080B51EC100B34F0D7F9CDE90A019DED2C0B53EC102B9DED8B
:40F940000A0B51EC100B34F0CBF9CDE90C019DED2C0B53EC102B9DED0C0B51EC100B34F0BFF9CDE91001389890ED6E0B8DED000B9DED2C0B53EC102B9DED000B51EC100B25
:40F9800034F0AEF9CDE902019DED2C0B53EC102B9DED020B51EC100B34F0A2F9CDE904019DED2C0B53EC102B9DED040B51EC100B34F096F9CDE906019DED2C0B53EC102B48
:40F9C0009DED060B51EC100B34F08AF9CDE908019DED2C0B53EC102B9DED080B51EC100B34F07EF9CDE90A019DED2C0B53EC102B9DED0A0B51EC100B34F072F9CDE90C019E
:40FA00009DED2C0B53EC102B9DED0C0B51EC100B34F066F9CDE90E019DED100B53EC102B9DED0E0B51EC100B33F046FECDE912019DED140B53EC102B9DED120B51EC100BDE
:40FA400033F03AFECDE916019DED180B53EC102B9DED160B51EC100B33F02EFECDE91A019DED1C0B53EC102B9DED1A0B51EC100B33F022FECDE91E019DED200B53EC102B9B
:40FA80009DED1E0B51EC100B33F016FECDE922019DED240B53EC102B9DED220B51EC100B33F00AFECDE92601389890ED7C0B8DED240B9DED240B53EC102B9DED260B51EC39
:40FAC000100B33F0F9FDCDE928016421369890FBF1F201FB120008BB9DED2A0B51EC100B33F0B8FD01466422369890FBF2F2521E389800F5027040F822109DED280B51EC5D
:40FB0000100B33F0A7FD01466422369890FBF2F2521E389800F50C7040F82210389890ED000AB1EE400A8DED250A259834F0CEFBCDE926019DED2A0B53EC102B9DED260B5A
:40FB400051EC100B34F0CAF92AD23598401C80B235909DED350AB8EE400ADFEDFE0A00E028E2B4EEE00AF1EE10FA1BDD389890ED530AB5EEC00AF1EE10FA13D19DED2C0BA1
:40FB800051EC100B33F066FD00EE100AB1EE400AF3EE040A30EE200A389880ED530A01E000203590389890ED000AB1EE400A8DED250A259834F08AFBCDE926019DED2A0BF4
:40FBC00053EC102B9DED260B51EC100B34F086F926D23498401C80B234909DED340AB8EE400ADFEDDC0AB4EEE00AF1EE10FA19DD9DED2C0B51EC100B33F02CFD00EE100A7D
:40FC0000F1EE400A9DED340AB8EE400AB2EE041AC0EE011A30EEA10A389880ED520A01E000203490389890ED010AB1EE400A8DED250A259834F04AFBCDE926019DED2A0B89
:40FC400053EC102B9DED260B51EC100B34F046F928D23198401C80B231909DED310AB8EE400AF1EE040AB4EEE00AF1EE10FA1BDD389890ED540AB5EEC00AF1EE10FA13D18E
:40FC80009DED2C0B51EC100B33F0E4FC00EE100AB1EE400AF6EE000A30EE200A389880ED540A01E000203190389890ED030AB1EE400A8DED250A259834F008FBCDE92601F7
:40FCC0009DED2A0B53EC102B9DED260B51EC100B34F004F928D22F98401C80B22F909DED2F0AB8EE400AF1EE040AB4EEE00AF1EE10FA1BDD389890ED550AB5EEC00AF1EE84
:40FD000010FA13D19DED2C0B51EC100B33F0A2FC00EE100AB1EE400AF6EE000A30EE200A389880ED550A01E000202F9038980068259034F0CBFACDE926019DED280B53ECC9
:40FD4000102B9DED260B51EC100B33F08DFF26D23398401C80B233909DED330AB8EE400ADFED7C0AB4EEE00AF1EE10FA19DD389890ED560AB5EEC00AF1EE10FA11D19DED8F
:40FD80002C0B51EC100B33F065FC00EE100AF3EE040A30EE600A389880ED560A01E00020339038980068259034F090FACDE926019DED280B53EC102B9DED260B51EC100B8E
:40FDC00033F052FF24D23298401C80B232909DED320AB8EE400ADFED5F0AB4EEE00AF1EE10FA17DD9DED2C0B51EC100B33F032FC00EE900A9DED320AB8EE400AB2EE041AC5
:40FE0000C0EE011A30EEE10A389880ED570A01E00020329038984068259034F057FACDE926019DED280B53EC102B9DED260B51EC100B33F019FF26D23098401C80B230907D
:40FE40009DED300AB8EE400AF1EE040AB4EEE00AF1EE10FA19DD389890ED580AB5EEC00AF1EE10FA11D19DED2C0B51EC100B33F0F1FB00EE100AF6EE000A30EE600A389819
:40FE800080ED580A01E0002030903898C068259034F01CFACDE926019DED280B53EC102B9DED260B51EC100B33F0DEFE26D22E98401C80B22E909DED2E0AB8EE400AF1EE0A
:40FEC000040AB4EEE00AF1EE10FA19DD389890ED590AB5EEC00AF1EE10FA11D19DED2C0B51EC100B33F0B6FB00EE100AF6EE000A30EE600A389880ED590A01E000202E90D7
:40FF0000389890ED5C0AB1EE400A8DED250A259834F0DCF9CDE926019DED2A0B53EC102B9DED260B51EC100B33F0D8FF19D29DED2A0B51EC100B33F08DFB3899C1F87001FB
:40FF40009DED2C0B51EC100B33F084FB00EE100A02E0000000004843B1EE400A389880ED5A0A3898D0F87401259034F0AFF9CDE926019DED280B53EC102B9DED260B51EC2D
:40FF8000100B33F071FE11D29DED280B51EC100B33F060FB3899C1F874019DED2C0B51EC100B33F057FB3899C1F86C013798401C80B237903798B0F57A7F7FF7D2A9389848
:40FFC00090ED540AB5EEC00AF1EE10FA0BD0389890ED540A80ED5A0A389890ED010AB1EE400A80ED5C0A389890ED580AB5EEC00AF1EE10FA09D0389890ED580A80ED5B0A06
:020000040801F1
:40000000389890ED010A80ED5D0A389890ED530AB5EEC00AF1EE10FA61D0389890ED560AB5EEC00AF1EE10FA59D0389890ED5A0AD0ED530AB7EE001A70EEC10AB4EEE00AF8
:40004000F1EE10FA4BDC389890ED5B0AD0ED560AB7EE001A70EE810AB4EEE00AF1EE10FA3DD3389890ED530AD0ED520A30EE600A8DED230A239834F029F9CDE924019DED1C
:40008000240B30F0FDFC8DED260B9FEDF80B53EC102B9DED260B51EC100B33F01FFF1ED3389890ED560AD0ED570A30EE600A8DED230A239834F00AF9CDE924019DED240B8F
:4000C00030F0DEFC8DED260B9FEDE80B53EC102B9DED260B51EC100B33F000FF03D22320E44981F8DA01389890ED550AB5EEC00AF1EE10FA04D19FEDE00A389880ED550AAB
:40010000389890ED590AB5EEC00AF1EE10FA04D19FEDDA0A389880ED590A39B000BD70B52DED088B064600246FE09FEDD50BB0EE408AF0EE608A9FEDD20BB0EE409AF0EE42
:40014000609A002551E006F1400000EB850090ED000A10EE101A084634F0B8F841EC1B0B04EB440000EBC400C74901EBC00000EBC50090ED001BB0EE410AF0EE610A53EC0D
:40018000102B51EC1B0B33F0ABFD53EC182B33F093FA41EC180B06F16C0000EB850090ED000A10EE101A084634F090F841EC1B0B04EB440000EBC400B34901EBC00000EB10
:4001C000C50090ED001BB0EE410AF0EE610A53EC102B51EC1B0B33F083FD53EC192B33F06BFA41EC190B681CC5B20B2DABDB06F5BC7000EBC40080ED008B06F5DC7000EBDB
:40020000C40080ED009B601CC4B2082C8DDBBDEC088B70BD70B504469C4890F82850022D14D19FED9B0A84ED000A9FED9A0A84ED010A9FED990A84ED020A9FED980A84EDF1
:40024000030A9FED970A84ED040A89E00D2D14D19FED8F0A84ED000A9FED8E0A84ED010A9FED8D0A84ED020A9FED8E0A84ED030A9FED8B0A84ED040A72E00C2D14D19FED1F
:40028000840A84ED000A9FED830A84ED010A9FED820A84ED020A9FED830A84ED030A9FED800A84ED040A5BE0032D14D19FED780A84ED000A9FED770A84ED010A9FED760A71
:4002C00084ED020A9FED780A84ED030A9FED740A84ED040A44E0012D14D19FED6D0A84ED000A9FED6C0A84ED010A9FED6B0A84ED020A9FED6C0A84ED030A9FED6C0A84EDC8
:40030000040A2DE00B2D17D127F0FCF9A0B19FED600A84ED000A9FED5F0A84ED010A9FED5E0A84ED020A9FED5F0A84ED030A9FED600A84ED040A13E09FED550A84ED000A91
:400340009FED540A84ED010A9FED530A84ED020A9FED540A84ED030A9FED540A84ED040A70BD70B52DED028B04465248FFF752FF5048FFF7D4FE4F48FEF7C7FF4D48D0EDB8
:40038000550AB0EE600A204610F01FFA4948D0ED550AB0EE600A204610F093FB4548D0ED590AB0EE600A204610F06DFA4148D0ED590AB0EE600A204610F0A7FB3D4890ED71
:4003C000000AFFEE000A20EE200AB0EE408A90ED5A0AD0ED530A30EE600AD0ED5C0A70EEC80A80EE801A80ED7E1AD0ED7E0A90ED531AB0EE480A00EEC10A80ED7F0A90ED2E
:40040000000AB0EE408A90ED5B0AD0ED560A30EE600AD0ED5D0A70EEC80A80EE801A80ED801AD0ED800A90ED561AB0EE480A00EEC10A80ED810A90ED040AD0ED7E0A80EE4D
:40044000201AB0EE418A9FED0D0A28EE000AB0EE408A9FED190AB4EEC08AF1EE10FA2DDD9FED150AB0EE408A33E00000000000000000F03F381100200000C8C20000C842CE
:400480000000000000000000880000203021002035FA0E3DC2B8323E00000000C2B8B23E8FDAA53B920A063F7CD9A03E88C3643B35FA0E3C2813002000007F43B7EE000AC9
:4004C000B4EEC08AF1EE10FA03D2B7EE000AB0EE408AB6EE000A38EE000ABCEEC00A10EE100AC5B22146284610F04FF82146284610F02FFBFE4890ED040AD0ED800A80EEB9
:40050000201AB0EE418A1FED230A28EE000AB0EE408A1FED170AB4EEC08AF1EE10FA04DD1FED1B0AB0EE408A0AE0B7EE000AB4EEC08AF1EE10FA03D2B7EE000AB0EE408A81
:40054000B6EE000A38EE000ABCEEC00A10EE100AC5B22146284610F04BF82146284610F016FBBDEC028B70BD2DE9F04F2DED088BC5B005468A4600241FED390AB0EE408ACC
:400580001FED3B0AF0EE408A1FED3D0AB0EE409A1FED3F0AF0EE409A032101A816F0FDFFBAF1000F0DD1DFF84C8308F12C0905F1400605F16C0708F11C0B08F14800449055
:4005C00024E0BAF1010F0FD1DFF8288308F1580808F12C0905F1980605F1C40708F11C0B08F14800449011E0BAF1020F0ED1DFF8048308F1B00808F12C0905F1F00605F51A
:400600008E7708F11C0B08F1480044901FED5E0A86ED000A1FED600A87ED000A1FED620A85ED050A032201A9584616F0CAFF032101A817F028F8F0EE409A032201A944980F
:4006400016F0BFFF032101A817F01DF8B0EE409AB6EE080A29EE80AABEEE000A69EE80AAB6EE080A29EE00BABEEE000A69EE00BA012476E000EE104AB8EE400AF2EE040A38
:4006800020EE200A05F1140000EB840080ED000A601E08EB800090ED000AB5EEC00AF1EE10FA06DD1FED840A06EB840080ED000A08E0601E08EB800090ED000A06EB840006
:4006C00080ED000A601E09EB800090ED000AB5EEC00AF1EE10FA06D21FED910A07EB840080ED000A08E0601E09EB800090ED000A07EB840080ED000A06EB840090ED000AFE
:40070000601E06EB8000D0ED000A30EE600AB0EE408A07EB840090ED000A601E07EB8000D0ED000A30EE600AF0EE408AB4EECA8AF1EE10FA0ED3B4EEEA8AF1EE10FA09DC8B
:40074000F4EECB8AF1EE10FA04DCF4EEEB8AF1EE10FA04D223206749283981F8DA01601CC4B20B2C86DB45B0BDEC088BBDE8F08F10B500215E48FFF7F7FE10BD10B52DEDB9
:40078000028B5D4890F828400E2C35D2DFE804F0340C0807130B34341A1B1C230A0900BF00BF00BF00BF00BF9FED540A5148283880ED500A27E09FED520A4E48283880ED08
:4007C000500A20E000BF00BF9FED4C0A4948283880ED500A17E026F07DFF30B1B3EE040A4448283880ED500A05E09FED450A4148283880ED500A06E01FEDD90A3D48283891
:4008000080ED500A00BF00BF08F095FC70B1FAF7D5FFB0EE408AFAF757FF00EE100AB8EE400AB4EEC08AF1EE10FA10DC08F074FC30B1FAF7D8FDB5EEC00AF1EE10FA06DC55
:4008400016F014F8B5EEC00AF1EE10FA09DD2948283890ED500AFFEE000A20EE200A80ED500ABDEC028B10BD73B52DED020B04460D460A2C21D200BF05EB85022149096863
:4008800001F5177101EBC20101EB8400042269460AF0D0FE50B99DED000A05EB85011A4800EBC10000EB840080ED000A00BF1748C16B0220DFF858C000DF7FBD10B5FAF7CB
:4008C00046FB10BD73B52DED020B04460D460A2C35D200BF05EB85020A49096801F59A7101EBC20101EB84000422694612E0000028130020601100203021002000008C42B5
:4009000000004842FC0300208C23002078520020012904080AF08EFE50B99DED000A05EB8501F94800EBC10000EB840080ED000A00BFF648C16B0220DFF8D4C300DF7FBDDF
:4009400073B52DED020B04460D460A2C22D200BF05EB8502EF49096801F5037101EBC20101EB8400042269460AF064FE58B99DED000A05EB8501E448D83000EBC10000EBE2
:40098000840080ED000A00BFE048C16B0220DFF880C300DF7FBD10B5FAF7D9FA10BD73B52DED020B04460D460A2C21D200BF05EB8502D8490968E43101EBC20101EB84006B
:4009C000042269460AF036FE58B99DED000A05EB8501CD48503800EBC10000EB840080ED000A00BFC948C16B0220DFF824C300DF7FBD70B50446C84890F828500E2D28D2FF
:400A0000DFE805F0270C0807120B2727272727180A0900BF00BF00BF00BF00BF1FED490ABE4880ED500A1AE01FED4B0ABB4880ED500A14E026F04EFE28B19FEDB90AB74824
:400A400080ED500A04E01FED530AB44880ED500A05E09FEDB30AB14880ED500A00BF00BF032C08D1AD4890ED500AFFEE000A20EE200A80ED500A70BDA74A92F8281006295A
:400A800005D19FEDA80AA54A82ED500A0CE0042905D11FED650AA14A82ED500A04E01FED690A9E4A82ED500A062808D19B4A92ED500AFFEE000A20EE200A82ED500A7047C4
:400AC000B5EEC00AF1EE10FA01D2012070470020FCE7B5EEC00AF1EE10FA01DD012070470020FCE72DE9F04106460C4615464FF00408894890F828702868A8B929F0C4F9A0
:400B00002860002088490870884890ED000A15F0FAFF20B1BFEE000A854880ED000A15F0A5FE844880ED000A0E2F38D2DFE807F0370C0807160B3737373737200A0900BF3B
:400B400000BF00BF00BF00BF794890ED000A5FED950A20EE200A84ED000A2AE0744890ED000A5FED990A20EE200A84ED000A20E026F0B0FD48B16E4890ED000ADFED680A6D
:400B800020EE200A84ED000A08E0694890ED000A5FEDA60A20EE200A84ED000A09E0644890ED000ADFED5E0A20EE200A84ED000A00BF00BF41F28831286829F06BF928B160
:400BC000212030704FF00108002599E040F6C411286829F05FF9F0B153480078D8B9564890ED000A15F08FFF28B9534890ED000A15F02EFF78B101204B4908704C4890ED89
:400C0000000AFFEE000A20EE200A80ED000A29F03BF9286074E0D4ED000AB0EE600AFFF758FF68B115F022FE4248D0ED000A30EE600ADFED420AB4EEE00AF1EE10FA14DC27
:400C4000D4ED000AB0EE600AFFF73AFFB0B115F00DFE3848D0ED000A30EE600ADFED380AB4EEE00AF1EE10FA08D24FF003089FED2C0A84ED000A0020286041E0D4ED000ABA
:400C8000B0EE600AFFF725FF68B115F0EFFD2948D0ED000A30EE600ADFED290AB4EEE00AF1EE10FA14D3D4ED000AB0EE600AFFF707FF28B315F0DAFD1E48D0ED000A30EE1C
:400CC000600ADFED1E0AB4EEE00AF1EE10FA17DD114890F89C0018B90120F9F758FB07E00D4890F89C00012802D10020F9F74FFB4FF003089FED0A0A84ED000A00202860B8
:400D00004046BDE8F0810000642200207852002001290408FC030020302100203811002000000000000020428D0300207C030020900300209403002074030020C2B8B23D3D
:400D4000C2B8B2BD70B52DED048B0425FE4890F8DC010A287DD2DFE800F00506EF477CEE487CEDEC00BFF84890F8DD0120B1102821D0112835D110E01120F34981F8DD0116
:400D800015F074FDF04880ED080AB6EE000A80ED500A0020EC49086024E0EB4A02F5A07101F19A00FFF79EFE032803D11020E64981F8DD0116E00620E34981F8DC01022000
:400DC00081F8DD010A2081F8E3010020086015F04DFDDD4880ED080AB6EE000A80ED500A00E000BF00BF0AE300BFD74890F8DD01801E0B287BD2DFE800F0067AA0FC60C87D
:400E00007A7A7A7A7B00D048006870B929F03CF8CD490860084690F8E1010A2805DD084690F8E101C01F81F8E101C74991F8DC01FFF722FEC44908684FF47A6129F02AF8BB
:400E4000B0B115F013FDC048D0ED080A30EEC00A00E0F4E3B0EEC00ADFEDBC0AB4EEE00AF1EE10FA04D22120B74981F8DA0123E0B74890ED000A15F046FE20B1B24890F887
:400E8000DC0103280AD0B24890ED000A15F0E0FD90B1AD4890F8DC0106280DD1B6EE000AA94880ED500A0620A74981F8DD010C2081F8DF0100200860A0E2B6EE000AA2484C
:400EC00080ED500A006818B928F0DEFF9E4908609D490868C82128F0DDFF38B19A4890F8DF01994981F8DD010020086086E284E2954991F8DC01FFF77CFD9348006818B9F2
:400F000028F0C2FF904908608F490868C82128F0C1FF68B1B6EE000A8B4880ED500A0620894981F8DD0100200860042081F8DF0164E2FDE3FDE363E263E215F097FCF0EED3
:400F4000409A4FF6FF71834816F08DFC7E48006818B928F099FF7C4908607B4908684FF4FA7128F097FF78B1774890ED680A80ED080A0720744981F8DD010020086001F50D
:400F8000C07000210162416238E26F48006818B928F07AFF6C4908606B4890F8E30100EB8000400000EE100AB8EEC00A664880ED500A90F8DC01032808D1634890ED500A80
:400FC000FFEE000A20EE200A80ED500A604890ED000A15F098FD20B15B4890F8DC0106280CD05B4890ED000A15F032FDC0B1564800E030E090F8DC01032811D102205249C3
:4010000081F8DD0101F5C07000210162416215F02DFC4D4880ED080A00204B49086019E0494908684FF4FA7128F034FF90B1B6EE000A454880ED500A0620434981F8DD016E
:40104000086828F049FF4049C86100200860052081F8DF01D2E115F009FCF0EE409A4FF6FF713C4816F0FFFB3748006818B928F00BFF35490860344908684FF4FA7128F0C7
:4010800009FF00285FD0304890ED680AD0ED080A30EE608AB0EEC80AF0EE409A15F0D8FC20B1294890F8DC01032821D0284890ED000A15F0CDFC20B1234890F8DC0103283E
:4010C00016D0B0EEC80AF0EE409A15F01CFD20B11D4890F8DC0106280AD01D4890ED000A15F011FD98B1184890F8DC0106280ED10220154981F8DD01084690ED680A80ED86
:40110000080A00F5C0700021016241620DE007200D4981F8DD01084690ED680A80ED080A00F5C070002101624162074890F8E301401E054981F8E301084690F8DC010328E6
:4011400062D1084608E057E13811002035FA0E3D74030020D812002090ED070AF8EE400A9FEDFE1A80EE810AC8EE000A90F8E311283000EB8100C0ED000AF94A92F8421019
:40118000F84A92F8E30192F8E331283202EB8302D2ED000AB0EE600AFFF701FCF14890F8E311283000EB8100D0ED000AB0EE600A0020FDF75EFEFFF7EEFBEA4890F8E3110C
:4011C000803000EB810080ED000AE54A92F84210E44A92F8E30192F8E331803202EB8302D2ED000AB0EE600AFFF7AAFBDD4890F8E311803000EB8100D0ED000AB0EE600AFB
:401200000020FDF7EBFD57E0D64890ED070AF8EE400A9FEDD21A80EE810AC8EE000A90F8E311543000EB8100C0ED000ACC4A92F84210CC4A92F8E30192F8E331543202EBC4
:401240008302D2ED000AB0EE600AFFF73BFBC54890F8E311543000EB8100D0ED000AB0EE600A0020FDF7E0FDFFF728FBBD4890F8E311AC3000EB810080ED000AB84A92F8CE
:401280004210B84A92F8E30192F8E331AC3202EB8302D2ED000AB0EE600AFFF7E5FAB14890F8E311AC3000EB8100D0ED000AB0EE600A0020FDF792FDAA4890F8E301002823
:4012C00013D1A84890F8DC0106280FD10320A54981F8DC01022081F8DD01B6EE000A084680ED500A0A2081F8E30182E0B7EE000A9C4880ED4E0A09209B49087026E0994857
:401300005430994991F9001000EB810090ED000A5FED720AB4EEE00AF1EE10FA10D2924890F9000000EE100AB8EEC00AF2EE040A20EE200A8B4880ED4E0AFF208A49087098
:4013400089480078401E40B287490870864890F900000028D3DAB7EE000A824880ED4D0A09208149087026E07E4828307E4991F9001000EB810090ED000ADFED7C0AB4EE4C
:40138000E00AF1EE10FA10DD774890F9000000EE100AB8EEC00AFAEE040A20EE200A714880ED4D0AFF20704908706F480078401E40B26D4908706C4890F900000028D3DAF3
:4013C000684890ED4E0A80ED4F0A0520654981F8DC010D2081F8DD01B6EE000A084680ED500A002081F8E3019FED610A084680ED4C0A00205B49086000E000BF00BFD9E169
:4014000000BF584890F8DD0106281DD00D2802D00E287DD132E0FFF7B1F9564890ED000A15F046FB78B1B6EE000A4E4880ED500A06204C4981F8DD010E2081F8DF0128F03F
:4014400023FD484908608EE1B6EE000A454880ED500A014608684FF4FA7128F01BFD60B1404890F8DF013F4981F8DD010020086015F0FCF93B4880ED080A74E1394890F88B
:40148000DC01052807D115F0F1F93648D0ED080A70EE608A06E015F0E9F93248D0ED080A70EEC08A2F48006860B928F0EDFC2D49086008460068C1F8E4019FED2D0A0846CC
:4014C00080ED7A0A264890F8430001282FD128F0DBFC2449D1F8E411441A224890ED7A0A30EE280A80ED7A0AB4F57A7F1AD3D0ED7A0A00EE104AB8EE400A80EE801AF0EE87
:40150000418A9FED1B0A80ED7A0A28F0BDFC00E028E11449C1F8E40115F0A8F9114880ED080A03E09FED120AF0EE408A00BF0C4890ED6E0AB4EEE80AF1EE10FA7ED20948B2
:4015400090ED4C0AD0ED500A30EE200A80ED4C0A90F8E301401C03490EE0000000007A4430210020381100208C03002035FA0EBD000000007803002081F8E301B6EE000A8D
:40158000084680ED500A0D2081F8DD01086828F0A3FC00EE100AB8EE400A5FED100A80EE209AFE4890F8DC01052816D1FB4890ED4F0A30EE090AF1EE040A30EE600A80EDFA
:4015C0004F0A90ED4F0AB5EEC00AF1EE10FA1AD21FED190A80ED4F0A15E0F04890ED4F0A30EE490AF1EE040A30EE200A80ED4F0A90ED4F0AB5EEC00AF1EE10FA03DD1FEDFE
:40160000240A80ED4F0AE54890F8E30103283ADBE248D0ED4C0A90F8E30100EE100AB8EE400A80EE801ADD4880ED4C1A90F8DC01052829D1DA4991F8420001E03FE0B8E02A
:40164000D649D1ED4C0AB0EE600A0FF016FA1FED380AD24880ED4C0AB6EE000A80ED500A0020CE4981F8E301022081F8DC010D2081F8DD0128F008FCC8490860084690ED90
:401680004D0A80ED4F0A6CE0C54991F84200C349D1ED4C0AB0EE600A0FF0CBF91FED4C0ABE4880ED4C0AB6EE000A80ED500A0820BA4981F8DC010F2081F8DD0151E0B74826
:4016C00090ED500AB0EEC00ADFEDB60AB4EEE00AF1EE10FA07DA0146086828F0FDFB4EF66021884207D92120AC4981F8DA01092081F8DC0135E0A94890F8DC01022819D10B
:40170000A649086828F0E8FB00EE100AB8EE400AFFEE000A20EE200A1FED701AC0EE010A9E4890ED4F0A30EE800A80ED500A18E01BE021E09949086828F0CEFB00EE100A7F
:40174000B8EE400AF7EE000A20EE200A1FED7D1AC0EE010A914890ED4F0A30EE800A80ED500A00E000BF00BF24E002251FED800A8A4880ED500A1DE0FEF7FAFF874890F8DE
:40178000DA0120B10920854981F8DC0110E0844991F84200FEF7E5FD1020804981F8DD0103251FED8D0A084680ED500AFDF797FD00E000BF00BF794890F8DE01774991F84A
:4017C000DD11884214D0754890F8E101401C734981F8E101084690F8E101642802DD642081F8E1016D4890F8DD016C4981F8DE016A4890ED500AB5EEC00AF1EE10FA08D0D2
:40180000D0ED500AB0EE600A01210846F8F75FFE08E06248D0ED500AB0EE600A00210120F8F755FE2846BDEC048B70BD2DE9F0412DED048B042607F07EFC10B1B3EE090AC5
:4018400001E0B1EE040AB0EE409A07F074FC08B1554800E05548044607F06DFC08B1544800E0544807464D4890F8DC010A2872D2DFE800F00506D77171D67171F9F800BF0D
:40188000464890F8DD0120B110287DD011280ED000BF1120414981F8DD01B6EE000A084680ED500A28F0F0FA3C490860B6E03B49086828F011FBB0F5FA7F04D2A04737483C
:4018C00080ED090A89E03549086828F005FB40F6B831884205D29FED380A304880ED500A7BE02E49086828F0F7FA40F6AC51884217D2B6EE000A294880ED500AA0472748BF
:40190000D0ED090A30EE600AB4EEC90AF1EE10FA63DD1E20214981F8DA01092081F8DC015BE01E49086828F0D7FAB0F57A6F04D2A0471A4880ED090A4FE01849086828F0F6
:40194000CBFA41F66411884206D29FED160A134880ED500A41E059E21049086828F0BCFA41F6583188422CD2B6EE000A0B4880ED500AA0470948D0ED090A30EE600AF1EED4
:40198000490AB4EEE00A00E028E0F1EE10FA24D21E20024981F8DA0109200FE0381100203021002000008C42BDB70008E7B30008C9B9000809B4000800008CC281F8DC01D3
:4019C0000BE0B6EE000AFE4880ED500A28F05CFAFB490860102081F8DD011FE00520F84981F8DC010D2081F8DD01B6EE000A084680ED500A002081F8E30128F045FAF04991
:401A000008609FEDF00A084680ED4C0A9FEDED0A80ED4F0A002081F8E10100BF00BFF6E100BFE74890F8DD0106282DD00D2802D00E287CD141E0FEF7A1FEB0EE000AB84729
:401A400090B1B6EE000ADE4880ED500A0620DC4981F8DD010E2081F8DF0128F015FAD849086010E068E16EE1D549086828F034FA44F62061884206D92120D14981F8DA0142
:401A8000092081F8DC0155E1B6EE000ACC4880ED500A014608684FF4FA7128F0FBF958B1C74890F8DF01C64981F8DD0100200860A047C34880ED090A3CE1C14890F8DC010C
:401AC000052806D1A047BE48D0ED090A70EE608A05E0A047BA48D0ED090A70EEC08AB848006818B928F0D0F9B5490860F4EEC98AF1EE10FA7EDDB24890F8E301002808DD2B
:401B0000AF4890ED4C0AD0ED500A30EE200A80ED4C0AAB4890F8E301401CA94981F8E301B6EE000A084680ED500A0D2000E000E181F8DD01086828F0CFF900EE100AB8EEA9
:401B4000400ADFEDA10A80EE208A9D4890F8E301012804D1B1EE040A28EE000A03E0B6EE000A28EE000AB0EE408A28F08DF994490860084690F8DC01052816D1084690EDE2
:401B80004F0A30EE080AF2EE040A30EE600A80ED4F0A90ED4F0AB5EEC00AF1EE10FA1AD29FED880A80ED4F0A15E0854890ED4F0A30EE480AF2EE040A30EE200A80ED4F0A60
:401BC00090ED4F0AB5EEC00AF1EE10FA03DD9FED7D0A80ED4F0A7A4890F8E30103283DDD7748D0ED4C0A90F8E30100EE100AB8EE400A00E04EE0B7EE001A30EE410A80EEB3
:401C0000801A6F4880ED4C1A90F8DC01052826D16E4991F842006A49D1ED4C0AB0EE600A0EF02BFF9FED670A654880ED4C0AB6EE000A80ED500A0020614981F8E301022053
:401C400081F8DC010D2081F8DD0128F01DF95C4908609FED5C0A084680ED4F0A68E05B4991F842005649D1ED4C0AB0EE600A0EF0E0FE9FED540A524880ED4C0AB6EE000A06
:401C800080ED500A08204E4981F8DC010F2081F8DD014DE04A4890ED500AB0EEC00ADFED4C0AB4EEE00AF1EE10FA07DA0146086828F012F94EF66021884207D92120404939
:401CC00081F8DA01092081F8DC0131E03C4890F8E30110B9B1EE040A01E0B6EE000AF0EE409A3749086828F0F7F800EE100AB8EE400A20EE290ADFED340A80EE201A3048F9
:401D000080ED501A90F8DC01022808D12C4890ED500AFFEE000A20EE200A80ED500A284890ED500AD0ED4F0A30EE200A80ED500A00E000BF00BF6AE002269FED220A2048C7
:401D400080ED500A63E01E4890F8DA0120B109201B4981F8DC0158E06425A8461B4991F84200694200EE101AB8EEC00A0EF02DFD164991F84200694200EE101AB8EEC00A46
:401D80000EF09FFE114991F8420000EE105AB8EE400A0EF078FD0D4991F8420000EE105AB8EE400A0EF0B1FE084890F8421040460EF0EBFB054890F8421040460AE0000067
:401DC000381100200000000000007A44302100200000A0420EF0BDFEFE4890F8421040460EF006FCFB4890F8421040460EF0CFFE1020F94981F8DD0103261FED0E0A084638
:401E000080ED500AFDF76BFA00BF00E000BF00BFF14890F8DE01F04991F8DD11884214D0ED4890F8E101001DEB4981F8E101084690F8E101642802DD642081F8E101E648EC
:401E400090F8DD01E44981F8DE01E34890ED500AB5EEC00AF1EE10FA08D0D0ED500AB0EE600A01210846F8F732FB08E0DA48D0ED500AB0EE600A00210120F8F728FB3046A9
:401E8000BDEC048BBDE8F081002070471FED330AD14880ED720A1FED350A80ED740A1FED370A80ED6C0A1FED390A80ED6A0A1FED3B0A80ED700A1FED3D0A80ED6E0A7047F5
:401EC00070B52DED048B0446F0EE408AB0EE609AF0EE419A0D46BF4890F83000702804D0BC4890F8300093280CD1F7EE000A80EEA80A5FED4B0A89EE201A20EE010A20EE77
:401F0000298A6FE0B34890F8300091280ED0B14890F83000922809D0AE4890F83000712804D0AC4890F83000B8280CD1F0EE000A80EEA80A5FED5C0A89EE201A20EE010A09
:401F400020EE298A4EE0A81E0C283DD2DFE800F02D3C063C13203C3C3C3C2F2EF0EE080A80EEA80A5FED680A89EE201A20EE010A20EE298A35E0DFED990A80EEA80A5FED3E
:401F80006E0A89EE201A20EE010A20EE298A28E0DFED930A80EEA80A5FED750A89EE201A20EE010A20EE298A1BE000BF00BFDFED8D0A80EEA80A5FED7C0A89EE201A20EEAA
:401FC000010A20EE298A0CE0DFED870A80EEA80A5FED830A89EE201A20EE010A20EE298A00BF00BFB2EE040AB4EEC08AF1EE10FA04D2B2EE040AB0EE408A0AE09FED7B0A60
:40200000B4EEC08AF1EE10FA03DD9FED780AB0EE408A012C0AD16F4A92F84210BCEEC80A10EE102AD0B20EF094FD09E0694A92F84210BCEEC80A10EE102AD0B20EF0A7FDC3
:40204000BDEC048B70BD00B52DED028B95B0624890ED500A8DED140A27F016FF0E9004200C9014F0A9FB5C4880ED520AC0685A4948610846006988615D48007829F0CBFE8F
:402080005549C86027F000FF53490861084680690B9027F021FF4FF47A71B1FBF0F00F904D48C0684C494969401A00EE100AB8EEC00AF7EE000A20EE200A9FED4E1AC0EE3E
:4020C000010A9DED0F0AB8EEC00A20EE800A8DED130A052148489DED130A15F0C4FB0521454808309DED140A15F0BDFB1EF0EEFB8DED0B0A1E21404818389DED0B0A15F0E1
:40210000B2FB3E4890ED000A8DED0B0A1E213A4820389DED0B0A15F0A6FB384890ED000A2D4880ED510A3648007810F029FB8DED0B0A0521304808389DED0B0A15F093FBFB
:402140003048007810F0D9FC8DED050A059832F0BDF8CDE906019DED060B2EF091FC8DED080B9DED080B51EC100B31F073FA05210B90214810389DED0B0A15F074FB1548A8
:40218000B0F8BE014FF4967190FBF1F000EE100AB8EEC00A8DED0D0A0E4890F8280006284ED00C4890F82800072849D00A4890F8DC01042804D0084890F8DC0107283FD1B0
:4021C000054890ED740ADFED100AB4EEE00AF1EE10FA1BE03021002038110020CDCC4C406666A6408FC2753E9A99193F00007F436007002052EC2F4500130020AC550020B2
:402200001B0700206C0700200000484219DD90ED721A9DED0D0AF2EE040AF1EE041A41EEC00AB4EEE01AF1EE10FA79D20920FE4981F8DC01242081F8DA01002081F8DD0116
:402240006EE0F94890ED740ADFEDF80AB4EEE00AF1EE10FA19D290ED721A9DED0D0AFAEE040AF1EE041A41EE800AB4EEE01AF1EE10FA55DD0920EC4981F8DC01242081F828
:40228000DA01002081F8DD014AE0E748D0F8D001079032F01BF8CDE908019DED080B2EF0EFFB8DED0A0B9FEDE20B53EC102B9DED0A0B51EC100B31F013FC31D1DDED0D0A1E
:4022C000B1EE040AB1EE041A01EE200A8DED070A079831F0FBFFCDE90A01D348D0F8C801059031F0F3FFCDE906019DED060B2EF0C7FB8DED080B9DED0A0B53EC102B9DED99
:40230000080B51EC100B31F0E9FD09D20920C64981F8DC01242081F8DA01002081F8DD01C14890F8DD01062813D1BF48806801460B900E9827F0DFFDBB494968884241F216
:402340009284B94890F8DF01B74981F8DD0101F08ABCB54890F8DC010A2881F08284DFE810F030000A0040006404800C54029007800C760C610CAC4890F8DB0180B1AA482D
:4023800090F8DB01A84981F8DC01062081F8DD01002081F8DF01192048600E9888600EE00020A14981F8DC01062081F8DD01002081F8DF014FF47A7048600E98886001F075
:4023C00051BC0220984981F8DC01062081F8DD01002081F8DF014FF47A7048600E988860EDE7914890F8DC018F4981F8DB01084690F8DD0108287CD003DC38B1052879D170
:4024000069E1092877D00B28F9D10BE00620864981F8DD010B2081F8DF01192048600E988860F0E18048806801460B900E9827F062FD41F28831884207D909207A4981F839
:40244000DC01262081F8DA0170E07B4890F8280006280ED0784890F82800072809D0724890ED520ADFED750AB4EEE00AF1EE10FA13DC714890F82800062804D06E4890F8B3
:40248000280007280FD1684890ED520ADFED6C0AB4EEE00AF1EE10FA05DDBBEE0E0A624880ED500A42E0644890F8280006280ED0614890F82800072809D05B4890ED520A2A
:4024C000DFED600AB4EEE00AF1EE10FA17D35A4890F82800062804D0574890F82800072813D1514890ED520ADFED570AB4EEE00A02E034E080E11AE0F1EE10FA05D2B3EEB4
:402500000E0A494880ED500A10E00620464981F8DD01092081F8DF014FF47A7048600E9888609FED4A0A084680ED500A6BE106203D4981F8DD01082081F8DF0119204860A4
:402540000E988860BAEE000A084680ED500A4048007829F060FC3449C1F8880153E1364890F82800062804D0334890F82800072810D12D48C0682C49D1F88811401A00EE77
:40258000100AB8EEC00ADFED330AB4EEE00AF1EE10FA40D3284890F8300091280FD0264890F8300092280AD0234890F83000712805D0214890F83000B82800D010E01A48D2
:4025C000C0681949D1F88811401A00EE100AB8EEC00ADFED210AB4EEE00AF1EE10FA1AD3154890F82800062851D0134890F8280007284CD00C48C0680B49D1F88811401A86
:4026000000EE100AB8EEC00ADFED120AB4EEE00AF1EE10FA3BD2084890F842000B909DED140A0EF006FA19E038110020000048C2000000000000204030210020CDCCCC3C7F
:40264000CDCC4C3DCDCCCCBCCDCC4CBD00000000600700206CE7DBC57390EAC40620FE4981F8DD01052081F8DF014FF47A7048600E9888609DED140A084680ED500AF748A9
:40268000007829F0C8FBF449C1F8880122E0F24890ED500A5FED1B0AB4EEE00AF1EE10FA0BD81FED160A80ED500A0920EA4981F8DC01272081F8DA010CE09DED140ADFEDCB
:4026C000E80A30EE600A8DED140A9DED140AE24880ED500A97E0E048D0ED500A9FEDE11A80EE810A8DED010A019831F0EFFDCDE902019DED020B2EF0C3F98DED060BD648FB
:40270000D0F8C001039031F0E1FDCDE904019DED060B53EC102B9DED040B51EC100B31F0DFFA9FEDD10B53EC102BCDE908019DED080B51EC100B31F07BF8CDE90A019DED4E
:402740000A0B51EC100B30F085FFC349C1F85801084690ED6E0ADFEDC60A80EE201A80ED5A1AC44890F8300091280ED0C14890F83000922809D0BF4890F83000712804D0E7
:40278000BC4890F83000B82804D1B3EE090A8DED100A03E0B1EE040A8DED100A9DED100ADFEDB50A80EE201A9FEDB40A21EE000ABDEEC00AB8EEC00AA74880ED5E0AB0F8B1
:4027C000D80140F00400A449A1F8D801052081F8DC010621A04880F8DD1100209E4981F8DF014FF47A7048600E9888601FED690A084680ED500A06E000209749A1F8D801CE
:4028000081F8DC0100BF00BFD9E5934890F8DC01914981F8DB01084690F8DD0108287CD003DC38B1052879D167E1092877D00B28F9D10BE00620884981F8DD010B2081F88E
:40284000DF01192048600E988860ECE18248806801460B900E9827F04EFB41F28831884207D909207C4981F8DC01282081F8DA0170E0804890F8280006280ED07D4890F80B
:402880002800072809D0744890ED520A5FED950AB4EEE00AF1EE10FA13DC764890F82800062804D0734890F8280007280FD16A4890ED520A5FED9E0AB4EEE00AF1EE10FA26
:4028C00005DDBBEE0E0A644880ED500A42E0694890F8280006280ED0664890F82800072809D05D4890ED520A5FEDAA0AB4EEE00AF1EE10FA17D35F4890F82800062804D097
:402900005C4890F82800072813D1534890ED520A5FEDB30AB4EEE00A02E034E07CE11AE0F1EE10FA05D2B3EE0E0A4B4880ED500A10E00620484981F8DD01092081F8DF0187
:402940004FF47A7048600E9888601FEDC00A084680ED500A67E106203F4981F8DD01082081F8DF01192048600E988860B2EE000A084680ED500A3948007829F04CFA364936
:40298000C1F888014FE13B4890F82800062804D0384890F82800072810D12F48C0682E49D1F88811401A00EE100AB8EEC00ADFED340AB4EEE00AF1EE10FA40DC2D4890F84E
:4029C000300091280FD02B4890F8300092280AD0284890F83000712805D0264890F83000B82800D010E01C48C0681B49D1F88811401A00EE100AB8EEC00ADFED220AB4EE36
:402A0000E00AF1EE10FA1ADC1A4890F8280006284FD0184890F8280007284AD00E48C0680D49D1F88811401A00EE100AB8EEC00ADFED130AB4EEE00AF1EE10FA39DD0D4844
:402A400090F842000B909DED140A0EF016F80620014981F8DD0117E03811002060070020CDCCCC3D0000C8420000000000408F4000007A4430210020000070428DED24480D
:402A80006CE7DB457390EA44052081F8DF014FF47A7048600E9888609DED140A084680ED500AF848007829F0B6F9F749C1F8880122E0F54890ED500ADFEDF40AB4EEE00A66
:402AC000F1EE10FA0BDB9FEDF20A80ED500A0920ED4981F8DC01292081F8DA010CE09DED140A5FED210A30EE200A8DED140A9DED140AE54880ED500A95E0E348D0ED500A28
:402B00001FED281A80EE810A8DED010A019831F0DDFBCDE902019DED020B2DF0B1FF8DED060BD948D0F8C001039031F0CFFBCDE904019DED060B53EC102B9DED040B51ECC1
:402B4000100B31F0CDF81FED380B53EC102BCDE908019DED080B51EC100B30F069FECDE90A019DED0A0B51EC100B30F073FDC649C1F86001084690ED6E0A5FED430A80EE95
:402B8000201A80ED5C1AC34890F8300091280ED0C04890F83000922809D0BE4890F83000712804D0BB4890F83000B82804D1B3EE090A8DED100A03E0B1EE040A8DED100A44
:402BC0009DED100A1FED541AC0EE010A1FED550A20EE800ABDEEC00AB8EEC00AAA4880ED600AB0F8D80140F02000A749A1F8D801032081F8DC01062081F8DD01002081F88B
:402C0000DF014FF47A7048600E9888609FEDA00A084680ED500A06E000209B49A1F8D80181F8DC0100BF00BFEEE5974890F8DC01954981F8DB01084690F8DD0130B10528CA
:402C40007ED007287DD00A287CD111E006208E4981F8DD010A2081F8DF01192048600E988860084690ED520A8B4880ED000A06E38548806801460B900E9827F03CF942F2BD
:402C80001071884234D9804890ED520A8248D0ED000A30EEC00A8DED070A079831F016FBCDE908019DED080B2DF0EAFE8DED0A0B9FED7A0B53EC102B9DED0A0B51EC100BD4
:402CC00031F00CF90CD2774890ED000ADFED760A20EE200A80ED000A6B490E988860D0E00920694981F8DC01262081F8DA01C8E0684890F8280006280ED0664890F8280060
:402D0000072809D0604890ED520A5FEDAB0AB4EEE00AF1EE10FA17DC5E4890F82800062804D05C4890F82800072834D1564890ED520ADFED5E0AB4EEE00AF1EE10FA02E0BF
:402D4000BAE03FE294E226DD524890F82800062804D0504890F8280007280ED100BF4D48D0ED300A4F4890ED001AB0EE040A11EE200A454880ED500A83E04648D0ED300AF3
:402D8000484890ED001AB2EE0E0A11EE200A3E4880ED500A75E03F4890F8280006280ED03C4890F82800072809D0374890ED520ADFED3F0AB4EEE00AF1EE10FA13D33548A5
:402DC00090F82800062804D0324890F82800072830D12D4890ED520A5FEDDF0AB4EEE00AF1EE10FA26D22B4890F82800062804D0284890F8280007280ED100BF2548D0ED9B
:402E0000320A284890ED001AB0EE040A01EE200A1D4880ED500A34E01E48D0ED320A214890ED001AB2EE0E0A01EE200A164880ED500A26E00620144981F8DD01052081F877
:402E4000DF0140F6B83048600E988860114890F8280007280AD10F4890ED320ADFED150A20EE200A084680ED500A04E09FED080A054880ED500A00200349C1F88801C1F8C6
:402E80009401FCE160070020381100200000484200000000302100208403002000000040E17A743F88030020CDCC8C3FCDCC4C3ECDCC4C3D9A99193FFA48D0F88801D0BBC3
:402EC000F948007828F0A7FFF649C1F88801084690ED6A0A80ED630A90ED6C0A80ED640A062081F8DD01072081F8DF01EF4890F82800072803D14FF47A70486003E04FF411
:402F00007A70E8494860E7490E988860E74890F82800062804D0E54890F8280007280BD1E24890ED300AF2EE0E0A30EE600ADD4880ED500A45E10AE0DC4890ED300A5FEDC3
:402F40002D0A30EE600AD74880ED500A39E1D548D0F8940100287DD1D348007828F05BFFD049C1F89401084690ED6A0A80ED660A90ED6C0A80ED670AD0F89401D1F888118A
:402F8000401A0B9014F0DAFE00EE100AB8EE400ADFEDC70A20EE200ADFEDC50A80EE201AC04880ED5F1AD0F89401BE49D1F88811401A00EE100AF8EEC00A9FEDBE0AF4EE34
:402FC000C00AF1EE10FA7DD2B84890F82800062804D0B64890F82800072804D19FEDB60A8DED130A04E0AF4890ED6C0A8DED130AAE4890F82800072839D1AA4890F8E001E9
:403000000B90AA4890ED0F0A8DED0A0AA54890ED660A8DED090A0B989DED0A1ADDED130A9DED090A12F017FC9E4880ED550A90F8E0010B909D4890ED0F0A8DED0A0A9948EE
:4030400090ED630A8DED090A0B989DED0A1ADDED130A00E0B5E09DED090A12F0FCFB9148D0ED550A30EEC00A80ED550A38E08D4890F8E0010B908D4890ED0F0A8DED0A0A03
:40308000884890ED660A8DED090A0B989DED0A1ADDED130A9DED090A12F0DDFB814880ED550A90F8E0010B90804890ED0F0A8DED0A0A7C4890ED630A8DED090A0B989DED2A
:4030C0000A1A00E071E0DDED130A9DED090A12F0C2FB7448D0ED550A30EEC00A80ED550A704890F8E0010B906E4890ED570AB1EE400A8DED0A0A90ED550A8DED090A0B99D8
:403100009DED0A1ADFED6A0A9DED090A0120FEF7D7FE644890ED550AF7EE000A80EE201A1FEDA50A31EE408A644800780FF028FB9FED5F1AC0EE010A5A4890ED570AB1EE33
:40314000400A80EE201A594890ED300ADFED5C0A11EE200AC8EE000A5248C0ED530AB0F8D80140F008004F49A1F8D8010846B0F8D80140F01000A1F8D801062081F8DC0186
:4031800081F8DD01002081F8DF014FF47A7048600E9888601FEDC20A084680ED500AB7EE000A484880ED000A0BE01FEDC70A3D4880ED500A09203B4981F8DC012B2081F85E
:4031C000DA015CE00620374981F8DD01052081F8DF010A2048600E9888600846D0ED500A9FED371A80EE810A8DED010A019831F06DF8CDE902019DED020B2DF041FC8DEDDA
:40320000060B2848D0F8C001039031F05FF8CDE904019DED060B53EC102B9DED040B51EC100B30F05DFD9FED280B53EC102BCDE908019DED080B51EC100B30F0F9FACDE988
:403240000A019DED0A0B51EC100B30F003FA1549C1F85C01084690ED6E0ADFED150A80EE201A80ED5B1ABAEE000A80ED500A06E000200C49A1F8D80181F8DC0100BF00BFE9
:40328000FDE3084890F8DC01064981F8DB01084690F8DD01E0B105287ED007287DD00A287CD121E038110020600700203021002000007A44FF4680C639B400401B07002000
:4032C0000000C842880300200000000000408F400620F74981F8DD010A2081F8DF01192048600E988860EEE3F148806801460B900E9826F000FE42F21071884234D9EC480D
:4033000090ED520AEB48D0ED000A30EEC00A8DED070A079830F0DAFFCDE908019DED080B2DF0AEFB8DED0A0B9FEDE30B53EC102B9DED0A0B51EC100B30F0D0FD0CD2E04820
:4033400090ED000ADFEDDF0A20EE200A80ED000AD7490E988860D0E00920D54981F8DC01282081F8DA01C8E0D74890F8280006280ED0D54890F82800072809D0CC4890EDE2
:40338000520ADFEDD20AB4EEE00AF1EE10FA17D3CD4890F8280002E0B0E0E3E3FEE3062804D0C94890F82800072830D1C04890ED520ADFEDC70AB4EEE00AF1EE10FA26D2EE
:4033C000C14890F82800062804D0BF4890F8280007280ED100BFBC48D0ED320AB84890ED001AB0EE040A01EE200AB14880ED500A83E0B548D0ED320AB14890ED001AB2EEEC
:403400000E0A01EE200AAA4880ED500A75E0AE4890F8280006280ED0AB4890F82800072809D0A34890ED520ADFEDAA0AB4EEE00AF1EE10FA13DCA44890F82800062804D0AA
:40344000A14890F82800072830D1994890ED520ADFED9E0AB4EEE00AF1EE10FA26DD9A4890F82800062804D0974890F8280007280ED100BF9448D0ED300A914890ED001AAA
:40348000B0EE040A11EE200A894880ED500A34E08D48D0ED300A8A4890ED001AB2EE0E0A11EE200A824880ED500A26E00620804981F8DD01052081F8DF0140F6B830486054
:4034C0000E988860804890F8280007280AD17E4890ED300ADFED800A20EE200A084680ED500A04E09FED7D0A714880ED500A00206F49C1F88801C1F8940191E36C48D0F8CD
:403500008801D0BB7648007828F085FC6849C1F88801084690ED6A0A80ED630A90ED6C0A80ED640A062081F8DD01072081F8DF01654890F82800072803D14FF47A7048609C
:4035400003E04FF47A705A49486059490E9888605D4890F82800062804D05B4890F8280007280BD1584890ED320AF2EE0E0A30EE200A4F4880ED500AF3E20AE0524890ED3E
:40358000320ADFED580A30EE200A494880ED500AE7E24748D0F894010028EDD15048007828F039FC4249C1F89401084690ED6A0A80ED660A90ED6C0A80ED670AD0F89401E6
:4035C000D1F88811401A0B9014F0B8FB4FF47A71B0FBF1F000EE100AB8EE400A5FEDCC0A20EE200A324880ED610AD0F894013049D1F88811401A00EE100AB8EEC00ADFED89
:403600003A0AB4EEE00AF1EE10FA50DD2E4890F82800062804D02C4890F82800072804D11FEDDB0A8DED130A04E0214890ED6C0A8DED130A244890F82800072856D11C481F
:4036400090F8E0010B90204890ED0F0A8DED0A0A174890ED660A8DED090A0B989DED0A1ADDED130A9DED090A12F0F5F8104880ED550A90F8E0010B90134890ED0F0A8DED8A
:403680000A0A0B4890ED630A8DED090A0B989DED0A1ADDED130A9DED090A12F0DCF80448D0ED550A30EEC00A80ED550A55E04CE2381100208403002000000040E17A743FA4
:4036C00088030020CDCC8C3F30210020CDCCCCBDCDCC4CBECDCC4CBD9A99193F000000006007002000004842FF468046F64890F8E0010B90F54890ED0F0A8DED0A0AF2485F
:4037000090ED660A8DED090A0B989DED0A1ADDED130A9DED090A12F09EF8EB4880ED550A90F8E0010B90E94890ED0F0A8DED0A0AE54890ED630A8DED090A0B989DED0A1A55
:40374000DDED130A9DED090A12F085F8DE48D0ED550A30EEC00A80ED550ADB4890F8E0010B90D94890ED590A8DED0A0A90ED550A8DED090A0B999DED0A1ADFEDD50A9DEDAA
:40378000090A0220FEF79CFBCF4890ED550AF7EE000A80EE201A1FED2F0A31EE408ACD4800780EF0EDFFDFEDCA0A80EE201AC64890ED590AC0EE010AC44890ED320A9FEDD9
:4037C000C61A10EE810AC8EE000ABF48C0ED540AB0F8D80140F04000BB49A1F8D8010846B0F8D80140F08000A1F8D8010846D0ED560A90ED580A30EE800A80ED560A90EDFA
:40380000560AF0EE000A80EE201A80ED561A90ED570AD0ED590A30EE200A80ED570A90ED570AF0EE000A80EE201A80ED571A90ED5A0AD0ED5C0A30EE200A80ED5A0A90EDC1
:403840005A0AF0EE000A80EE201A80ED5A1A90ED5B0AD0ED5D0A30EE200A80ED5B0A90ED5B0AF0EE000A80EE201A80ED5B1A90ED5E0AD0ED600A30EE200A80ED5E0A90ED59
:403880005E0AF0EE000A80EE201A80ED5E1A90ED5E0ADFED920A20EE200A80ED5E0A90ED5F0AD0ED610A30EE200A80ED5F0A90ED5F0AF0EE000A80EE201A80ED5F1A90EDCC
:4038C0005F0ADFED860A20EE200A80ED5F0A90ED5B0AD0ED5A0A70EE600A90ED570A90ED561A30EE411A80EE810A8DED0B0A9DED0B0A0AF0CEF8744890ED5B0A7348D0EDE9
:40390000700A714890ED571A00EEC10A8DED0B0A9DED0B0A0AF0A3F86B4890ED5F0AD0ED5E0A70EE600A90ED570A90ED561A30EE411A80EE810A8DED0B0A9DED0B0A0AF0FF
:4039400074F8614890ED5F0A6048D0ED720A5E4890ED571A00EEC10A8DED0B0A9DED0B0A0AF049F85B4800780EF00AFFDFED580A80EE201A554890ED700A21EE000AD0ED53
:40398000710AB2EE001A71EE600A80EE801A9FED520A21EE000A8DED130A90F82800062804D19FED4F0A8DED110A1CE0474890F8300091280ED0454890F83000922809D08A
:4039C000424890F83000712804D0404890F83000B82804D19FED420A8DED110A03E09FED410A8DED110A3848D0ED530A9DED110A80EE201A354890ED300A31EE400A8DED69
:403A0000120A9DED130ADFED340AB4EEE00AF1EE10FA10DD9DED120ADFED2F0AB4EEE00AF1EE10FA07DD90F842009FED2F0A0B900DF047F81DE09DED130ADDED120AB4EEC1
:403A4000E00AF1EE10FA0ADD204890F842000B909DED120AB1EE400A0DF033F809E01B4890F842000B909DED130AB1EE400A0DF028F8154890ED541A9DED110A00E0F1E00C
:403A8000C0EE010A114890ED320A30EE800A8DED120A9DED130ADFED100AB4EEE00AF1EE10FA23DD9DED120ADFED0B0AB4EEE00AF1EE10FA1ADD90F842009FED070A0B9006
:403AC0000DF023F82CE0ABE0381100203021002000007A441B0700200000C8425F43BA393333B33F3333B33E0000C8C29DED130ADDED120AB4EEE00AF1EE10FA08DDFE4838
:403B000090F842000B909DED120A0CF0FEFF07E0F94890F842000B909DED130A0CF0F5FF0820F64981F8DC01062081F8DD01002081F8DF014FF47A7048600E9888609FEDBB
:403B4000F00A084680ED500A0BE09FEDED0AEB4880ED500A0920E94981F8DC012B2081F8DA015DE00620E54981F8DD01052081F8DF010A2048600E9888600846D0ED500A53
:403B80001FED2B1A80EE810A8DED030A039830F09DFBCDE904019DED040B00E034E02CF06FFF8DED080BD548D0ED700A1FED381A80EE810A8DED050A059830F087FBCDE959
:403BC00006019DED080B53EC102B9DED060B51EC100B30F085F8CDE90A019DED0A0B51EC100B2FF037FDC549C1F86401084690ED6E0A5FED490A80EE201A80ED5D1AB2EED2
:403C0000000A80ED500A0BE00020BC49A1F8D80181F8DC019FEDBA0A084680ED500A00BF00BF1FE002200C900620B44981F8DD01002081F8DF01192048600E9888609FED4D
:403C4000B00A084680ED500AFEF720F90AE003200C909FEDAB0AA94880ED500AFBF73FFB00E000BF00BFA54890ED500AB5EEC00AF1EE10FA0AD090ED500A8DED0B0A0121BF
:403C800008469DED0B0AF6F722FC0AE09B4890ED500A8DED0B0A002101209DED0B0AF6F716FC0C9815B0BDEC028B00BD10B50124924890F8DA0170BB23F00CFD68B18E493F
:403CC00091F8300005F006FA18B1FDF7AFFD04461FE0FEF7B8F904461BE023F013FDC0B1854890F82800072803D1FEF7CDF804460FE005F011FA28B97F4991F8300005F01B
:403D0000E9F918B1FDF792FD044602E0FDF71AF80446FBF76CF9204602F06BFA774890F8DA0120B1754991F8DA0102F06BFF204610BD10B5714890F8DC010A284CD2DFE827
:403D400000F04C4D20054B21064B4B4E00BF02206A4981F8DD010020086012F087FD674880ED080A90F8E301401C644981F8E301084690F8E3010A2802DD0A2081F8E301F4
:403D800030E000BF0D205D4981F8DD0126F07CF85A4908609FED5A0A084680ED4C0A002081F8E30105F0B8F970B1544890F8E101322804DD3220514981F8E1010BE000209D
:403DC0004E4981F8E10106E04C4890F8E101C01E4A4981F8E10105E000BF00BF00BFFBF76DF800BF00BF47480021016241620020424981F8DA01B6EE000A084680ED500AB2
:403E000010BD10B523F066FC10B302F0F7FE2B2802D1FBF753F81DE0384890F8DB01374981F8DC01062081F8DD01002081F8DF014FF47A70486026F027F8304988609FEDCA
:403E4000300A084680ED500A002081F8DA0101E0FFF76FFF10BDB7EE000A7047274890F8DA01704710B52848FCF7D4F92648FCF756F92548FBF749FA10BD10B52248FCF748
:403E8000C9F92148FCF74BF91F48FBF73EFA10BD1A4890F8DC017047184890F8DD01704710B50424154890F8DC01012804D10620124981F8DC0193E04FF4FA7113480088BF
:403EC00025F0E8FF002871D025F0DEFF0F4908800A4890F8DC01801E07287FD2DFE800F052057E51047E7D0000BF044890F8DD01801E0B2842D20BE03021002038110020BF
:403F000000000000B81200202813002098030020DFE800F00634151F0B1A3434343410000620654981F8DD0129E00C20624981F8DD0124E00420604981F8DD011FE00720A7
:403F40005D4981F8DD011AE005205B4981F8DD0115E0594890F8DC01062807D10320564981F8DC01022081F8DD0106E00520524981F8DC010D2081F8DD0100E000BF00BFBA
:403F80002DE000BF4C4890F8DD01062804D00D2807D00E281ED10BE00D20474981F8DD0119E00E20444981F8DD0114E018E015E0414890F8DC01052807D102203E4981F808
:403FC000DC01062081F8DD0103E008203A4981F8DC0100E000BF00BF01E000E000BF00BF204610BD10B52DED088BB0EE408A05F0A2F818B3F7F768FB00EE100AB8EE400A36
:4040000038EE400A10EE104A204630F05FF941EC1B0BB0EE4B0AF0EE6B0A2CF031FDB0EE40AAF0EE60AA9FED250B53EC102B51EC1A0B2FF0FDFB41EC100B0BE018EE100A85
:4040400030F044F941EC1A0BB0EE4A0AF0EE6A0A2CF016FDB0EE409AF0EE609A51EC190B2FF0F8FA00EE100ABDEC088B10BD01B500BF0122694613480068433007F0DAFA03
:4040800020B99DF80000104981F8430000BF08BD10B52DED020B00BF042269460948006800F5DC7007F0C6FA20B99DED000A064880ED6E0A00BF1CBD381100200000000027
:4040C00000005940FC0300203021002010B5044623F000FB00287DD0092C7CD005DC4CB1032C31D0062C77D158E00B2C75D00C2CF9D1E5E00120FE490870FA208861FA2183
:40410000FB48C16125F0C0FEF94948620121F84880F82810D0ED080AB0EE600AF548007827F01EFF0020F24948604FF47A71F0488160416A0161002101759FEDEF0AEF48DF
:40414000007827F00DFFF5E00120E9490870FA204860FA21E648816025F096FEE44908610121E3480175D0ED030AB0EE600AE348007827F0F5FE0020DD4988614FF47A713A
:40418000DB48C16101694162002180F828109FEDDA0AD848007827F0E3FECBE00120D44908704FF47A7088610021D148C16125F06BFECF4948620121CD4880F82810D0ED25
:4041C000080AB0EE600ACB48007827F0C9FE0020C74903E0AFE011E0ABE03AE048604FF47A71C3488160416A0161002101759FEDC20AC248007827F0B3FE9BE00120BC495B
:4042000008704FF47A7048600021B948816025F03BFEB74908610121B5480175D0ED030AB0EE600AB548007827F09AFE0020B04988614FF47A71AE48C16101694162002176
:4042400080F828109FEDAC0AAA48007827F088FE70E00220A6490870642048600021A448816025F011FEA24908610121A0480175D0ED030AB0EE600AA048007827F070FEA3
:4042800064209B49886100219948C16101694162002180F828109FED980A9648007827F05FFE0020924981F87C000121904880F87D10022180F88B10002180F88C1039E040
:4042C00002208B4908704FF47A70486001468848816025F0D9FD86490861012184480175D0ED030AB0EE600A8448007827F038FE4FF47A707E49886101467D48C161016924
:404300004162002180F828109FED7B0A7948007827F026FE0020764981F87C000121744880F87D10022180F88B10002180F88C1000E000BFDDE223F0E5F90028FAD0102CE5
:4043400075D2DFE804F074083E75ABFA74E7E6E5E47474E3E2E10120654908704FF4FA70C86201466248016325F08EFD6049886301215F4880F83C106148007823F0ECF982
:4043800000205B4948604FF47A7159488160816B0161002101750020554908644FF47A7153484164816BC164002180F850105348007823F0D1F900215248007823F0CCF95F
:4043C00096E201204A4908704FF4FA70086401464748416425F058FD4549C8640121444880F850104748007823F0B6F90020404948604FF47A713E488160C16C016100217C
:40440000017500203A49C8624FF47A7138480163C16C8163002180F83C103848007823F09BF900213648007823F096F960E25EE201202F4908704FF4FA70486001462C4836
:40444000816025F021FD2A4908610121284801752A48007823F080F90020254908644FF47A71234841640169C164002180F8501000201F49C8624FF47A711D4801630169FB
:404480008163002180F83C101D48007823F064F900211C48007823F05FF929E20120144908704FF4FA70C86201461148016325F0EBFC0F49886301210D4880F83C101048D0
:4044C000007823F049F94FF4FA700949086401460748416425F0D8FC0549C8640121044880F850100748007823F036F9002013E0481600203507002000000000360700204D
:404500008D07002084070020B5E172E129E1EEE0B7E080E049E010E0F74948600021F648816025F0B1FCF44908610021F2480175F248007823F010F9DAE10120EE49087091
:404540003220C8623221EC48016325F09DFCEA4988630121E84880F83C10E948007823F0FBF83220E44908643221E348416425F08BFCE149C8640121DF4880F85010E148F9
:40458000007823F0E9F80020DB4948600021DA48816025F079FCD84908610021D6480175D648007823F0D8F8A2E10120D24908704FF47A70C8620021CF48016325F064FC9E
:4045C000CD4988630121CC4880F83C10CC48007823F0C2F80020C84948604FF47A71C6488160816B0161002101750020C24908644FF47A71C0484164816BC164002180F870
:404600005010BE48007823F0A7F80021BD48007823F0A2F86CE10120B74908704FF47A7008640021B448416425F02EFCB249C8640121B14880F85010B248007823F08CF8FC
:404640000020AD4948604FF47A71AB488160C16C0161002101750020A749C8624FF47A71A5480163C16C8163002180F83C10A348007823F071F80021A148007823F06CF8CD
:4046800036E101209C4908704FF47A70486000219948816025F0F8FB974908610121964801759648007823F057F80020924908644FF47A71904841640169C164002180F8F4
:4046C000501000208C49C8624FF47A718A48016301698163002180F83C108948007823F03BF800218748007823F036F800E10120814908704FF47A70C86200217E48016386
:4047000025F0C2FB7C49886301217B4880F83C107B48007823F020F84FF47A707649086400217548416425F0AFFB7349C8640121714880F850107348007823F00DF8002048
:404740006D49486000216C48816025F09DFB6A4908610021684801756848007822F0FCFFC6E00220644908704FF47A70486000216148816025F088FB5F49086101215E4802
:40478000017500215D48007822F0E6FF4FF47A705949C86200215848016301698163012180F83C1000215648007822F0D5FF4FF47A705149086400214F4841640169C164C0
:4047C000012180F8501000214E48007822F0C4FF0020494981F87C000221474880F87D10032180F87E1080F88B10002180F88C107EE00220404908706420486000213E4897
:40480000816025F041FB3C49086101213A4801753A48007822F0A0FF64203749C86200213548016301698163012180F83C103448007822F091FF64202F49086400212E489A
:4048400041640169C164012180F850102D48007822F082FF0020284981F87C000221264880F87D10032180F87E1080F88B10002180F88C103CE001201F4908704FF47A70B2
:40488000486001461C48816025F0FEFA1A49086100211948017501211948007822F05CFF4FF47A701449C86200211348016325F0EBFA1149886301210F4880F83C10104823
:4048C000007822F049FF00200B4908644FF47A710948416425F0D8FA0749C8640021064880F850100748007822F036FF00E000BF00BF0548047010BD481600203607002063
:404900008D070020840700209A03002001B59DF8000000EE100AB8EE400AFE4880ED030A9DF8000000EE100AB8EE400AF94880ED080A00BF01226946F7480068403006F06D
:4049400079FE20B99DF80000F44981F8400000BF0120F349087008BD08B506464FF4C8774FF000080121EF4880F8A8119421E9482AF001FF307818B94620FFF7C7FF11E01B
:40498000E64890F84050642D03DD6420FFF7BEFF08E00A2D03DA0A20FFF7B8FF02E02846FFF7B4FF0020DB4981F88D0022F092FEE8B10020FFF78AFBDB48DFEDDC0A9FEDBC
:4049C000DC0A01230022DB490090DB48007826F029FFD548DFEDD50A9FEDD50A01230022D6490090D648007826F01CFF05E022F089FE10B10120FFF769FB0321C94880F8A8
:404A0000A81100BF012239464FF6FF70DFF834C300DF25F039FA0446BE4890F88D00002874D1012017F0D5FB18BB22F053FE68B1C548007818B9BA480078012805D10020AB
:404A4000FFF744FB0020B64908709EE022F05AFE0028FAD0BC480078052803D1B04800780128F2D10520FFF731FB0020AC4908708BE001F0FAFA20BB22F02CFE70B1B24861
:404A80000078092803D1A648007801287DD10920FFF71CFB0020A249087076E022F032FE002872D0A8480078022803D19C48007801286AD10220FFF709FB00209849087026
:404AC00063E022F007FE70B19F480078062803D193480078012858D10620FFF7F7FA00208F49087051E022F00DFE28B396480078042803D18A480078012846D10420FFF795
:404B0000E5FA0020864908703FE0FFE7814890F88D00012823D122F0DDFD70B18A4800780C2803D17E48007801282ED10C20FFF7CDFA00207A49087027E022F0E3FD20B35A
:404B4000814800780D2803D17548007801281CD10D20FFF7BBFA00207149087015E06D4890F88D00022810D122F0CCFD68B1764800780F2803D16A480078012805D10F201F
:404B8000FFF7A4FA00206649087062480078012802D002287ED115E15E48007D28BB5D48406810B35B480169204625F0A4F95949896888423FD3012156480175046122F037
:404BC00089FD48B15348D0ED030AB0EE600A5C48007827F0C5F92EE022F094FD10B301215748007822F0B8FD25E04A48007D012821D148488068A8B146480169204625F0F1
:404C00007AF944494968884215D3002141480175046122F05FFD30B19FED4C0A4848007827F09EF907E022F06DFD20B100214448007822F091FD374890F82800C8B935487F
:404C40008069B0B13348416A204625F054F93149C96988422BD301212E4880F828104462D0ED080AB0EE600A3348007827F078F91DE0284890F82800012818D12548C06983
:404C8000A8B12448416A204625F035F921498969884200E0F6E10AD300211E4880F8281044629FED2A0A2448007827F059F9194890F85000A8B91748006C90B11548C16C07
:404CC000204625F018F91349496C884245D30121104880F85010C4641D48007822F03CFD3BE00C4890F85000012836D10948406C80B30848C16C204625F0FDF80549096C3C
:404D000088422AD30021034880F85010C4641048007820E048160020FC030020302100209B0300207852002080EC00200000FA4300247449001C00403507002000200040F8
:404D400036070020612904089A030020000000008407002001E022F0FFFCD84890F83C00A8B9D648C06A90B1D448816B204625F0C2F8D249096B884223D30121CF4880F8DF
:404D80003C108463CE48007822F0E6FC19E0CB4890F83C00012814D1C848006B88B1C748816B204625F0A7F8C449C96A884208D30021C24880F83C108463C148007822F049
:404DC000CBFC5FE1BD4890F88C107C30405C78BBBA48007D01282CD1B8480169204625F08AF8B6494968884221D30021B3480175046122F06FFC30B11FED2C0AB148007886
:404E000027F0AEF80DE022F07DFC50B11FED310AAC48007827F0A4F80021AA48007822F09BFCA6488068002801D14FF00108C1E00BE0A2480169204625F05DF89F49896801
:404E4000884201D34FF00108B4E09C4890F88C107C30405C01282BD1984890F8280001281AD19648416A204625F045F893498969884210D30021914880F8281044621FED87
:404E80004D0A9148007827F06BF88C48C069002801D14FF001088DE08848416A204625F02AF88649C969884201D34FF0010881E0824890F88C107C30405C022836D17F4896
:404EC00090F83C00012825D17C48816B204625F012F87A49C96A88426CD30021774880F83C1084637648007822F036FC22F00AFC50B100217248007822F02EFC1FED6D0A6B
:404F00006F48007827F02CF86C48006B90BB4FF001084FE06948816B204624F0ECFF6749096B884246D34FF0010843E0634890F88C107C30405C03283CD1604890F85000E3
:404F400001282CD15D48C16C204624F0D4FF5B49096C88422ED30021584880F85010C46422F0B8FB38B11FED870A5748007826F0F7FF0EE01EE022F0C5FB50B11FED8D0A77
:404F80005248007826F0ECFF00215048007822F0E3FB4A48406C68B94FF001080AE04748C16C204624F0A7FF4449496C884201D34FF00108B8F1010F63D14FF000083F486D
:404FC00090F88C00401CC1B23C4880F88C1090F88C1090F88B00814203DB0021374880F88C10364890F88C107C30405C022809D10121324880F83C1084633148007822F072
:40500000ABFB3EE02D4890F88C107C30405C01280DD10121294880F828104462D0ED080AB0EE600A2848007826F09AFF29E0234890F88C107C30405C032809D101211F48FF
:4050400080F85010C4642148007822F085FB18E001211A480175046122F03CFB48B11748D0ED030AB0EE600A1648007826F078FF07E022F047FB20B101211248007822F07E
:405080006BFB00BFBEE42DE9F04106460C4617469846069D2078642803DD6420FFF736FC09E020780A2803DA0A20FFF72FFC02E02078FFF72BFCBDE8F081000048160020B0
:4050C0008D07002036070020350700208407002070B544201CE0C41700EBD4646511CD4C54F82540C51700EBD5656D11A0EB45160125B5402C40C51700EBD5656D11A0EBDF
:4051000045160125B540AC4200D103E0411EC8B20028E0DC00BF70BD30B5C31700EBD3635C11BC4B183353F824300246C41700EBD4646411A0EB44150124AC402343014613
:40514000C41700EBD4646511B24C183444F8253030BD13B50C4600BFAF49096801F5B07108190122694606F065FA18B99DF80010AA48015500BF1CBD13B50C4600BFA64934
:40518000096801F25F2108190122694606F052FA20B99DF80010A148FF30015500BF1CBD70B504469E480470E21704EBD2625311984A52F823202146E31704EBD3635B11A8
:4051C000A4EB43150123AB409A432046E31704EBD3635D118F4B43F82520E21704EBD26253118C4A0C3252F82320E31704EBD3635B11A4EB43150123AB409A43E31704EB27
:40520000D3635D11834B0C3343F82520E21704EBD26253117F4A183252F82320E31704EBD3635B11A4EB43150123AB409A43E31704EBD3635D11774B183343F82520002085
:40524000FFF79AFF70BD30B50146CB1701EBD3635C11704B53F82430CC1701EBD4646411A1EB44150124AC4023400BB1012030BD0020FCE76B49087070476A480078704715
:4052800070B52DED048B04460025452C70D2DFE804F02324292E2F303139414951596169737C8891ACB1FFFEFDFCFBFAF9F8F7F6F5F4F3F2F1F0EFEEEDECEBEAE9E8E7E6D8
:4052C000E5E4E3E2E1E0DFDEDDDCDBDAD9D8D7D6D5D4D3D2D19DD00003E30EF0D5FD80F00105FEE222F0EEF980F00105F9E2F8E2F7E2F6E20FF09CFC18B1F8F72FF800B142
:405300000125EEE20FF094FC18B1F8F71FF800B10125E6E20FF08CFC18B1F8F727F800B10125DEE20FF084FC18B1F8F730F800B10125D6E20FF07CFC18B1F8F720F800B19F
:405340000125CEE20FF074FC18B1F8F728F800B10125C6E211F007FC012800D100E000200546BEE211F0FFFB032802D1012001E0B6E200200546B4E22B4890F838000128B8
:4053800000D100E000200546ABE20FF051FC38B1254890F8380008B9012000E0002005469FE2214890F89000012800D100E00020054696E20FF03CFC38B11B4890F890005B
:4053C00008B9012000E0002005468AE2164890F83800022804D0144890F89000022801D1012000E0002005467BE20CF078F980F0010576E20D48007DD0B90648001F006953
:4054000000F48020B0F5802F43D002F039FB78B101203FE0F41800200404002030270020A4030020A503002054290020E82B00202FE051E24CE23EE210E203E2FAE1EDE1A8
:40544000E1E1D5E1CCE1C3E1B7E1AEE1A2E199E190E187E17EE175E16CE163E15AE151E148E13FE136E12AE11EE10CE1E3E0D6E0C9E0BCE0AFE0A2E095E08BE080E075E0F8
:405480005DE050E043E032E025E018E00FE00BE002E00020054624E2F748007D08B9012000E0002005461CE2F448057819E2F5F7F7F808B1012000E00020054611E20EF094
:4054C00077FAB0EE408A9FEDEE1ADFEDEE0A0EF0EEF9054605E20EF06BFAB0EE408A9FEDEA1ADFEDEA0A0EF0E2F90546F9E102F0ADFFB0F57B4F07DB02F0A8FF4FF6FF710E
:40550000884201DA012000E000200546E9E102F05EFF28B1DE488078FE2801D0012000E000200546DDE1DA488078FE2806D0F7F736FE18B101250020D6490872D1E1D4487B
:405540008078FE2805D0D448007810B103F06CFD20B101251C20FFF78DFE06E0FFF78DFE1C2802D10020FFF785FEBAE1CB48007800F0A40008B1012000E000200546B0E14C
:40558000C648007800F0580008B1012000E000200546A6E1C2480088102801D0012000E0002005469DE10EF052FAB0EE408A9FEDB41ADFEDB60A0EF07AF9054691E10EF028
:4055C0004EFAB0EE408A9FEDAE1ADFEDB00A0EF06EF9054685E10EF04AFAB0EE408A9FEDA81ADFEDAA0A0EF062F9054679E10EF007FAB0EE408A9FEDA21ADFEDA40A0EF06E
:4056000056F905466DE10DF070FAB0EE408A9FED9C1ADFED9E0A0EF04AF9054661E10EF0F7F9B0EE408A9FED961ADFED980A0EF03EF9054655E122F04DF818B3F5F787FCE8
:40564000B0EE408AF5F758FC38EE400A10EE106A30462EF03BFE41EC190BB0EE490AF0EE690A2BF00DFAB0EE408AF0EE608A9FED8D0B53EC102B51EC180B2EF02FFC00D2CF
:40568000012500BF2DE1F5F762FCDFED880AB4EEE00AF1EE10FA04DDF4F75DFA08B1012000E0002005461CE102F0EAF920B903F04FF908B9012000E00020054611E102F09B
:4056C000DFF920B108F0CEFC08B1012000E00020054606E10FF0ACFA18B103F0AFFD80F00105FEE0F4F7E7FF08B1012000E000200546F6E0F4F7FEFF08B1012000E0002044
:405700000546EEE0F5F783F808B1012000E000200546E6E0F5F7BBF808B1012000E000200546DEE0F5F7F0F808B1012000E000200546D6E0F5F73CF908B1012000E00020D2
:405740000546CEE0F5F774F908B1012000E000200546C6E0F5F7A8F908B1012000E000200546BEE0F5F7DCF908B1012000E000200546B6E0F5F714FA08B1012000E000206C
:405780000546AEE0F5F748FA08B1012000E000200546A6E00FF04CFA30B1F5F7B1FA08B1012000E0002005469BE0F5F7C7FA08B1012000E00020054693E00FF039FA30B182
:4057C000F5F7DAFA08B1012000E00020054688E0F5F7F8FA08B1012000E00020054680E0F5F70EFB08B1012000E00020054678E00FF01EFA30B1F5F721FB08B1012000E0CD
:40580000002005466DE00FF013FA30B1F5F734FB08B1012000E00020054662E00EF0B3F906460EF033FA06430EB1012000E00020054656E00EF062FA08B1012000E0002042
:4058400005464EE00FF0F4F938B108F0A1FE012803D103F045FC00B9012542E0F4F7BFFE28B9F5F7AEFB10B9F5F7C5FB00B303F037FCE8B901201CE0002C0020E90300208F
:4058800000FF7F4700A0254600007A460000000098DA00206832002048050020F9030020CA070020000000000070A7400000FA450020054615E00EF0C7FA20B9FE48007846
:4058C00022F04CFB08B1012000E00020054608E003F07AF8054604E024F023FC054600E000BF00BF05B100BF3DB9F4480078002807DDF2480078844203D10120BDEC048B02
:4059000070BD0020FAE74FF00008C1464FF0010A4FF0500B0321EA4880F8B810002491E0E848005D04EB840101EBC401E64A02EB810189680870E348FF30005D00287FD0F4
:40594000E21704EBD2625311E04A52F82320E31704EBD3635B11A4EB431C012303FA0CF31A43E31704EBD3634FEA631CD74B43F82C20E21704EBD2625311D44A0C3252F854
:405980002320E31704EBD3635B11A4EB431C012303FA0CF31A43E31704EBD3634FEA631CCA4B0C3343F82C2004EB840000EBC400C54901EB8000007BE0B1E21704EBD26238
:4059C0005311C24A183252F823202146E31704EBD3635B11A4EB431C012303FA0CF31A432046E31704EBD3634FEA631CB74B183343F82C2024F048FAB54941F8240000BF82
:405A0000E21704EBD2625311B04A243252F823202146E31704EBD3635B11A4EB431C012303FA0CF39A432046E31704EBD3634FEA631CA64B243343F82C2000E000E000BFA1
:405A4000601CC4B2452CFFF66BAF4FF47A60DFF884C200DF9A48D0F8DC100120DFF878C200DF4FF47A60DFF86CC200DF00BF002259460320DFF864C200DF0646022E21D106
:405A8000DFF85CC200DF074607F00200D0B1002416E0002004EB840101EBC4018A4A02EB81018968087004EB840101EBC40102EB8101896808782146FFF74BFB601CC4B2A6
:405AC000452CE6DB0024A9E22046FFF7D9FB05462046FFF7B8FBA8427ED0002D7DD1A946E31704EBD3634FEA631C784B0C3353F82C304FEAE47C04EBDC6C4FEA6C1CA4EBF9
:405B00004C1E4FF0010C0CFA0EFC03EA0C034FEAE47C04EBDC6C4FEA6C1CA4EB4C1E4FF0010C0CFA0EFC634501D04FF0010904EB840000EBC400644901EB800090F8330005
:405B400000F0010008B14FF0010904EB840000EBC4005D4901EB800090F8330000F0020020B10BF078FC08B14FF0010904EB840000EBC400544901EB800090F8330000F039
:405B8000040038B108F076FA10B921F0CEFD08B14FF0010904EB840000EBC4004A4901EB800090F8330000F0080020B1BAF1000F01D04FF0010904EB840000EBC4004249C3
:405BC00001EB800090F8330000F0100038B14548005D012803D101E00FE00FE08146B9F1010F0AD100203F4908554FF001082046FFF7D6FA3720F7F7B3FC02E1E31704EB5A
:405C0000D3634FEA631C314B53F82C304FEAE47C04EBDC6C4FEA6C1CA4EB4C1E4FF0010C0CFA0EFC03EA0C034FEAE47C04EBDC6C4FEA6C1CA4EB4C1E4FF0010C0CFA0EFC8B
:405C40006345DAD000202749085500BF01F018FFE8B1E21704EBD26253111C4A243252F823202146E31704EBD3635B11A4EB431C012303FA0CF31A432046E31704EBD363DA
:405C80004FEA631C114B243343F82C2034E0E21704EBD26253110D4A243252F823202146E31704EBD3635B11A4EB431C012303FA0CF39A43204617E09A070020A603002060
:405CC0007852002030270020B4440408F4180020DC170020A12804080129040861290408A928040895170020E31704EBD3634FEA631CF84B43F82C20E21704EBD262531195
:405D0000F44A243A52F82320E31704EBD3635B11A4EB431C012303FA0CF31A43E31704EBD3634FEA631CEB4B243B43F82C2024F0ABF8E94941F8240004EB840000EBC400E9
:405D4000E64901EB800080680078401C04EB840101EBC401E14A02EB81018968087004EB840000EBC400114601EB8000806800787E2808DD7E2004EB840101EBC40102EB24
:405D800081018968087000BF00BF01F079FE01281BD1E21704EBD2625311CE4A52F823202146E31704EBD3635B11A4EB431C012303FA0CF31A432046E31704EBD3634FEABD
:405DC000631CC44B43F82C201AE0E21704EBD2625311C04A52F823202146E31704EBD3635B11A4EB431C012303FA0CF39A432046E31704EBD3634FEA631CB64B43F82C20DB
:405E000000BF002D7DD0E21704EBD2625311B14A183A52F82320E31704EBD3635B11A4EB431C012303FA0CF31A40002A53D104EB840000EBC400A94901EB8000406AE8BBC1
:405E4000E21704EBD2625311A24A183A52F82320E31704EBD3635B11A4EB431C012303FA0CF31A43E31704EBD3634FEA631C994B183B43F82C204FF0010804EB840000EBA6
:405E8000C40001EB8000806800787E2811DA04EB840000EBC40001EB800080680078401C04EB840101EBC4018C4A02EB81018968087021460120FFF75FF900E00CE004EB13
:405EC000840101EBC401854A02EB8101896808782146FFF73EF95BE004EB840202EBC4027E4B03EB8202516A7B4A52F8240023F0D1FFE8B3E21704EBD2625311754A183A8E
:405F000000E083E052F82320E31704EBD3635B11A4EB431C012303FA0CF31A43E31704EBD3634FEA631C6B4B183B43F82C204FF0010804EB840000EBC400684901EB8000AD
:405F4000806800787E2811DA04EB840000EBC40001EB800080680078401C04EB840101EBC4015E4A02EB810189680870214600E00EE00120FFF700F904EB840101EBC401D7
:405F8000564A02EB8101896808782146FFF7E1F804EB840202EBC402504B03EB8202127BA2B3E21704EBD26253114A4A0C3A52F82320E31704EBD3635B11A4EB431C012390
:405FC00003FA0CF31A400ABB01F05AFD10B901F00CFCE0B104EB840000EBC4003F4901EB8000806A68B104EB840202EBC4020B4603EB8202916A384A52F8240023F04AFFA0
:4060000020B12046FFF788F84FF0010804E02046FFF782F84FF00108601CC4B2452CFFF653ADB8F1010F0BD12D48D0F8DC100120DFF8B0C000DF4FF000083720F7F790FAF6
:406040004FF0000AFFF744F8044610E5002108E02048243850F8210008B101207047481CC1B20329F4DB0020F8E7002108E019480C3850F8210008B101207047481CC1B24F
:406080000329F4DB0020F8E770B544201DE0C41700EBD46465110F4C0C3C54F82540C51700EBD5656D11A0EB45160125B5402C40C51700EBD5656D11A0EB45160125B5402C
:4060C000AC4200D103E0411EC8B20028DFDC00BF70BD000018190020DC170020B4440408785200200129040870B5002401F0C8FC78B344242AE0E31704EBD3635D11364B25
:4061000053F82530E51704EBD5656D11A4EB45160125B5402B40E51704EBD5656D11A4EB45160125B540AB420ED104EB840303EBC4032A4D05EB830393F83330102B03D123
:40614000274B1B5D03B903E0601EC4B2002CD2DC00BF204670BD0121214A1154704701460020FF2906DA1E4A525C0AB1012200E000221046704700B5002304E01846FFF74B
:40618000EAFF581CC3B2452BF8DB00BD0EB5154A07CA8DE807001CF0F9FB1DF08BFC0C226946FF201CF0BEFB0EBD014601EB810000EBC100094A52F820007047014601EB77
:4061C000810000EBC100054A02EB800000797047704705490870704700190020B444040895170020B8520408A6030020FE48007B7047FD490873704770B52DED068B044660
:406200000D46284623F068FE00EE100AB8EE400AB0EE408A9FEDF50AC8EE000AB0EE608A94ED000AD4ED020A00EE880ADFEDF00A68EE200A20EE200A10EE101A08462EF007
:4062400045F841EC1A0BB0EE4A0AF0EE6A0A2BF0D7FAB0EE409AF0EE609A51EC190B2DF0F9F908EE100A94ED040A20EE080AB0EE408AB0EE480ABDEC068B70BD10B52DED42
:40628000088BF0EE409AF0EE608A04469FEDD90AF0EE40AA9FEDD50AC0EE290AB0EE608AB1EE000A28EE800AC0EE080AB0EE60AA9FEDD00AB0EE40BA204623F00DFEBCEE99
:4062C000C80A10EE101AB0FBF1F201FB120000EE100AB8EE400AB0EE409AB5EE000A28EE000AB4EEC90AF1EE10FA15D8B6EE080A28EE000AB4EEC90AF1EE10FA0CDDBFEEB6
:40630000000A2AEE000AB0EE40AAB0EE000A28EE800AB0EE40BA0EE0B6EE080A28EE000AB4EEC90AF1EE10FA05D8B9EE000A28EE800AB0EE40BAB0EE4B0A0AEE090AF0EE05
:4063400040AAB0EE6A0ABDEC088B10BD2DE9F0412DED028B05460F4690460024002600BF32E0322108FB01F000EE100AB8EEC00ADFED9E0A80EE201A05F1300000EB840029
:4063800090ED000A30EE410A05F1300000EB840080ED000A08FB01F000EE100AB8EEC00ADFED920A80EE201A05F1700000EB840090ED000A30EE410A05F1700000EB8400CB
:4063C00080ED000A601CC4B2082CCADB0024D8E007F1300000EB840090ED000A07F1700000EB8400D0ED000A30EE600AF0EE000A20EE200AB0EE408A05F1300000EB84001E
:4064000090ED000A07F1300000EB8400D0ED000A30EE600A05F1900000EB860080ED000A05F1900000EB860090ED000AC0EE080A9FED710A20EE800A05F1CC0000EB860071
:4064400080ED000A05F1500000EB840090ED000A05F1100000EB8400D0ED000A30EE600A07F1500000EB8400D0ED000A07F1100000EB840090ED001A70EEC10A80EE201A48
:4064800005F5847000EB860080ED001AB7EE000AC0EE080A05F5A27000EB8600C0ED000A701CC6B20F2E6ADA07F17000611C00EB810090ED000A07F1300000EB8400D0EDA2
:4064C000000A30EE600AF0EE000A20EE200AB0EE408A05F1700000EB810090ED000A07F1700000EB8100D0ED000A30EE600A05F1900000EB860080ED000A05F1900000EB27
:40650000860090ED000AC0EE080A9FED3B0A20EE800A05F1CC0000EB860080ED000A05F1500000EB810090ED000A05F1100000EB8400D0ED000A30EE600A07F1500000EB4B
:406540008100D0ED000A07F1100000EB840090ED001A70EEC10A80EE201A05F5847000EB860080ED001AB7EE000AC0EE080A05F5A27000EB8600C0ED000A701CC6B2601CEB
:40658000C4B2082CFFF624AF1C4B0F221C4901F13C0013F02EFD1B4B0F2219493C3901F1780013F026FD154890ED010A0E4880ED1D0A124890ED000A0B4880ED230A11481C
:4065C00090ED010ADFED100A30EEC00AD0ED000A80EE201A044880ED261A0F210848783813F0EDFC004811E03819002000007A44DB0FC940000000000000B443AC030020A0
:40660000E81A0020B40300200000344380ED200ABDEC028BBDE8F08170B52DED028B0446B0EE408A0D46207800F0100000280AD094ED020A84ED030A84ED028AA07808284C
:4066400002D10420208086E0207800F00100D8B394ED020AD4ED030AB4EEE00AF1EE10FA20DD94ED020AFE48817804F1500000EB810080ED000AFB49486823F02DFC00EE2A
:40668000100AB8EE400A5FED270A80EE201AF448817804F1700000EB810080ED001A0020E07002E0E078401CE070E0782179884251DD208840F002002080208820F00100AB
:4066C00020800020E07046E0FFE7207800F00200F0B394ED020AD4ED030AB4EEE00AF1EE10FA1ED294ED020AA17804F1100000EB810080ED000ADB49486823F0EDFB00EE46
:40670000100AB8EE400A5FED470A80EE201AA17804F1300000EB810080ED001A0020E07002E0E078401CE070E0782179884212DD208840F001002080208820F00200208005
:40674000A078401CA0700020E0700DB1207900E001E0401E2071BDEC028B70BD10B52DED028BF0EE408AB0EE608ABE49486823F0B3FBB0F57A7F0BD90121B0EE480ABA4811
:40678000FFF74AFF0021B0EE680AB548FFF744FFB548008804280DD1B1480088042809D10222AF49B048FFF7D1FD2020AE490880AB490880BDEC028B10BD70B52DED0C8B31
:4067C000044602F074FD60B1F6F726FEB0EE408AD4ED098AF1EE009AB1EE00AAB0EE009A57E002F09DFD40B3F4F772FF0546F4F773FF281A00EE100AB8EEC00ADFED9B0A2F
:4068000020EE200AB0EE40BAF4F7D8FFDFED980A20EE208A94ED090ADFED950A60EE208AB1EE000A6BEE009AB1EE000A2BEE00AAB0EE000A2BEE009A2BE00FF0BDFFB0EEE2
:40684000408A8C4991F8280091ED0F0AF0EE400AB0EE480A0FF0B4FEDFED870A20EE200AB0EE408A834991F8280091ED0F1AF0EE410A94ED091AB0EE410A0FF0A1FEDFED27
:406880007E0A60EE208AF0EE009AB0EE00AAB7EE009A4020005D40B994ED0B0A38EEC00A84ED0E0A01214020015519EE900A2DF00DFD41EC1B0B94ED0B0A30EE480A10EE9D
:4068C000101A08462DF002FD41EC1D0BB0EE4D0AF0EE6D0A2AF0D4F8B0EE40CAF0EE60CA53EC1B2B51EC1C0B2DF0F8FA0ED24C20005D58B9606823F0EFFA00EE100AB8EEAB
:40690000400A84ED110A01214C2001551AEE100A2DF0DCFC41EC1B0B38EEC80A10EE101A08462DF0D3FC41EC1C0BB0EE4C0AF0EE6C0A2AF0A5F8B0EE40DAF0EE60DA53EC77
:406940001B2B51EC1D0B2DF08FF90ED25820005D58B9606823F0C0FA00EE100AB8EE400A84ED140A01215820015519EE100A2DF0ADFC41EC1B0B38EEC80A10EE101A08464D
:406980002DF0A4FC41EC1C0BB0EE4C0AF0EE6C0A2AF076F8B0EE40DAF0EE60DA53EC1B2B51EC1D0B2DF09AFA0DD8002164200155607B324951F8200000EE100AB8EE400AF4
:4069C00084ED170A31E019EE100A2DF07FFC41EC1B0B38EEC80A10EE101A08462DF076FC41EC1C0BB0EE4C0AF0EE6C0A2AF048F8B0EE40DAF0EE60DA53EC1B2B51EC1D0B3B
:406A00002DF032F911D26420005D70B9012164200155606823F060FA00EE100AB8EE400A84ED170A23F030FAA06078EEC8AA94ED0E0AB5EEC00AF1EE10FA0BD2B4EEE88A71
:406A4000F1EE10FA06D294ED1B0AB4EEEA0AF1EE10FA24D394ED0E0AB5EEC00A10E00000601B002038190020E019002017B7D1380AD7233C30210020E02E6542C4520408BF
:406A8000F1EE10FA25DDB4EEE88AF1EE10FA20DD94ED1B0AB4EEEA0AF1EE10FA19DDC4ED1BAA94ED1B0A10EE101A08462DF00EFC41EC1C0BB0EE4C0AF0EE6C0A29F0E0FF89
:406AC000B0EE40BAF0EE60BA51EC1B0B2CF0C2FDA066BDEC0C8B70BD00200022002100BF33E0FE4B03EB820393ED000AB5EEC00AF1EE10FA01D14B1C99B2F84B403303EB5C
:406B0000820393ED000AB5EEC00AF1EE10FA01D14B1C99B2F24B03EB820393ED000AB5EEC00AF1EE10FA01D14B1C99B2EC4B403303EB820393ED000AB5EEC00AF1EE10FA5B
:406B400001D14B1C99B2531CDAB2082AC9DB00224FE0E44B93ED1D0ADFEDE30AB4EEE00AF1EE10FA06DC93ED1D0AB5EEC00AF1EE10FA01D24B1C99B2DA4B93ED230ADFED69
:406B8000DA0AB4EEE00AF1EE10FA08DC93ED230ADFEDD60AB4EEE00AF1EE10FA01D24B1C99B2D04B93ED260ADFEDCF0AB4EEE00AF1EE10FA06DC93ED260AB5EEC00AF1EE82
:406BC00010FA01D24B1C99B2C64B93ED200ADFEDC60AB4EEE00AF1EE10FA06DC93ED200AB5EEC00AF1EE10FA01D24B1C99B2531CDAB20F2AADDB01B901207047B94890F8FC
:406C0000A4007047B74981F8A4007047B548407B0C2823D0B348407B0B281FD0B148407B07281BD0AF48407B112817D0AD48407B082813D0AB48407B0A280FD0A948407BA0
:406C400004280BD0A748407B052807D0A548407B0F2803D0A348407B102801D1012070470020FCE79F48407B08281BD09D48407B042817D09B48407B052813D09948407B68
:406C80000A280FD09748407B0B280BD09548407B0F2807D09348407B102803D09148407B112801D1012070470020FCE78D48407B082817D08B48407B042813D08948407B8A
:406CC00005280FD08748407B0A280BD08548407B0B2807D08348407B102803D08148407B0F2801D1012070470020FCE77D48407B082803D07B48407B0A2801D10120704789
:406D00000020FCE770B5002428F0FEF9002872D101F05DFB18B10720FFF774FF80E00AF0DEFC30B9FFF7E2FF18B90220FFF76AFF76E019F0EBFDB5EEC00AF1EE10FA06D230
:406D4000FFF7B4FF18B90920FFF75CFF68E019F0DDFDDFED670AB4EEE00AF1EE10FA02D2FFF780FF60B15F48407B0F280CD119F0D1FDDFED5F0AB4EEE00AF1EE10FA03D21C
:406D80000420FFF73FFF4BE019F0C0FDDFED590AB4EEE00AF1EE10FA06DDFFF763FF18B90520FFF72FFF3BE05348007D18B90120FFF728FF34E0F3F712FC50B102F090F9C7
:406DC00038B94848407B0F2803D10D20FFF71AFF26E007F04FFA28B107F04CFA0546FFF711FF1DE0F6F7E4FA30B1F6F7E1FA0546FFF708FF14E01AE007F034F938B139482E
:406E0000407B0B2803D02420FFF7FCFE08E0FFF72CF928B1FFF7FAFE10B90A20FFF7F2FEFFF7ECFE18B10120FFF7E3F90124204670BDC9B1DFED310AC0ED000ADFED300A28
:406E4000C0ED010A2F4AD2ED060AB8EE601ADFED2E1AC1EE210A9FED2D1AC1EE201AC0ED021A80ED040A1CE0DFED290AC0ED000ADFED280AC0ED010A224AD2ED0D0AB8EEB4
:406E8000601ADFED211AC1EE210ADFED231A81EEA01AF6EE000A61EE200AC0ED020A80ED040A704710B501219FED1C0A0D481030FFF7BFFF4FF4C0710848303828F05BFC76
:406EC0004FF4C0710648303828F055FC0A2003493039087102493039087121E0101A0020901B00203819002000409C4500409CC52FDDE43E2FDDE43F002C0020CDCCCC3DE6
:406F000014AE473FC452040800007A447A142E3FCDCC4C3E0000204233331F42C2B8B23E1120FC490880FC49088010BD2DED028B84B04FF47A66A821F84828F01CFC142174
:406F4000F74828F018FC00BF002231460320DFF8D4C300DF0546022D70D1DFF8CCC300DF0446022C6BD1EE480078002867D0EC480078122863DC0120EC490870E848007882
:406F8000E649487322F080FFE4494860E44890ED010A084680ED090A407BE54908700020DE498860084600218166C1660167C165016641668163C163016441648164C1643A
:406FC0000165416581650020D44981F8A4000846407BD84951F82000D04908600846407B122877D2DFE800F0A5505354555609454D4E4CA0412C3A515246C8480021416769
:407000008167C1678030C160016141618161C1610162016041608160FFF744FF04208DF8040003208DF8050005208DF80600022201A9FF201BF076FC04267BE0B0E07DE002
:4070400000219FEDBD0AB5481030FFF7F2FE9FEDBB0AB24880ED090A04266BE09FEDB80AAE4880ED090A042664E0F7F75AFFC82660E000BFF7F755FFFCF7C3FEC82659E0B6
:4070800000BF00BF042655E000BF00BF00BF00BF00BF00BF02F00BF950B1F6F7BDF9B0EE408A9E4880ED0B8A012180F834102BE002F036F978B1F4F781FBDFEDA20A20EE6F
:4070C000200AB0EE408A954880ED0B8A012180F8341019E02DE00FF06FFBB0EE408A9A4991F8280091ED0F0AF0EE400AB0EE480A0FF066FADFED950A20EE200A874880EDE9
:407100000B0A012180F8341004208DF8040003208DF8050005208DF80600032201A9FF201BF000FC042605E04FF4C87607F09BF900E000BF00BF042078490873012C2FD157
:40714000002076494873002101209FED7C0AF3F7BEF90020754908709FED780A704880ED010A9FED760A6D4880ED090A012180F864104FF47A665820F6F7F2F95920F6F7C4
:40718000EFF9FFF733F8042802D10020FFF731F811201AF0F1F8002201A9FF201BF0C2FB5E48407B00287DD05C4A1168506822F071FE18BBFFF71AF804280FD05748407B43
:4071C00007281BD05548407B112817D05348407B0B2813D05148407B0C280FD0FFF792FD60B94E4890F8640001286DD14B49886840F6C41122F04EFE002865D04748407B0F
:40720000022807D04548407B012803D04348407B032819D1414890F8640030B93F4890ED000AB8EE400A80ED170A3C4890F8580030B93A4890ED000AB8EE400A80ED140AF3
:407240005920F6F78DF91FE03448407B06281BD1FFF742FC80B99FED3E0A304880ED1D0A9FED3B0A80ED230A9FED390A80ED260A9FED370A80ED200A0020264908802649C4
:4072800008805820F6F76CF911201AF075F8002022494873FEF7AAFF042802D10020FEF7A8FF00E010E0002101209FED240AF3F70EF900201D4908709FED200A184880EDF7
:4072C000010A4FF47A663FE61448407B122879D2DFE800F0095279F5F3F2F1F0EFEEEDECEBEAE90A0BE81CE200BF02F019F888B3F4F702FB00EE100AB8EE400A074880ED51
:40730000090AD0ED090AB0EE600A0121032008F07CFF2DE0E0190020601B0020381900202419002061290408A9280408A8030020C4030020C45204080000A04200000000F2
:40734000000070420AD7233C30210020E02E6542003C1C46FFE71FED070AFC4880ED090AD0ED090AB0EE600A0121032008F0C3FDF648FFF722FAD4E101F0D2FF88B1F4F7D0
:40738000A3F900EE100AB8EE400AF04880ED090AD0ED090AB0EE600A0121032008F035FF0CE01FED1A0AE94880ED090AD0ED090AB0EE600A0121032008F09DFDE348FFF79B
:4073C000FCF9AEE193E101F072FF68B19FEDE00ADE4880ED090AD0ED090AB0EE600A0121032008F06CFE59E001F09AFF00B3F4F76BF900EE100AF8EE408AF4F765F98046F3
:40740000F4F76AF9A8EB000000EE100AB8EEC00ADFEDD00A40EEC08ACC48C0ED098AD0ED090AB0EE600A0121032008F0EEFE35E020F07BF9D8B1C84890ED640ADFEDC70AC6
:4074400020EE200A5FED410A20EE200AB0EE408A014691F8280091ED0F0AF0EE400AB0EE480A0EF0C9FAB94880ED090A0DE0BA4991F8280091ED0F0AF0EE400A9FEDB80A06
:407480000EF0BAFAB14880ED090AB048D0ED090AB0EE600A0121032008F02DFDAB48FFF78CF93EE1F9E0D0E0E5E00BE104E1F7E001E1F6E0F0E08FE07FE06FE0FFE701F06B
:4074C000F6FE68B19FEDA50AA04880ED090AD0ED090AB0EE600A0121032008F0F0FD59E001F01EFF00B3F4F7EFF800EE100AF8EE408AF4F7EDF88046F4F7E6F8A8EB000064
:4075000000EE100AB8EEC00ADFED920A40EE808A8E48C0ED098AD0ED090AB0EE600A0121032008F072FE35E020F0FFF8D8B18A4890ED650ADFED890A20EE200A5FED7F0AC9
:4075400020EE200AB0EE408A014691F8280091ED0F0AF0EE400AB0EE480A0EF04DFA7B4880ED090A0DE07C4991F8280091ED0F0AF0EE400A9FED7B0A0EF03EFA734880EDAB
:40758000090A7248D0ED090AB0EE600A0121032008F0B1FC6D48FFF710F9C2E06E4890F84210D03000EB8100D0ED000AB0EE600A01210846F2F78BFFB3E0674890F842101C
:4075C000D83000EB8100D0ED000AB0EE600A01210846F2F77CFFA4E05C4841681030FEF70BFE5A4880ED090A5B4991F8280091ED0F1AF0EE410A554991ED091AB0EE410AF6
:407600000EF0FAF9F0EE408A0121032008F073FC4E4890F82900B8B100204C4981F829000FF020F9F0EE408A03214F4810F01BF94D4890ED001AF0EE410A444890ED091AEE
:40764000B0EE410AFFF78AF86BE0404948684749D1ED000A464991ED000AFEF70FFE3B4880ED090AD0ED090AB0EE600A01210846F2F72DFF55E0354841681030FEF7BCFD0B
:40768000324880ED090AD0ED090AB0EE600A01210846F2F71CFF44E000BFFCF707FB40E000BF2A48D0ED090AB0EE600A01210846F2F70DFF35E034E006F0F7FD8046FEF750
:4076C00098FD2EE0214A083202F11C0101F18000F9F708FA8046FEF78CFD1C48D0ED090AB0EE600A01210846F2F7F1FE19E00020164948730873002101201FEDF00AF2F727
:40770000E6FE00201B4908701FEDF40A1A4880ED010A002201A9FF201BF004F94FF47A6600BF00BFFEF762FD04287FF4CCAD4FF4FA71384622F0AEFB00283FF4C4AD22F0C0
:40774000A3FB0746112019F017FEBCE53819002000008CC23333333F3021002000008C42C2B8B2BEC2B8B23EBC030020CC030020C8030020A80300202419002070B52DEDE4
:40778000028B0446B0EE408A0025B5EEC08AF1EE10FA0AD04CB1122C07DCAF4890ED010AB4EE480AF1EE10FA0DD1AC48D0F890110120DFF8ACC200DF9FEDAA0AA64880ED20
:4077C000010A00250DE00CB1A3480470A24880ED018AA248D0F890110220DFF884C200DF01252846BDEC028B70BD9F480078704701209E4981F8290070477A2303709B4B99
:40780000D3ED0E0A9FED9A0AB2EE041A00EE810ABDEEC00A10EE103A1AB24270130A8370924B93ED110ABCEEC00A10EE103A99B2C1700B0A03718D4B93ED140ABCEEC00A9B
:4078400010EE103A99B241710B0A8371874B93ED170ABCEEC00A10EE103A99B2C1710B0A0372824BD3ED1A0A9FED810AB2EE041A00EE810ABDEEC00A10EE103A1AB2427248
:40788000130A837270477B230370784BD3ED1D0A9FED781A9FED760A00EE810ABDEEC00A10EE103A19B241700B0A83706F4BD3ED230A9FED701A9FED6E0A00EE810ABDEE7B
:4078C000C00A10EE103A19B2C1700B0A0371674BD3ED260A9FED671A9FED650A00EE810ABDEEC00A10EE103A19B241710B0A83715E4B93ED200ADFED600A20EE200ABCEE20
:40790000C00A10EE103A9AB2C271130A0372704710B500245548407B122813D2DFE800F013141718191A1B091E1F1D0E121C1215160A00BFFCF7ACFA044611E006F08DFDB9
:4079400004460DE000BF00BF00BF00BF00BF00BF00BF00BF00BF00BF00BF00BF00BF00BF00BF204610BD10B500244048407B122813D2DFE800F013141718191A1B091E1F80
:407980001D0E121C1215160A00BFFCF785FA044611E006F062FD04460DE000BF00BF00BF00BF00BF00BF00BF00BF00BF00BF00BF00BF00BF00BF00BF204610BD2B48407B9D
:4079C00070472A4890F86400704710B500242748407B122816D2DFE800F01718191A1B1C1D0920211F16151E150E0F0A00BFF7F7C8FA044613E000BFFFF7E3FF642110FB58
:407A000001F40CE000BF00BF00BF00BF00BF00BF00BF00BF00BF00BF00BF00BF00BF00BF204610BD002011490873704713480078704710B500F0DBFF044644F6206122F0E4
:407A400029FA38B900F0D3FF40F2DC51884201D9012010BD0020FCE724190020785200200129040800000000A803002038190020000000470000C84200007A44C40300208D
:407A8000FE490979042901D1012100E000210846704770B50023012113E0CC1701EBD4646511F74C54F82540CD1701EBD5656D11A1EB45160125B5402C4004B10B46481CA8
:407AC000C1B24029E9DB184670BD70B504460D46E21704EBD2625311E94A52F823202146E31704EBD3635B11A4EB43160123B3401A432046E31704EBD3635E11E04B43F8B1
:407B000026202846FDF7B6FB002C37D00821DD48DFF874C300DF012813D0DA482038817F807F401CD74A203A907710464454807F1E2802DB002011468877D248DFF84CC395
:407B400000DF0821D248DFF840C300DF012815D022F09AF9CF4901EBC4014860CD4810F83400FF2806DACB4810F83400401CC94901F83400C648DFF814C300DF70BDC649ED
:407B80000870704710B5BD48007905287BD2DFE800F003152581DE00FEF767FA10B90220B6490871BD48007838B10120BC490870FFF7E5FF0020B94908701AE1FEF755FA16
:407BC00010B90220AD490871B448007828B10120B34908700020B14908700AE1FEF745FA18B10020A549087153E0AC48007898B30120AB490870FEF738FA50B1FEF744FA76
:407C0000044621460920FFF760FF0120FFF7B7FF3FE006F027FA38B129210320FFF755FF0120FFF7ACFF34E09E48007800F0080038B91A213120FFF748FF0120FFF79FFFD7
:407C400027E003208D49087122F01EF9964908600020FDF70FFB1CE0FFE7FFF7B2FEC0B909F044F8A8B1FFF7C0FD90B9FFF7E1FE78B118F04FFEDFED8D0AB4EEE00AF1EE51
:407C800010FA06DD00E0B3E09FED890A0F20FFF775FDAEE08148007800284DD006F0E2F950B129210320FFF710FF0120FFF767FF01207B49087049E0FEF7D7F968B1012054
:407CC000FFF75DFF012076490870FEF7DDF9044621460920FFF7F9FE38E04FF47A717248006822F0D7F890B16E48007800F0020008BB0120FFF743FF1A213120FFF7E5FE1D
:407D000001206749087000205C4908711EE06548007800F00B0070B1FFF767FD30B16548D0F890110120DFF890C100DF04205349087109F0B4FB09E01A210220FFF7C5FE24
:407D400001205749087002204C49087151E05348007850B91A210220FFF7B7FE01205049087002204549087137E006F07BF968B129210320FFF7A9FE022040490871012001
:407D8000FFF7FDFE01204649087026E0FEF76DF980B10020394908710120FFF7F0FEFEF773F9044621460920FFF78FFE01203C49087012E0F5F709FB78B100202F49087100
:407DC0000120FFF7DCFEF5F700FB044621460920FFF77BFE01203249087028480079042805D022F051F82549086009F057FB00E000BF00BF214800792049487110BD204851
:407E0000001F0021016041608160C16070472B490870704710B52A4991F8300001F02AF930B1002213466421264813F03FFD11E0234991F8300001F03FF928B9204991F8FF
:407E4000300001F041F928B10022134631211D4813F02CFD10BD10B50024194991F8300001F008F948B9164991F8300001F024F918B9134991F8300026E028E0D40300209B
:407E8000801F00206C1F0020C92D0408E52C0408081D00204C1D0020DE030020DF030020E0030020E8030020E40300202FDDE43E0000C8427852002001290408DC030020FC
:407EC00030210020D8DF002001F0FEF800B10124204610BDFE480078704710B50446FD480078844204D0FB480470162019F044FA10BD00EE900AB8EE601ADFEDF70AF5EE16
:407F0000001A51EE210AB0EE600ADFEDF40A80EE201AB0EE410A7047F1480078704710B52DED028BFFF7F8FF022807D0FFF7F4FF032803D0FFF7F0FF052812D10CF063FEA8
:407F400030B10CF05AFE022802D19FEDE68A0AE00CF059FE10B19FEDE48A04E01FED2D8A01E01FED2E8AB0EE480ABDEC028B10BD10B52DED028B18F0ADFCB0EE408AFFF721
:407F8000CEFFB4EEC08AF1EE10FA03DB0120BDEC028B10BD0020FAE710B52DED048BF0EE408AB0EE609A0446F0EE689AFFF7E0FF00EE100AB8EE400AB4EEC90AF1EE10FA19
:407FC00007DDFFF7D5FF00EE100AB8EE400AB0EE409A29EE090ADFEDC50A80EE808AECB1F4EEC88AF1EE10FA05DDF0EE489A0120BF49087015E0B1EE480AF4EEC08AF1EE38
:4080000010FA07D2B1EE480AF0EE409A0120B849087006E00020B649087002E00020B4490870B0EE690ABDEC048B10BD10B504460020206060606071207121F025FF20608A
:4080400010BD2DED048B92B04FF05008002405E04FF6FF702DF81400601CC4B2022CF7DB0020FFF7D4FE00208DF80400A1490870FFF785FD0020A0490870A048DFF880C2DC
:4080800000DFA048DFF878C200DF9F48DFF870C200DF00209949183908759C48FFF7C6FF03219B4880F8441100BF002241460720DFF860C200DF0746022F7AD1DFF858C2D6
:4080C00000DF054605F00200002873D010218B48DFF848C200DF012809D028228749183908A827F00EFB8548DFF834C200DFBDF82060FFF7C5FC08B1012000E000208146ED
:4081000018F0E8FBF0EE408A3046FFF7F2FEB0EE409A4846F0EE680AFFF73EFFB0EE408AFFF7AEFC00B375481838007D01280BD1DDED0A0AB0EE600A0121042007F052FF09
:408140008146FFF7CAFE2FE06C481838007D02280BD1DDED090AB0EE600A0121052007F0AEFF8146FFF7B9FE1EE064481838007D03280BD1DDED0B0AB0EE600A01210620F3
:4081800008F043F88146FFF7A8FE0DE05B481838007D042808D101210220B0EE480A07F0AAFE8146FFF799FE9DF83500012802D102E047E032E000205A4908709DF83500BA
:4081C00040B95948007840F00800574908700020FFF7D5FC4FF6FF7086421FD05248007800F00200D0B95048007800F00800A8B1002410E03DF81410711A08B20FF097FD98
:40820000022806DC4848007840F002004649087003E0601CC4B2022CECDB00BF05F0040080B1424801889DF80420501CC0B28DF804002DF812109DF80400022802DB002004
:408240008DF804001CF017FA88B10BF01DFE70B1FFF740FE58B9364813F06AFB38B1FFF7FAFD08B1FFF7D6FD0120FFF7D0FD9DF8360090B10C9821F02FFEB0F5C87F0CD3C8
:4082800001201C4908702248D0F8B4100120DFF8A4C000DF0CF0D8FC02E00020154908702548007D012854D19DF81C0028B900201D49087021F0E8FD824640F2E241504676
:4082C00021F0E8FDD0B31FF030FAB8BB012036E0DC030020D20300200000FB4500007A44D00300200AD7A33C9A99193ED222FB3FE1030020DD030020E9030020301D002048
:40830000D52C04086C1F0020081D0020D40300207852002061290408A9280408C92D0408E52C0408DF030020E8030020401D002080E1002001290408D02B002028E0FE4922
:408340000870FE48D0F8B4100120DFF8F4C300DF1EE09DF81C0001281AD1FA48007DB8B90020F5490870FFF74AFDF448D0F8B4100120DFF8CCC300DFF348007840F001000D
:40838000F14908700120F149087021F07DFD82461822EC4902A827F0B4F9FFF7F3FBEB480078012809D1FFF774FBE94908700020E6490870172018F0DFFFFFF761FB08B178
:4083C000012000E000208146F3F799FB6DE6E14800787047E04800787047E0480078704770B50025DE48007D012801D1002405E0DB48007D08B9012400E002242543D948B8
:40840000C472FDF732FE08B9012400E0002445EA8400C5B2D3484472D348007D08B9012406E0D148007D012801D1002400E0022445EA0410C5B2CB488472FFF7CEFF04460E
:4084400045EA8415C7480472284670BDC748008870472DE9F04105460C4617469846069EB5F52D4F28D12821C0481830DFF800C300DF012820D0A078BC49C875A07800F057
:40848000030048752078617840EA0120B749088021F0FAFCB54908610120887504200875A648D0F840110220DFF894C200DFAF481830DFF8C0C200DFBDE8F081F0EE400AA1
:4084C0009FEDAD0A30EEC01ADFEDAC1A81EE210A70472DE9F0412DED028B04460D4616461F462078AD2833D12821A0481830DFF880C200DF01282AD0E0789C49C875E0783B
:4085000000F0030048756078A17840EA012000EE100AB8EEC00AB0EE408AB0EE480AFFF7CDFF924880ED020A21F0AEFC8F4908610120887508758148D0F840110220DFF8F8
:4085400000C200DF89481830DFF828C200DF6BE02078A92834D1282184481830DFF810C200DF012860D0E0788049C875E07800F0030048756078A17840EA012000EE100A00
:40858000B8EEC00AB0EE408AB0EE480AFFF796FF764880ED010A21F077FC7449086101208875022008756548D0F840110220DFF890C100DF6D481830DFF8B8C100DF33E09D
:4085C0002078AF2830D1282168481830DFF8A0C100DF012828D0E0786449C875E07800F0030048756078A17840EA012000EE100AB8EEC00AB0EE408A5C4880ED038A21F07D
:4086000043FC5A49086101208875032008754B48D0F840110220DFF828C100DF53481830DFF850C100DF00BFBDEC028BBDE8F0811FEDD61A5FEDD80A40EE010AF1EE001AB3
:40864000B6EE001A00EEA11AFCEEC10A10EE901A88B2704710B52DED028B0EF0ADF8B0EE408A9FED470AB4EE408AF1EE10FA06D0B0EE480AFFF7DCFF3A49088003E04FF6D2
:40868000FF70384908802D48D0F840110420DFF8B0C000DF33480088BDEC028B10BD70B58CB006460025002E6ED01FF03EF8002878D040F2B240012102220023CDE90532F7
:4086C000CDE90710042017210193CDE902310490972013460022114600900AA812F0E8FE0AA9304612F0C7FB044640F292400440844204D11DB9042022490870012540F23E
:40870000B240012102220023CDE90532CDE90710042017210193CDE902310490972001230022114600900AA812F0C2FE0AA9304612F0A1FB044629E0E9030020785200204F
:4087400001290408D02B0020E8030020E0030020D1030020DD030020D2030020DE030020002C0020401D0020102A0020181D0020C92D0408E52C040800401C460000C8426D
:4087800000FF7F47D00300200BE00BE040F292400440844205D1002DFCD10520954908700125B7E040F2B240012102220023CDE90532CDE9071017210193CDE90231972062
:4087C000049300900123002211460AA812F070FE0AA9304612F04FFB044640F292400440844204D11DB9032082490870012540F2B240012102220023CDE90532CDE9071048
:4088000017210193CDE902319720049300901346002211460AA812F04BFE0AA9304612F02AFB044640F292400440844204D11DB9022070490870012540F2B24001210222A0
:408840000023CDE90532CDE9071017210193CDE902319720049300900323002211460AA812F026FE0AA9304612F005FB044640F292400440844204D11DB903205D490870A2
:40888000012540F2B240012102220023CDE90532CDE9071017210193CDE902319720049300900423002211460AA812F001FE0AA9304612F0E0FA044640F292400440844208
:4088C00004D11DB902204B490870012540F2B240012102220023CDE90532CDE9071017210193CDE9023197201A461946049300900AA812F0DDFD0AA9304612F0BCFA044627
:4089000040F292400440844204D11DB9012039490870012515B15620F4F722FE28460CB070BD10B5344890F8280007280DD117F0D1FFDFED320AB4EEE00AF1EE10FA01DB71
:40894000012000E00020044600E00124204610BD10B517F0BFFFDFED2A0AB4EEE00AF1EE10FA01D8012010BD0020FCE710B5FFF7FFFA20B9204890F8FF01032801D10120F0
:4089800010BD0020FCE79FED1F0A70479FED1E0A70471848007803280FD01648007802280BD014480078012807D012480078042803D010480078052801D1012070470020E7
:4089C000FCE712480079704710B500F05AFC10B10F48047800E00024204610BDF0EE400A1FED9A1A1FED9C0A00EE810A7047074800687047D0030020302100202FDDE43E6A
:408A000083C00041B81E4141A2454841D4030020E103002010B5044600BF28222146FE48006802F007FE20B928222146FB4826F023FE00BF10BD10B504462822F74920463C
:408A400026F01AFE10BD01B500BF04226946F2480068283002F0EEFD18B99DF80000EF49886200BFEE48C16B0220DFF8B8C300DF08BD01B500BF04226946E74800682C30DC
:408A800002F0D8FD18B99DF80000E449C86200BF08BD01B5E14890F830000099884219D000BF04226946DC480068303002F0C2FD10B9DA490098086300BFD84890F8300014
:408AC000922804D0D54890F83000932802D101201BF008F808BD10B52DED020B00BF04226946CD4800683C3002F0A4FD20B99DED000ACA4880ED0F0A00BF04F028F8C848B0
:408B0000C16B0220DFF81CC300DF0220F4F728FD5020F4F725FD1CBD01B500BF01226946BD480068483002F085FD20B99DF80000BA4981F8480000BF08BD08B50020009007
:408B40001EF0E0FDA0B10021B74800781EF004FEB64800781FF002FA28B10220FFF7DCFF0120009004E00120FFF7D6FF0220009000BF01226946A8480068493002F05AFDE6
:408B800020B99DF80000A54981F8490000BFA448016D0120DFF88CC200DF08BD01B500BF042269469C480068443002F043FD10B99A490098486400BF08BD01B5974890F8C7
:408BC00041009DF80010884215D000BF0122694691480068413002F02DFD20B99DF800008E4981F8410000BF19F0D0FE08F08DF81F20F4F7B5FC08BD01B500BF0122694688
:408C000085480068423002F015FD20B99DF80000824981F8420000BF19F0B8FE2620F4F79FFC7F48C16B0220DFF8F8C100DF08F06CF808BD01B500BF042269467C48006830
:408C4000AC3002F0F7FC18B974480099C0F89C1400BF08BD70B52DED028B04460D4616461EF038FDF8B16D49E0314A5D891C495D501800EBD071491000EE101AB8EEC00A42
:408C8000B0EE408ABCEEC80A10EE101AC8B2294607F07BFCBCEEC80A10EE101AC8B2294607F0A6FC0EE01EF02DFD58B15B49E031485D294607F069FC5849E231485D29460F
:408CC00007F096FC5B4800EB8400D0ED000AB0EE600A2946204607F010FB56490831085D2A46214607F05AFB52490A31085D2A46214607F0CFFB4F490C31085D2A462146EF
:408D000007F005FC46B11D2018F036FB4448016D0120DFF810C100DFBDEC028B70BD70B500240CE0002506E0002229462046FFF791FF681CC5B2022DF6DB601CC4B2022CF1
:408D4000F0DB1D2018F018FB3548016D0120DFF8D4C000DF70BD70B52DED028B04460D461EF0B8FC00B32D48D03000EB840090ED000AB1EE400A2948D83000EB8400D0ED76
:408D8000000A30EE200AF0EE000A80EE201AB0EE418A2046B1EE480A07F017FD2046B0EE480A07F070FD18E01EF0ACFCA8B11B48D03000EB8400D0ED000AB0EE600A20463E
:408DC00007F003FD1548D83000EB8400D0ED000AB0EE600A204607F056FD1048C03000EB8400D0ED000AB0EE600A204607F033FC0A48C83000EB8400D0ED000AB0EE600A8F
:408E0000204607F086FCFDB1192018F0B5FA1D2018F0B2FA19200FE0FC0300203021002078520020012904087F0700209F070020000400201423002018F09EFAF748016DB8
:408E40000120DFF8DCC300DFBDEC028B70BD10B5002405E000212046FFF77DFF601CC4B2022CF7DB192018F087FA1D2018F084FA192018F081FAE948016D0120DFF8A0C325
:408E800000DF10BD70B505460C4600212046FFF762FF002221462846FFF7DCFE70BD70B52DED028B05460024A1E0DE4890F8491005F1380000EB81100E3030F9140000EE9C
:408EC000900AF8EEE00AB0EE600A204607F0B1FDD44890F8491005F1380000EB8110123030F9140000EE900AF8EEE00AB0EE600A204607F0C2FDCB4890F8491005F1380031
:408F000000EB8110163030F9140000EE900AF8EEE00AB0EE600A204607F0D3FDC14890F8491005F1380000EB81101A3030F9140000EE900AF8EEE00AB0EE600A204607F0CD
:408F4000E4FDB84991F8492005F1380101EB82110A31085D214607F0FCFDB24991F8492005F1380101EB82110C31085D214607F00EFEAC4890F8491005F1380000EB811052
:408F8000401C005D00EE100AB8EE400ADFEDA60A80EE201AB0EE418A2046B0EE480A07F014FEA04991F8492005F1380101EB8211091D085D214607F021FE9A4991F84920AE
:408FC00005F1380101EB8211891D085D214607F029FE944991F8492005F1380101EB82110831085D214607F031FE601CC4B2022CFFF65BAF8B4890F8491005F1380000EB9F
:409000008110D0ED080AB0EE600A07F0D6FC854991F8492005F1380101EB8211C87807F0F9F9BDEC028B70BD7E4890F8280008B9012070470020FCE710B501201AF091FD75
:4090400001467A4880F8391000201AF08AFD7749487401201AF085FD04462146012011F0FBFE00201AF07DFD04462146002011F0F3FE10BD01460020282901D1012200E0BF
:409080000022402901D1012300E000231A43492901D1012300E000231A434A2901D1012300E000231A434B2901D1012300E000231A4302B10120704701460020562901D032
:4090C000782900D10120704701460020592900D10120704701460020712900D10120704710B500244F4890F8300091280ED04D4890F83000922809D04A4890F83000712858
:4091000004D0484890F83000B82803D11EF0FAFA00B10124204610BD424890F82810082905D0092903D00A2901D00E2901D1012070470020FCE73B4890F828100A2901D1CF
:40914000012070470020FCE7364890F82810082901D1012070470020FCE7324890F82810092901D1012070470020FCE72D4890F828100E2901D1012070470020FCE710B501
:4091800004461EF0BFFA70B11EF0CFFA00B92CB90121274800781EF0DFFA04E00021244800781EF0D9FA10BD1E4890F8300000EBC00101EB00101F4901EB0010408E7047D2
:4091C0000246012109E001EB01101B4B13F81000904201D1C8B27047491C2229F3DB0020F9E7104890ED0F0A70470E4890F84900022801D1012070470020FCE7094890F8CF
:409200004900012800D170470020FCE7054890F8490008B9012070470020FCE77852002001290408302100200000C84258E100207A070020905704080C53040810B500249B
:40924000FFF7E4FF08B1012419E01EF05BFAB0B1FFF7D4FF20B1634800781EF07FFE68B9FFF7C3FF58B1F1F7C7F938B9F1F7C4F928B95C4800781EF071FE00B90124204654
:4092800010BD594890F8970020B1574890F89700012801D1012070470020FCE7524890F82800072801D1012070470020FCE74E4890F89700022804D04B4890F89700032806
:4092C00001D1012070470020FCE7474890F89700032801D1012070470020FCE7424890F89700022801D1012070470020FCE73E4890F8970008B9012070470020FCE73A48F8
:4093000090F89700012800D170470020FCE7364890F89700042801D1012070470020FCE7314890F89700042801D1012070470020FCE701B500BF012269462C480068973089
:4093400002F078F920B99DF80000274981F8970000BF08BD01B500BF012269462348006800F2853002F066F920B99DF800001E4981F8850300BF08BD10B500241A4890F8D9
:409380003000282827D0184890F83000402822D0154890F8300049281DD0134890F830004A2818D0104890F830004B2813D00E4890F8300059280ED00B4890F830005C2882
:4093C00009D0094890F83000782804D0064890F830001D2800D101242046FFF7BBFF204610BD00009F07002030210020FC0300201FB51EF0AEF9062808D01EF0AAF90728C8
:4094000004D01EF0A6F9082841F077821EF08DF900287DD0002000900190029003460122FE4903901EF06FFA002000900190029003460322FA49039001201EF064FA0020F4
:4094400000900190029003460322F649039002201EF059FA002000900190029003460322F149039010461EF04EFA002000900190029003460322ED49039004201EF043FA43
:40948000002000900190029003460422E849039005201EF038FA002002220123CDE901200093039003460322E24906201EF02BFA002000900190029003460246DE490390CC
:4094C00007201EF020FA002000900190029003460322DA49039008201EF015FA002000900190029003460122D549039009201EF00AFA002000900190029003460122D1495D
:4095000003900A201EF0FFF900200090019000E0E0E3029003460122CB4903900B201EF0F2F9002001210090CDE9010103460A46C64903900C201EF0E6F90020009001909C
:40954000029003460246C249039011201EF0DBF9002000900190029003460322BD49039012201EF0D0F900200222CDE9000202900346B949039016201EF0C5F90020012184
:409580000090CDE9010103460A46B449039017201EF0B9F9002000900190029003460222AF49039019201EF0AEF900200222CDE9000202900346AB4903901A201EF0A3F948
:4095C000002000900190029001230222A64903901B201EF098F9002000900190029001230222A24903901C201EF08DF900200222CDE90002029003469D4903901E201EF0EF
:4096000082F900200222CDE90002029003460246984903901F201EF076F90020009001900290034603229449039021201EF06BF90020009001900290034603228F49039050
:4096400022201EF060F90020009001900290034603228B49039023201EF055F90020009001900290034603228649039024201EF04AF90020009001900290034603228249B6
:40968000039025201EF03FF90020009001900290034603227D49039026201EF034F90020009001900290034601227949039027201EF029F900200090019002900346012227
:4096C0007449039028201EF01EF90020009001900290034601227049039029201EF013F90020009001900290034602226B4903902B201EF008F900200090019002900346C2
:409700000222674903902C201EF0FDF8002000900190029003460122624903902D201EF0F2F80020009001900290034601225E4903902E201EF0E7F800200090019002902A
:4097400003460122594903902F201EF0DCF80020009001900290034601225549039031201EF0D1F80020009001900290034601225049039032201EF0C6F800200121CDE9FE
:40978000000103460A46CDE902104B4936201EF0BAF8002000900190029003460122474903903B201EF0AFF8002000900190029003460122424903903C201EF0A4F80020A8
:4097C0000122CDE90002029003463E4903903D201EF099F800200122CDE9000202900346394903903E201EF08EF8002001210090CDE9010103460A463449039041201EF01E
:4098000082F80020009001900290034601223049039042201EF077F800205BE043070020600700205F070020A3070020A40700206307002064070020AF07002061070020AA
:40984000770700207607002075070020970700202C070020690700201F070020360700202007002025070020A5070020A60700202407002029070020190700201B07002084
:409880006C0700206D0700206E0700206F070020710700207007002072070020730700207407002065070020670700206607002078070020790700207A0700207C0700202F
:4098C0007D0700207E0700207F070020800700204A07002000900190029003460122FE49039043201EF00FF8002000900190029003460122F949039044201EF004F800204E
:4099000001210090CDE9010103460A46F449039048201DF0F8FF002001210090CDE9010103460A46EF4903904B201DF0ECFF002001210090CDE9010103460A46EA490390AE
:409940004D201DF0E0FF002000900190029003460322E64903904F201DF0D5FF012000220092CDE9012013460246E149039050201DF0C9FF002001210090CDE90101034619
:409980000A46DC49039051201DF0BDFF002000900190029003460122D749039052201DF0B2FF002000900190029003460322D349039054201DF0A7FF002000900190029059
:4099C00003460322CE49039055201DF09CFF002000900190029003460322CA49039056201DF091FF002000900190029003460322C549039057201DF086FF00200222CDE953
:409A00000002029003460246C049039057201DF07AFF002000900190029003460322BC49039058201DF06FFF002000900190029003460322B749039059201DF064FF0020BF
:409A400000900190029003460322B34903905A201DF059FF002000900190029003460322AE4903905B201DF04EFF002001210090CDE9010103460A46A94903905C201DF086
:409A800042FF002000900190029003460122A54903905D201DF037FF002000900190029003460122A04903905E201DF02CFF0020009001900290034601229C4903905F203E
:409AC0001DF021FF00200222CDE900020290034601229749039061201DF015FF00200222CDE900020290034601229249039062201DF009FF002000900190029003460122EC
:409B00008D49039064201DF0FEFE0020009001900290034601228949039065201DF0F3FE002001210090CDE9010103460A468449039067201DF0E7FE002001210090CDE984
:409B4000010103460A467F49039069201DF0DBFE00200222CDE900020290034602467A4903906A201DF0CFFE01200021009101910B460246CDE9021074496B201DF0C3FECB
:409B800000200222CDE9000202900346704903906D201DF0B8FE00200222CDE90002029003466C4903906E201DF0ADFE00200222CDE9000202900346674903906F201DF017
:409BC000A2FE002001210090CDE9010103460A466249039073201DF096FE00200222CDE900020290034602465D49039079201DF08AFE0020009001900290034602225949C8
:409C000003907A201DF07FFE002000900190029003460122544903907B201DF074FE002000900190029003460122504903907C201DF069FE0020009001900290034601222A
:409C40004B4903907D201DF05EFE002001210090CDE9010103460A46464903907E201DF052FE002000900190029003460122424903907F201DF047FE002001210090CDE9A1
:409C80000101034602223D49039082201DF03BFE002001210090CDE90101034602223849039083201DF02FFE002001210090CDE90101034602223349039084201DF023FE74
:409CC00001200021009101910B460222CDE902102D495BE0DAE000008107002082070020A7070020A80700209607002062070020830700208407002085070020AC0700204F
:409D0000AD070020AE070020B0070020310700208A0700208B0700208C070020270700208D0700208F070020900700208E0700206B0700206A07002091070020920700207D
:409D400093070020950700205707002044070020A9070020AA070020AB070020980700209A0700209B0700203D0700203E0700209C0700209D070020990700204707002051
:409D800048070020490700209F07002086201DF0BAFD01200021009101910B460222CDE90210FE4987201DF0AEFD01200021009101910B460246CDE90210F94988201DF08F
:409DC000A2FD002000900190029003460322F54903908E201DF097FD002000900190029003460322F04903908F201DF08CFD002000900190029003460322EC4903908F2059
:409E00001DF081FD012009F060FD0021E84800781DF0A2FC0021E74800781DF09DFC0021E54800781DF098FC0021E44800781DF093FC01200021009101910B460222CDE9E6
:409E40000210DF4986201DF05EFD01200021009101910B460222CDE90210DA4987201DF052FD0121D84800781EF0FBF80121D74800781EF0F6F80121D54800781EF0F1F8B4
:409E80000121D44800781EF0ECF8E1E3002000900190029003460122CF4903901DF033FD002000900190029003460322C649039001201DF028FD00200090019002900346BD
:409EC0000322C249039002201DF01DFD002000900190029003460322C049039010461DF012FD002000900190029003460322BC49039004201DF007FD002000900190029026
:409F000003460422B749039005201DF0FCFC002002220123CDE901200093039003460322B14906201DF0EFFC002000900190029003460322A749039007201DF0E4FC002012
:409F400000900190029003460322A149039008201DF0D9FC002000900190029003460122A249039009201DF0CEFC0020009001900290034601229E4903900A201DF0C3FCCD
:409F8000002000900190029003460122994903900B201DF0B8FC002001210090CDE9010103460A46944903900C201DF0ACFC002000900190029003460322904903901120AF
:409FC0001DF0A1FC0020009001900290034603228B49039012201DF096FC00200222CDE90002029003468749039016201DF08BFC002001210090CDE9010103460A466E4960
:40A00000039017201DF07FFC0020009001900290034602227C49039019201DF074FC00200222CDE9000202900346784903901A201DF069FC0020009001900290012302228E
:40A04000734903901B201DF05EFC0020009001900290012302226F4903901C201DF053FC00200222CDE90002029003466A4903901E201DF048FC00200222CDE900020290B7
:40A0800003460246654903901F201DF03CFC00200222CDE900020290034602466049039020201DF030FC0020009001900290034603225C49039021201DF025FC00200090DE
:40A0C00001900290034603225749039022201DF01AFC0020009001900290034603225349039023201DF00FFC0020009001900290034603224E49039024201DF004FC002090
:40A10000009001900290034603224A49039025201DF0F9FB0020009001900290034603224549039026201DF0EEFB0020009001900290034601224149039027201DF0E3FB66
:40A140000020009001900290034601223C49039028201DF0D8FB0020009001900290034601223849039029201DF0CDFB002000900190029003460222334903902B201DF048
:40A18000C2FB0020009001900290034602222F4903902C201DF0B7FB002059E0A0070020A107002050070020510700204F0700208D070020840700203607002079070020E3
:40A1C0003307002032070020600700205F070020610700205E07002043070020A3070020A40700206307002064070020770700207607002075070020970700202D07002095
:40A20000690700201F0700202007002025070020A5070020A6070020240700202907002030070020190700201B0700206C0700206D0700206E0700206F07002071070020BE
:40A240007007002072070020730700207407002000900190029003460122FE4903902D201DF051FB002000900190029003460122F94903902E201DF046FB002000900190E9
:40A28000029003460122F54903902F201DF03BFB002000900190029003460122F049039031201DF030FB002000900190029003460122EC49039032201DF025FB00200121E1
:40A2C000CDE9000103460A46CDE90210E64936201DF019FB002000900190029003460122E24903903B201DF00EFB002000900190029003460122DE4903903C201DF003FBD2
:40A3000000200122CDE9000202900346D94903903D201DF0F8FA00200122CDE9000202900346D54903903E201DF0EDFA002001210090CDE9010103460A46D049039041202D
:40A340001DF0E1FA002000900190029003460122CB49039042201DF0D6FA002000900190029003460122C749039043201DF0CBFA002000900190029003460122C2490390DC
:40A3800044201DF0C0FA002001210090CDE9010103460A46BD49039048201DF0B4FA002001210090CDE9010103460A46B84903904B201DF0A8FA002001210090CDE9010138
:40A3C00003460A46B34903904D201DF09CFA002000900190029003460322AF4903904F201DF091FA012000220092CDE9012013460246AA49039050201DF085FA0020012141
:40A400000090CDE9010103460A46A549039051201DF079FA002000900190029003460122A049039052201DF06EFA0020009001900290034603229C49039054201DF063FA90
:40A440000020009001900290034603229749039055201DF058FA0020009001900290034603229349039056201DF04DFA0020009001900290034603228E49039057201DF0AB
:40A4800042FA0020009001900290034603228A49039058201DF037FA0020009001900290034603228549039059201DF02CFA002000900190029003460322814903905A209D
:40A4C0001DF021FA0020009001900290034603227C4903905B201DF016FA002001210090CDE9010103460A46774903905C201DF00AFA002000900190029003460122734905
:40A5000003905D201DF0FFF90020009001900290034601226E4903905E201DF0F4F90020009001900290034601226A4903905F201DF0E9F900200222CDE90002029003463B
:40A5400001226549039061201DF0DDF900200222CDE900020290034601226049039062201DF0D1F90020009001900290034601225B49039064201DF0C6F90020009001907D
:40A580000290034601225749039065201DF0BBF9002001210090CDE9010103460A465249039067201DF0AFF9002001210090CDE9010103460A464D49039069201DF0A3F919
:40A5C00000200222CDE90002029003460246484903906A201DF097F901200021009101910B460246CDE9021042496B201DF08BF900200222CDE90002029003463E49039093
:40A600006D201DF080F900200222CDE90002029003463A4903906E201DF075F900200222CDE9000202900346354903906F201DF06AF9002001210090CDE9010103460A4607
:40A640003049039073201DF05EF9002002225BE053E1000065070020670700206607002078070020790700207A0700207C0700207D0700207E0700207F0700208007002064
:40A680004A0700208107002082070020A7070020A80700209607002062070020830700208407002085070020AC070020AD070020AE070020B00700208A0700208B0700203E
:40A6C0008C070020270700208D0700208F070020900700208E0700206B0700206A070020910700209207002093070020950700205707002044070020A9070020AA070020EF
:40A70000AB07002098070020CDE90002029003460246FE49039079201DF0F5F8002000900190029003460222F94903907A201DF0EAF8002000900190029003460122F54925
:40A7400003907B201DF0DFF8002000900190029003460122F04903907C201DF0D4F8002000900190029003460122EC4903907D201DF0C9F8002001210090CDE90101034602
:40A780000A46E74903907E201DF0BDF8002000900190029003460122E24903907F201DF0B2F8002001210090CDE9010103460222DD49039082201DF0A6F800200121009004
:40A7C000CDE9010103460222D849039083201DF09AF8002001210090CDE9010103460222D349039084201DF08EF801200021009101910B460222CDE90210CE4986201DF0F5
:40A8000082F801200021009101910B460222CDE90210C94987201DF076F801200021009101910B460246CDE90210C44988201DF06AF8002000900190029003460322C04994
:40A8400003908E201DF05FF8002000900190029003460322BB4903908F201DF054F8002000900190029003460322B74903908F201DF049F8012009F028F80021B3480078B4
:40A880001CF06AFF0021B24800781CF065FF0021B04800781CF060FF0021AF4800781CF05BFF01200021009101910B460222CDE90210AA4986201DF026F8012000210091F5
:40A8C00001910B460222CDE90210A54987201DF01AF80121A34800781DF0C3FB0121A24800781DF0BEFB0121A04800781DF0B9FB01219F4800781DF0B4FB1FBD1FB50020EB
:40A90000009001900290034603229A49039001201CF0F9FF0020009001900290034603229549039002201CF0EEFF0020009001900290034603229149039010461CF0E3FF9C
:40A940000020009001900290034603228C49039004201CF0D8FF0020009001900290034604228849039005201CF0CDFF0020009001900290034603228349039006201CF0B2
:40A98000C2FF0020009001900290034603227F49039007201CF0B7FF0020009001900290034603227A49039008201CF0ACFF00200090019002900346022255490390092041
:40A9C0001CF0A1FF0020009001900290034602227049039017201CF096FF0020009001900290034602466C49039019201CF08BFF0020009001900290034603226749039048
:40AA000021201CF080FF0020009001900290034603226349039022201CF075FF0020009001900290034602224D49039027201CF06AFF002000900190029003460222474913
:40AA4000039028201CF05FFF0020009001900290034602465349039029201CF054FF01200021009101910B460A46CDE902104E492A201CF048FF0020009001900290034638
:40AA800002464A4903902B201CF03DFF002000900190029003460122454903902D201CF032FF002000900190029003460246414903902E201CF027FF0020009001900290D7
:40AAC000034602463C4903902F201CF01CFF0020009001900290034602463849039030201CF011FF0020009001900290034602463349039046201CF006FF00200090019028
:40AB00000290034602462F4903905DE09A0700209B0700203D0700203E0700209C0700209D070020990700204707002048070020490700209F070020A0070020A107002075
:40AB400050070020510700204F0700208D0700208407002036070020790700203307002032070020600700205F070020610700205E0700206C070020190700201A07002033
:40AB80001B0700201C0700206F0700201D0700201E0700204B070020230700202607002027070020340700202D0700202A07002054070020550700205607002057070020A8
:40ABC000280700205907002047201CF09CFE002000900190029003460246F649039048201CF091FE002000900190029003460122F149039057201CF086FE002000900190EC
:40AC0000029003460222ED49039059201CF07BFE002000900190029003460222E84903905A201CF070FE002000900190029003460122E44903905B201CF065FE00200090BD
:40AC40000190029003460122DF4903905C201CF05AFE002000900190029003460122DB4903905D201CF04FFE002000900190029003460122D64903905E201CF044FE002001
:40AC800000900190029003460122D24903905F201CF039FE002000900190029003460122CD49039060201CF02EFE002000900190029003460122C949039061201CF023FED3
:40ACC000002000900190029003460122C449039064201CF018FE002000900190029003460122C049039065201CF00DFE002000900190029003460122BB49039066201CF0F0
:40AD000002FE002000900190029003460122B749039067201CF0F7FD002000900190029003460122B249039068201CF0ECFD002000900190029003460122AE49039069201E
:40AD40001CF0E1FD002000900190029001231A46A94903906A201CF0D6FD002000900190029003460122A54903906C201CF0CBFD002000900190029003460122A0490390C9
:40AD80006D201CF0C0FD0020009001900290034601229C4903906E201CF0B5FD01200021009101910B460A46CDE9021096497C201CF0A9FD01200021009101910B460A4639
:40ADC000CDE9021091497D201CF09DFD002001210090CDE9010103460A468D49039081201CF091FD0020009001900290034602228849039082201CF086FD00200090019091
:40AE00000290034602228449039083201CF07BFD0020009001900290034602227F49039084201CF070FD0020009001900290034602227B49039086201CF065FD0020009079
:40AE400001900290034602227649039087201CF05AFD0020009001900290034602467249039088201CF04FFD0020009001900290034603226D4903908D201CF044FD002090
:40AE800000900190029003460322694903908E201CF039FD002000900190029003460322644903908F201CF02EFD0121584800781CF052FC0121604800781CF04DFC012188
:40AEC0005E4800781CF048FC1FBD1FB500240CE000205B4901EB041189680870584901EB0411C9680870601CC4B2902CF0DB1CF085FB1DF023FA20F0B7FD0121022023F061
:40AF00002CF90020009001900290034601224D49039016201CF0F7FC002001210090CDE9010103460A46484903901E201CF0EBFC0020009001900290034601224349039079
:40AF40006B201CF0E0FC1CF004FCFF2831D00121084623F002F90121042023F0FEF80121082023F0FAF80121102023F0F6F80121202023F0F2F80121402023F0EEF80121BF
:40AF8000802023F0EAF80121080223F0E6F81CF0E0FB0A2862D2DFE800F06105060708095B5C5D5E00BF00BF00BF00BFFFF7A6FC55E055E0290700205D07002035070020B7
:40AFC000360700203707002038070020390700205A0700205B0700205C0700203A0700207D0700207E0700203D0700203E0700203F0700204007002041070020440700203E
:40B000004507002046070020300700202F0700204A070020470700204807002049070020600700205F0700204C0700204F07002050070020510700204D0700204E070020FE
:40B04000187E04081F070020240700204307002000BF00BF00BFFEF7CBF900E000BF00BF1FBD10B50120FE4908701EF00DFFFC494860012022F022FF1CE0612022F0C0FEB6
:40B0800078B145F25550F74908600120486040F6B83088604CF6CC4008600220F049087008E0EF4948681EF017FF642802D90320EB490870EA4800780128DED010BD10B54E
:40B0C0000020E74908704FF4FA701EF0B1FEFA201EF0F4FEFFF7C5FFFFF7F7FE1CF0FAFAC8B1E14800781CF039FF40B90121DF4800781CF031FB0020DD4908700BE0DD4841
:40B1000000781CF02BFF18B10220D949087002E00120D74908701BF04FFDEDF7D3F800221146D548DFF854C300DF002010BD10B572B66FF0040000F059FA6FF0010000F008
:40B1400055FA4FF0FF3000F051FA042000F04EFA052000F04BFA062000F048FA072000F045FA082000F042FA092000F03FFA0A2000F03CFA0B2000F039FA0C2000F036FAE3
:40B180000D2000F033FA0E2000F030FA0F2000F02DFA102000F02AFA112000F027FA122000F024FA132000F021FA142000F01EFA152000F01BFA162000F018FA172000F0DE
:40B1C00015FA182000F012FA192000F00FFA1A2000F00CFA1B2000F009FA1C2000F006FA1D2000F003FA1E2000F000FA1F2000F0FDF9202000F0FAF9212000F0F7F9222053
:40B2000000F0F4F9232000F0F1F9242000F0EEF9252000F0EBF9262000F0E8F9272000F0E5F9282000F0E2F9292000F0DFF92A2000F0DCF92B2000F0D9F92C2000F0D6F969
:40B240002D2000F0D3F92E2000F0D0F92F2000F0CDF9302000F0CAF9312000F0C7F9322000F0C4F9332000F0C1F9342000F0BEF9352000F0BBF9362000F0B8F9372000F087
:40B28000B5F9382000F0B2F9392000F0AFF93A2000F0ACF93B2000F0A9F93C2000F0A6F93D2000F0A3F93E2000F0A0F93F2000F09DF9402000F09AF9412000F097F942205A
:40B2C00000F094F9432000F091F9442000F08EF9452000F08BF9462000F088F9472000F085F9482000F082F9492000F07FF94A2000F07CF94B2000F079F94C2000F076F989
:40B300004D2000F073F94E2000F070F94F2000F06DF9502000F06AF9512000F067F96FF0040000F06CF96FF0010000F068F94FF0FF3000F064F9042000F061F9052000F08D
:40B340005EF9062000F05BF9072000F058F9082000F055F9092000F052F90A2000F04FF90B2000F04CF90C2000F049F90D2000F046F90E2000F043F90F2000F040F910207C
:40B3800000F03DF9112000F03AF9122000F037F9132000F034F9142000F031F9152000F02EF9162000F02BF9172000F028F9182000F025F9192000F022F91A2000F01FF979
:40B3C0001B2000F01CF91C2000F019F91D2000F016F91E2000F013F91F2000F010F9202000F00DF9212000F00AF9222000F007F9232000F004F9242000F001F9252000F0F2
:40B40000FEF8262000F0FBF8272000F0F8F8282000F0F5F8292000F0F2F82A2000F0EFF82B2000F0ECF82C2000F0E9F82D2000F0E6F82E2000F0E3F82F2000F0E0F8302086
:40B4400000F0DDF8312000F0DAF8322000F0D7F8332000F0D4F8342000F0D1F835200FE0F0030020003000402A07002046070020EC030020570700209F4D0208153104086D
:40B4800000F0BDF8362000F0BAF8372000F0B7F8382000F0B4F8392000F0B1F83A2000F0AEF83B2000F0ABF83C2000F0A8F83D2000F0A5F83E2000F0A2F83F2000F09FF891
:40B4C000402000F09CF8412000F099F8422000F096F8432000F093F8442000F090F8452000F08DF8462000F08AF8472000F087F8482000F084F8492000F081F84A2000F064
:40B500007EF84B2000F07BF84C2000F078F84D2000F075F84E2000F072F84F2000F06FF8502000F06CF8512000F069F862B610BD38B5044660680090009D206880F3088881
:40B5400000BFA84738BD00BFBFF34F8F3048006800F4E0602F490843001D2D490860BFF34F8F00BF00BFFEE710B500212A4800781CF0F2F80021294800781CF0EDF8002132
:40B58000274800781CF0E8F801DF10BD01B500BF04226946234800688C3000F04BF818B921480099C0F87C1400BF08BD01B500BF042269461B480068903000F03BF818B997
:40B5C00019480099C0F8801400BF08BD01B500BF0422694613480068943000F02BF818B911480099C0F8841400BF08BD00F01F02012191400D4A430942F82310704700F04B
:40B600001F02012191400A4A430942F8231070470CED00E00000FA057E0700207C0700207D070020000400203021002080E100E080E200E070B504460D4616463246294651
:40B640002046EDF7E8FB70BD2DE9F34F82B0844600BF00210A460B460E460F46002001908046009064E09CF80000A0F13004E5179CF800002E2838D1B8F1000F0CD1FA4987
:40B680004FF00009A2FB010A03FB01A102FB0919861949EB07071FE0B8F1010F0CD1F3494FF00009A2FB010A03FB01A102FB0919861949EB07070FE0B8F1020F0CD14FF4D0
:40B6C0007A714FF00009A2FB010A03FB01A102FB0919861949EB070708F1010000F0FF0800200090002213461CE09CF80000C8B1009810B922462B4610E0009801280DDBD7
:40B700004FF00A0A4FF0000B1146A1FB0A1E03FB0AE902FB0B900A1940EB05030098401CC0B200900CF1010C0198401CC0B2019003990198884296DBB6185F4130463946A7
:40B7400004B0BDE8F08F2DE9F04F83468946924600BF00BF51465846FFF776FF05460E4651464846FFF770FF07468846781B78EB060001DA012407E0E81B76EB080002DA9F
:40B780004FF0FF3400E000242046BDE8F08F70B586B00546B6A2B9A102A823F087FE1022294602A8FFF7CFFF00283EDD0026002001900090012435E0062C0CD2DFE804F031
:40B7C0000B0C09070503AE4E08E0AE4E06E0AE4E04E0AE4E02E000BFAD4E00BF00BF9120019021200090AB4890F830000A2817D1042201A906F13000FFF71CFF04226946A9
:40B8000006F12C00FFF716FFA24890F82404A04206D19DF804009F4908639DF80000C862601CC4B2052CC7DD00BF06B070BD70B586B0054698A291A102A823F037FE10223D
:40B84000294602A8FFF77FFF00282DDD002600200190012425E0062C0CD2DFE804F00B0C09070503864E08E0864E06E0864E04E0864E02E000BF864E00BF00BFFF20019069
:40B88000012201A906F2FF10FFF7D4FE814890F82404A04203D19DF80400F0F70EFA601CC4B2052CD7DD00BF06B070BD70B586B005467CA271A102A823F0F8FD1022294693
:40B8C00002A8FFF740FF00283FDD0026002001909FED770A8DED000A012433E0062C0CD2DFE804F00B0C09070503654E08E0654E06E0654E04E0654E02E000BF644E00BFFB
:40B9000000BF002001909FED6A0A8DED000A012201A906F14300FFF78DFE0422694606F5DC70FFF787FE5B4890F82404A04207D19DF80400F8F79BFB9DED000AF8F7A8FBA3
:40B94000601CC4B2052CC9DD00BF06B070BD70B586B0054657A249A102A823F0A7FD1022294602A8FFF7EFFE00282DDD002664200190012425E0062C0CD2DFE804F00B0CCB
:40B98000090705033E4E08E03E4E06E03E4E04E03E4E02E000BF3E4E00BF00BF64200190012201A906F56970FFF744FE394890F82404A04203D19DF8040004F02BFD601CDC
:40B9C000C4B2052CD7DD00BF06B070BDF0B585B005463BA229A101A823F068FD1022294601A8FFF7B0FE00283CDD2A4890F82464012434E0062C0CD2DFE804F00B0C090781
:40BA000005031F4F08E01F4F06E01F4F04E01F4F02E000BF1E4F00BF00BF40F6C41000900222694607F56070FFF704FEB44204D1BDF800001749A1F880034FF47A5000903E
:40BA40000222694607F28230FFF7F4FDB44204D1BDF800000F49A1F88203601CC4B2052CC8DD00BF05B0F0BD00CA9A3B40420F0032312E322E302E3130000000257300000A
:40BA8000581B00687017006888130068A00F0068B80B00683021002032312E322E302E360000000032312E322E302E350000000035FA8E3C32312E312E302E39000000007D
:40BAC000322E342E302E3533000000002DE9F04105460E4617463A4631462846EDF712FA044604B103DF2046BDE8F081F0B585B00546F7A2AFF27C0101A823F0D7FC10222C
:40BB0000294601A8FFF71FFE00282FDDF34890F82474012427E0062C0CD2DFE804F00B0C09070503EE4E08E0EE4E06E0EE4E04E0EE4E02E000BFEE4E00BF00BF042206F507
:40BB4000C6716846FFF7C2FF0422694606F56270FFF770FDBC4204D19DED000ADF4880EDE20A601CC4B2052CD5DD00BF05B0F0BDF0B585B00546DFA2AFF2001101A823F033
:40BB800095FC1022294601A8FFF7DDFD00282BDDD24890F82464012423E0062C0CD2DFE804F00B0C09070503CD4F08E0CD4F06E0CD4F04E0CD4F02E000BFCD4F00BF00BF01
:40BBC000002000900122694607F19700FFF732FDB44204D19DF80000C04981F89700601CC4B2052CD9DD00BF05B0F0BD2DE9F04186B00546C2A2AFF27C1102A823F056FC33
:40BC00001022294602A8FFF79EFD002836DD002001900026B14890F8247400242BE0062C13D2DFE804F0130F0C090603DFF8B0820FE0DFF8B0820CE0DFF8AC8209E0DFF80A
:40BC4000AC8206E0DFF8A88203E000BFDFF8BC8200BF00BF042201A908F1B400FFF7EAFCBC4206D19D490198C1F8B4000846C0F89860601CC4B2052CD1DD00BF06B0BDE877
:40BC8000F081F0B587B00646A1A2AFF2102103A823F00CFC1022314603A8FFF754FD002857DD8E4890F8247400244FE0062C0ED2DFE804F00E0B09070503894D0AE0894D3C
:40BCC00008E0894D06E0894D04E0894D02E000BF8E4D00BF00BF042205F1300101A8FFF7F5FE13208DF809000198FDF7C3F918B90198FDF7E9F918B190208DF808000AE0FD
:40BD00000198FDF7D9F918B113208DF8080002E0FF208DF8080001220DF1090105F1B300FFF788FC012202A905F1B200FFF782FCBC4209D19DF80910684880F8B3109DF84F
:40BD40000800664981F8B200601CC4B2052CADDD00BF07B0F0BDF0B585B005466FA2AFF2E42101A823F0A2FB1022294601A8FFF7EAFC00282DDD594890F824640120009022
:40BD8000002423E0062C0ED2DFE804F00E0B09070503534F0AE0534F08E0534F06E0534F04E0534F02E000BF584F00BF00BF0122694607F14B00FFF73DFCB44204D19DF82E
:40BDC0000000464981F84B00601CC4B2052CD9DD00BF05B0F0BDF0B587B0054651A2AFF2643103A823F062FB1022294603A8FFF7AAFC002839DD394890F82474002431E08F
:40BE0000062C0ED2DFE804F00E0B09070503344E0AE0344E08E0344E06E0344E04E0344E02E000BF394E00BF00BF012206F1280102A8FFF74BFE9DF80800042810D0B2EEC3
:40BE4000040A8DED010A042201A906F5FC70FFF7F1FBBC4204D19DED010A204880ED7E0A601CC4B2052CCBDD00BF07B0F0BDF0B585B006462DA2AFF2FC3101A823F016FBD3
:40BE80001022314601A8FFF75EFC00287EDD072729A2AFF2184101A823F008FB1022314601A8FFF750FC002800DD092700200090002468E0062C49D2DFE804F049464407E4
:40BEC0000503074D45E0074D43E0074D41E00000322E342E302E34340000000030210020581B00687017006888130068A00F0068B80B0068322E332E302E3330000000004B
:40BF0000322E322E302E343600000000D0070068322E322E302E313800000000322E322E302E3200322E322E302E3100322E312E302E373300000000322E312E302E353407
:40BF400000000000F64D04E0F64D02E000BFF64D00BF00BF042205F130016846FFF7B6FD009838440090009814280BD30422694605F13000FFF75EFBEB48854202D1EB49B0
:40BF800000980863641C062C94D300E000E000BF05B0F0BD2DE9F3410D46E449ADEB010408460719DF482618AAB239463046FFF741FBDE480719DA482618AAB239463046D0
:40BFC000FFF738FBD9480719D9482618AAB239463046FFF72FFBD5480719D6482618AAB239463046FFF726FBD0480719D2482618AAB239463046FFF71DFBBDE8FC812DE9DF
:40C00000FE4F81468A46174698460020009000262D2200233846414623F0BDF905462D2200233846414623F0B6F9934615B9BBF1000F35D0D5B1002416E0C4EB041000EB92
:40C04000400048440290C4EB041000EB4000504401902D22DDE90110FFF7ECFA0646009931430091601CC4B2AC42E6D3BBF1000F18D0C5EB051000EB400048440290C5EB69
:40C08000051000EB4000504401901FFA8BF2DDE90110FFF7CFFA064600993143009101E0402000900098BDE8FE8F01B500BF01226946A24800682D30FFF7BCFA20B99DF85A
:40C0C00000109A4880F81D1400BF08BD2DE9FE4F81468A46174698460020009000262D2200233846414623F056F905462D2200233846414623F04FF9934615B9BBF1000FBE
:40C1000035D0D5B1002416E0C4EB041000EB400048440290C4EB041000EB4000504401902D22DDE90110FFF7D1FC0646009931430091601CC4B2AC42E6D3BBF1000F18D02C
:40C14000C5EB051000EB400048440290C5EB051000EB4000504401901FFA8BF2DDE90110FFF7B4FC064600993143009101E0402000900098BDE8FE8F3EB5002002900A2035
:40C180000190002000904FF47C71684823F0F3FAB0216B4823F0EFFA4FF458716848B03023F0E9FA012201A9644800689830FFF741FA012261480168983102A8FFF786FC52
:40C1C0009DF80800401CC0B20190012201A95B4800689830FFF72EFA012258480168983102A8FFF773FC9DF808009DF80410884207D05448007840F080005249087001249E
:40C200008CE001224D4801682E316846FFF75EFC9DF8000044284CD0FF224FF47C71434823F0A1FA4FF47C72002340493E48FFF7E6FE4FF47C7200233C493A48FFF7DFFE02
:40C240004FF47C72002339493548FFF7D8FE4FF47C72002335493648FFF7D1FE4FF47C72002332493348FFF7CAFE4FF47C7200232E493148FFF7C3FE4FF47C712B4823F0D1
:40C280007AFAB02200232E494FF0D040FFF7B7FE4FF4587200232A49B0312B48FFF7AFFE4420009001226946244800682E30FFF7C1F9B02200234FF0D0412148FFF706FFB9
:40C2C0004FF45872002320491D48B030FFF7FEFE01221A4801682D3119482D30FFF7F6FB124890F81D04672810D001246720FFF7DCFE4FF47C710D4823F03DFA4FF47C728F
:40C3000000230A490848FFF77AFE07E002244FF47C72002304490548FFF7D8FE20463EBDA00F0068B80B0068D0070068302100208813006870170068581B006800040020BE
:40C3400020250020F9030020F401006810B5FA48ECF710FD0446204610BD70B58CB000240020089009900A900B9004900590069007900090019002900390F0490870F049DA
:40C38000087001200870FFF7E1FFFFF7F5FEED490870ED4AAFF61C1108A823F087F804A81BF0C4FFE9A104A823F00CFA08B1012000E00020054645B1E6A01BF0A3FFE3A01A
:40C3C0001BF0A0FFE7A01BF083FF04A81BF092FF102204A908A8FFF7B6F90446D9480078012806D10020D649087008A81BF070FFCFE0002CFCD0002006F0B0F8002006F0C4
:40C4000000F908A81BF064FF002C39DA0020FFF74CFEFF224FF47C71D44823F0A4F94FF47C720023D149D248FFF7E9FD4FF47C720023CE49CF48FFF7E2FD4FF47C7200231A
:40C44000CA49CD48FFF7DBFD4FF47C720023C749CA48FFF7D4FD4FF47C720023C349C848FFF7CDFD4FF47C720023C049C548FFF7C6FD4FF47C71BD4823F07DF903DF88E02E
:40C48000C1A2AFF60821684623F010F8102204A96846FFF758F9002838DD0020FFF705FEFF224FF47C71B14823F05DF94FF47C720023AE49AE48FFF7A2FD4FF47C7200237B
:40C4C000AA49AC48FFF79BFD4FF47C720023A749A948FFF794FD4FF47C720023A349A748FFF78DFD4FF47C720023A049A448FFF786FD4FF47C7200239C49A248FFF77FFD25
:40C500004FF47C71994823F036F903DFA1A2AFF69421684622F0CAFF102204A96846FFF712F9002811DD012008F07DF901218F48B130FFF72FFD1BF0CDF830B10320EFF7B7
:40C5400077FD01219648FFF725FD04A8FFF78FFC04A8FFF740FC04A8FFF7FDFB04A8FFF790FB04A8FFF742FB04A8FFF701FB04A8FFF7BCFA04A8FFF729FA04A8FFF7E7F941
:40C5800004A8FFF793F904A8FFF751F904A8FFF7FEF80020FCF74EFBFCF7EEFE0646FCF7EEFD674800780CB070BD65480078704701B500BF012269467A4800683430FFF7AD
:40C5C00039F820B99DF80010684880F8241400BF7548C16B0220DFF8D4C100DF08BD2DE9FC470746884615461E46714890F84200C006C10A6E4890F8410041EA00206C498C
:40C6000091F8401040EA010908F01EF910B907F03BFC00B3FDB1F6B14D4504D1012E02D10120BDE8FC874D4503D1022E01D10220F7E74D4503D1032E01D10320F1E74D45CF
:40C6400003D1042E01D10420EBE74D4573D1052E71D10520E5E7002D6DD1464C042204F1340101A8FFF732FA012204F1B1016846FFF72CFA0198874205D19DF800004045B2
:40C6800001D10120CDE73C4C042204F1340101A8FFF71CFA012204F1B1016846FFF716FA0198874205D19DF80000404501D10220B7E7324C042204F1340101A8FFF706FA77
:40C6C000012204F1B1016846FFF700FA0198874205D19DF80000404501D10320A1E7284C042204F1340101A8FFF7F0F9012204F1B1016846FFF7EAF90198874205D19DF899
:40C700000000404501D104208BE71E4C042204F1340101A8FFF7DAF9012204F1B1016846FFF7D4F90198874244D19DF80000404540D1052075E73DE000380040F9030020D1
:40C74000FA030020F80300209CBE0008322E302E3100000030303030303030303030303000000000322E302E302E310030210020D0070068B80B0068A00F006888130068AE
:40C7800070170068581B0068322E302E302E363500000000322E312E302E333900000000E322002000040020785200200129040858E10020002034E738B5F84C042204F552
:40C7C000EC716846FFF782F940F2FD110098884201D0012038BDF24C042204F5EC716846FFF774F940F2FD110098884201D00220F0E7EC4C042204F5EC716846FFF766F946
:40C8000040F2FD110098884201D00320E2E7E64C042204F5EC716846FFF758F940F2FD110098884201D00420D4E7E04C042204F5EC716846FFF74AF940F2FD110098884273
:40C8400001D00520C6E70020C4E710B54FF47C71D74822F090FF4FF47C720023D449D548FFF7CDFB10BD10B54FF47C71D04822F082FF4FF47C720023CD49CE48FFF7BFFBAC
:40C880004FF47C720023CA49C448FFF7B8FB4FF47C720023C649C248FFF7B1FB4FF47C720023C349BF48FFF7AAFB4FF47C720023BF49BD48FFF7A3FB4FF47C720023BC49FD
:40C8C000BA48FFF79CFB4FF47C71B94822F053FF10BD2DE9F0410446884615461F463CB9B4482E183A4641463046FEF7A3FE30E0012C07D1A9482E183A4641463046FEF720
:40C9000099FE26E0022C07D1A5482E183A4641463046FEF78FFE1CE0032C07D1A1482E183A4641463046FEF785FE12E0042C07D19D482E183A4641463046FEF77BFE08E003
:40C94000052C06D199482E183A4641463046FEF771FEBDE8F0812DE9F04104460F46154698463CB993482E18424631463846FFF7ADF830E0012C07D188482E18424631461A
:40C980003846FFF7A3F826E0022C07D184482E18424631463846FFF799F81CE0032C07D180482E18424631463846FFF78FF812E0042C07D17C482E18424631463846FFF7C4
:40C9C00085F808E0052C06D178482E18424631463846FFF77BF8BDE8F08110B5744890F82444062C2CD2DFE804F02C030B131B234FF47C7200236E496848FFF700FB21E034
:40CA00004FF47C7200236A496548FFF7F8FA19E04FF47C72002366496248FFF7F0FA11E04FF47C72002362495F48FFF7E8FA09E04FF47C7200235E495C48FFF7E0FA01E02C
:40CA400000BF00BF00BF10BD2DE9F04105460E461746984643463A4631462846FFF7BFFD0446062C5ED2DFE804F05E031527394B4FF47C72002349494D48FFF727FB4FF48D
:40CA80007C7200234A494B48FFF7B9FA0120FFF78FFD54E04FF47C72002341494448FFF715FB4FF47C72002341494248FFF7A7FA0220FFF77DFD42E04FF47C7200233949C6
:40CAC0003B48FFF703FB4FF47C72002338493948FFF795FA0320FFF76BFD30E04FF47C72002331493248FFF7F1FA4FF47C7200232F493048FFF783FA0420FFF759FD1EE005
:40CB00004FF47C72002329492948FFF7DFFA4FF47C72002326492748FFF771FA0520FFF747FD0CE000BFFFF790FE0020FFF740FD002021494860272014F01EFC00BF00BF66
:40CB400004B103DFBDE8F0814FF40050704710B5174890F82404062840D2DFE800F040030C152F370D4C042211493C3104F13C00FEF760FD34E00A4C04220D493C3104F118
:40CB80003C00FEF757FD2BE0064C042208493C3104F13C00FEF74EFD22E00000B80B0068A00F00688813006870170068581B006830210020D0070068683200200B4C042246
:40CBC0000B4904F13C00FEF735FD09E0094C0422074904F13C00FEF72DFD01E000BF00BF00BF10BD0448042170470000701700686C210020581B00683E9BEFE310B51DF07E
:40CC000043F9FE49086009F031FEFC4880ED010A10BD10B5FA4890F84A00022824D1F84890F8BD0102281FD1F64890ED020ADFEDF60AB4EEE00AF1EE10FA0ADBFAF720FFC3
:40CC4000C4B223467D22ED490C3101200DF008FB2EE0FAF715FFC4B223467D22E7490C3100200DF0FDFA23E0E648D0ED010AE448B0F8BE0100EE100AB8EE400AF4EEC00A60
:40CC8000F1EE10FA0ADBFAF7FBFEC4B22346FA22DA490C3101200DF0E3FA09E0FAF7F0FEC4B22346FA22D5490C3100200DF0D8FA10BD10B52DED048B1AF024FD002867D094
:40CCC000FFF7A7FFEDF798FC18B10020CB49087261E0CA48007A60B9C84890F82000002859D10120C54908721DF0CEF8C349086051E0C248007A01280CD1C049C86947F29B
:40CD000030511DF0C7F8A0B30220BC490872FFF775FF40E0B948007A02283CD109F0A6FDB648D0ED010A30EEC00A10EE104A204627F0CCFA41EC190BB0EE490AF0EE690AFE
:40CD400023F09EFEB0EE408AF0EE608A9FEDAF0B53EC102B51EC180B27F0C0F80ED2A74890F82000012805D10020A44948720120087210E00120A14948720CE09F49086814
:40CD80004FF4FA611DF086F828B1FFF737FF02E000209A494872BDEC048B10BD994981F890007047974981F838007047F0EE400A9FED980A20EE800A704770B52DED0A8B3E
:40CDC00082B004468E4890F8BD010F287ED2DFE800F07D365EFC37FBFAF97D7D087DF8F7F600EDF704FC10EE105A284627F06EFA41EC1A0BB0EE4A0AF0EE6A0A23F040FEA7
:40CE0000B0EE409AF0EE609A51EC190B26F022FCA0619FED810A84ED1C0A94ED060A84ED010AEDF72EFC18B10020FFF7BBFF02E00420FFF7B7FF0420FFF7B0FF6AE200BF24
:40CE4000764800781BF08AF820B19FED750A84ED060A03E09FED700A84ED060A714800781BF07CF820B19FED6E0A84ED1C0A03E09FED690A84ED1C0A0420FFF793FF0420C3
:40CE8000FFF78CFF94ED060A84ED010AEEE3634800781AF027FE00EE100AF8EE400A9FED621A9FED620A10EE810A84ED0C0AE16821611CF0E9FFE060D4E90310091A6161C5
:40CEC000D4ED0C0AB0EE600A0A2100E0BFE304F118000AF0C8FC94ED060ADFED550AB4EEE00AF1EE10FA03D20020FFF75BFF0FE094ED060AF0EE040AB4EEE00AF1EE10FA84
:40CF000003DD0120FFF74EFF02E00420FFF74AFF0420FFF743FF94ED0C0AB5EEC00AF1EE10FA02D29FED3C8A01E094ED068A94ED0F0A84ED100A84ED0F8A94ED050AB8EEA2
:40CF4000400ADFED370A80EE201A11EE105A284627F0BCF941EC1A0B94ED0F0AD4ED100A30EE600A10EE101A084627F0AFF941EC1C0BB0EE4C0AF0EE6C0A23F081FDB0EEC0
:40CF800040BAF0EE60BA53EC1A2B51EC1B0B26F04FFC41EC190B26F05DFB60639FED1E0A84ED1C0AB0EE480AFFF700FF84ED010AD4ED0D0AB0EE600AFFF7F8FE06E0D9E29C
:40CFC000A9E1E6E2FBE112E103E069E084ED020A4CE3124800781AF085FD00EE100AB8EE400ADFED110A20EE200ADFED120A80EE201A84ED0C1AD4ED0C0A1DE0302900204F
:40D00000302100205429002000C0DA44000000401857B63FC0A90646000000005E07002000007A44620700203333533A9A99193FCDCCCCBE0CAC233FB0EE600A0A2104F1FC
:40D0400018000AF010FC94ED060ADFEDFE0AB4EEE00AF1EE10FA03D20020FFF7A3FE0FE094ED060ADFEDF80AB4EEE00AF1EE10FA03DD0120FFF796FE02E00420FFF792FE52
:40D080000420FFF78BFE1FED1C0A84ED1C0AD4ED060AB0EE600AFFF789FE84ED010AE5E2EA4800781AF01EFD00EE100AF8EE400A1FED231A1FED230A10EE810A84ED0C0AD2
:40D0C000D4ED0C0AB0EE600A0A2104F118000AF0CAFB94ED060A5FED2A0AB4EEE00AF1EE10FA03D20020FFF75DFE0FE094ED060AF0EE040AB4EEE00AF1EE10FA03DD0120AC
:40D10000FFF750FE02E00420FFF74CFE94ED0C0AB5EEC00AF1EE10FA02D21FED418A01E094ED068ACA4800781AF0DCFC00EE100AF8EE400A1FED441A1FED440A10EE810AEA
:40D1400084ED220AD4ED220AB0EE600A0A2104F170000AF088FB94ED1C0A5FED4B0AB4EEE00AF1EE10FA03D20020FFF717FE0FE094ED1C0AF0EE040AB4EEE00AF1EE10FA5C
:40D1800003DD0120FFF70AFE02E00420FFF706FE94ED220AB5EEC00AF1EE10FA02D25FED628A01E0D4ED1C8AB0EE480AFFF7FEFDB0EE401AB0EE680AFFF7F8FD31EE400ADC
:40D1C00010EE105A284627F081F841EC1A0BB0EE4A0AF0EE6A0A23F053FCB0EE409AF0EE609A51EC190B26F035FA60603EE2974800781AF077FC00EE100AB8EE400A5FEDE3
:40D20000760A20EE200A5FED750A80EE201A84ED0C1AD4ED0C0AB0EE600A0A2104F118000AF021FB94ED060ADFED860AB4EEE00AF1EE10FA03D20020FFF7B4FD0FE094ED91
:40D24000060ADFED810AB4EEE00AF1EE10FA03DD0120FFF7A7FD02E00420FFF7A3FD7C4800781AF03FFC00EE100AB8EE400A5FED920A20EE200A5FED910A80EE201A84ED02
:40D28000221AD4ED220AB0EE600A0A2104F170000AF0E9FA94ED1C0ADFED6A0AB4EEE00AF1EE10FA03D20020FFF778FD0FE094ED1C0ADFED650AB4EEE00AF1EE10FA03DDEE
:40D2C0000120FFF76BFD02E00420FFF767FD94ED060AD4ED1C0A30EE600A10EE101A084626F0F4FF41EC1B0BB0EE4B0AF0EE6B0A23F0C6FBB0EE40AAF0EE60AA51EC1A0B91
:40D3000026F0A8F909EE100AB0EE490AFFF74EFD84ED010AAAE16421E0681CF0BBFDE8B31CF0B2FDE06094ED0F0A84ED100A494800781EF070FD00EE100AB8EEC00A84ED33
:40D340000F0A94ED0F0AD4ED100A30EE600A10EE101A084626F0BAFF41EC1A0BB0EE4A0AF0EE6A0A23F08CFBB0EE409AF0EE609A51EC190B26F06EF92063D4ED0C0A9FED0E
:40D38000361A80EE810AF2EE040A80EE201A84ED0C1AD4ED0C0AB0EE600A00E00EE0032104F118000AF05FFA94ED060A84ED010A0420FFF7F7FC0420FFF7F0FC56E16421EA
:40D3C000E0681CF067FD00287DD01CF05DFDE06094ED0F0A84ED100A1C4800781EF01BFD00EE100AB8EEC00A84ED0F0A94ED0F0AD4ED100A30EE600A10EE101A084626F0A8
:40D4000065FF41EC1A0BB0EE4A0AF0EE6A0A23F037FBB0EE409AF0EE609A51EC190B26F019F9206394ED0C0ADFED0B0A80EE201A84ED0C1A94ED250A84ED260A0748007882
:40D440000EE00000CDCCCC3C33339F405E0700206107002060070020CDCCCC3D620700201EF0D9FC00EE100AB8EEC00A84ED250A94ED250AD4ED260A30EE600A10EE101ACD
:40D48000084626F023FF41EC1A0BB0EE4A0AF0EE6A0A23F0F5FAB0EE409AF0EE609A51EC190B26F0D7F88821085194ED220A5FED160A80EE201A84ED221AD4ED0C0AB0EED3
:40D4C000600A032100E054E004F118000AF0CBF9D4ED220AB0EE600A032104F170000AF0C2F994ED060AD4ED1C0AB4EEE00AF1EE10FA04DD94ED060A84ED010A03E094ED4D
:40D500001C0A84ED010AEDF7BCF818B10020FFF749FC13E094ED1C0AD4ED060A30EE600AF3EE090AB4EEE00AF1EE10FA03DD0220FFF738FC02E00420FFF734FCEDF7AEF84F
:40D5400018B10020FFF72AFC13E094ED060AD4ED1C0A30EE600AF3EE090AB4EEE00AF1EE10FA03DD0220FFF719FC02E00420FFF715FC7BE09FEDFB0A84ED0C0A9FEDF90A2E
:40D5800084ED010A0420FFF70DFC0420FFF706FC6CE0FA21E0681CF07DFCE8B36A4601A9F14800781EF08AFD05461CF06DFCE06094ED0F0A84ED100A9DED000A84ED0F0AFE
:40D5C00094ED0F0AD4ED100A30EE600A84ED0C0A94ED0C0AF5EE000A80EE201A11EE106A304626F073FE41EC1A0BB0EE4A0AF0EE6A0A23F045FAB0EE409AF0EE609A51EC90
:40D60000190B26F027F82063D4ED0C0AB0EE600A022104F1180000E018E00AF024F994ED060A84ED010A012D06D19DED010AB5EEC00AF1EE10FA03D10020FFF7B3FB02E099
:40D640000420FFF7AFFB0420FFF7A8FB0EE09FEDC50A84ED0C0A9FEDC30A84ED010A0020FFF7A0FB0020FFF799FB00BF00BF02B0BDEC0A8B70BD10B51AF057F8D0B1FAF7FE
:40D68000FFF9C4B22346FA22B84900200CF0E8FD9FEDB40AB64880ED060A9FEDB20A80ED060A042180F8381080F890100020B14948722EE0AE48FFF780FBAF48B0F8BE0147
:40D6C00018B90220A949087521E0A948D0ED010AA948B0F8BE0100EE100AB8EE400AF4EEC00AF1EE10FA09DBFAF7CAF9C4B22346FA229E4901200CF0B3FD08E0FAF7C0F950
:40D70000C4B22346FA22994900200CF0A9FDFFF7D0FA10BD97494872704731B50024BDF80000C82803DDC8200090022406E0BDF80000012802DA01200090032400BF0222E4
:40D7400069468E48006800F5DF70FDF773FF20B9BDF800008849A1F8BE0100BF204638BD31B50024BDF80000642803DD64200090022406E0BDF80000012802DA012000908B
:40D78000032400BF022269467C48006800F5DF70FDF750FF20B9BDF800007749A1F8BE0100BF204638BD31B50024BDF80000B0F5FA7F04DD4FF4FA700090022406E0BDF881
:40D7C0000000012802DA01200090032400BF022269466A48006800F5DF70FDF72BFF20B9BDF800006449A1F8BE0100BF204638BD31B50024BDF80000322803DD32200090B6
:40D80000022406E0BDF80000012802DA01200090032400BF022269465848006800F5DF70FDF708FF20B9BDF800005349A1F8BE0100BF204638BD31B50024BDF80000C82826
:40D8400003DDC8200090022406E0BDF80000012802DA01200090032400BF022269464748006800F5DF70FDF7E5FE20B9BDF800004149A1F8BE0100BF204638BD31B500247A
:40D88000BDF8000040F26351884203DD08460090022406E0BDF80000012802DA01200090032400BF022269463448006800F5DF70FDF7C0FE20B9BDF800002F49A1F8BE01DD
:40D8C00000BF204638BD31B50024BDF8000045F2CC01884203DD08460090022406E0BDF80000012802DA01200090032400BF022269462248006800F5DF70FDF79BFE20B917
:40D90000BDF800001C49A1F8BE0100BF204638BD10B52DED028BB0EE408A0024164890F8BD010E2853D2DFE800F0072B08122C091336522D4052493700BF00BFBCEEC80A58
:40D9400010EE101A88B2FFF7BEFF044648E000BFBCEEC80A10EE101A88B2FFF78FFF04463EE00000000000005E070020102A0020542900203029002030210020FC03002012
:40D9800000BF00BFBCEEC80A10EE101A88B2FFF752FF044624E000BFBCEEC80A10EE101A88B2FFF725FF04461AE0BCEEC80A10EE101A88B2FFF7F7FE044611E0BCEEC80AFB
:40D9C00010EE101A88B2FFF7CBFE044608E0BCEEC80A10EE101A88B2FFF79FFE044600BF00BF4120EFF7BCFD0020FFF793FE2046BDEC028B10BD10B52DED020B00BF0422BA
:40DA00006946FC48006800F5E670FDF713FE20B99DED000AF84880ED730A00BFF748016D0120DFF8DCC300DF1CBD10B52DED020B00BF04226946EF48006800F5E470FDF78D
:40DA4000F9FD20B99DED000AEB4880ED720A00BFEA48016D0120DFF8A8C300DF1CBD10B52DED020B00BF04226946E248006800F5E270FDF7DFFD20B99DED000ADE4880ED84
:40DA8000710A00BFDD48016D0120DFF874C300DF1CBD10B52DED020B00BF04226946D548006800F5E070FDF7C5FD20B99DED000AD14880ED700A00BFD048016D0120DFF808
:40DAC00040C300DF1CBD10B5CB4890F8300091280ED0C94890F83000922809D0C64890F83000712804D0C44890F83000B82818D1C14890F8BD010A2813D19FEDC20AFFF775
:40DB000007FF9FEDC10AFFF7C4FF9FEDC00AFFF7A6FF9FEDBF0AFFF788FF9FEDBE0AFFF76AFFB54890F83000702804D0B24890F83000932819D1B04890F8BD010A2814D18C
:40DB40009FEDB50AFFF7E4FE9FEDB40AFFF7A1FF9FEDB30AFFF783FF9FEDB20AFFF765FF9FEDB10AFFF747FF18E0A34890F8BD010A2813D19FEDA80AFFF7CAFE9FEDA20A49
:40DB8000FFF787FF9FEDA10AFFF769FF9FEDA70AFFF74BFFBBEE040AFFF72DFF964890F8BD01012804D1B7EE000AFFF7B1FE53E0914890F8BD01022804D19FED9D0AFFF70E
:40DBC000A7FE49E08C4890F8BD01032804D1B3EE040AFFF79DFE3FE0874890F8BD01042804D11FEDA00AFFF793FE35E0824890F8BD01052804D19FED8F0AFFF789FE2BE0B7
:40DC00007D4890F8BD01062804D19FED8B0AFFF77FFE21E0784890F8BD01072804D0764890F8BD010D2804D1B1EE040AFFF770FE12E0714890F8BD01092804D19FED7E0A0E
:40DC4000FFF766FE08E06C4890F8BD010C2803D1B2EE040AFFF75CFE10BD10B5664890F8BD010A281CD1644890F8300091280ED0614890F83000922809D05F4890F830006F
:40DC8000712804D05C4890F83000B82803D1FA20FFF789FD03E04FF49670FFF784FD00E000BF00BF10BD00B589B019F02BFD002879D0514890F8BD010E2875D2DFE800F0E0
:40DCC00074072A2B4E7576C274FDFCFBFAF9002000900190029003460246584903900846007819F010FE002000900190029003460246534903900846007819F004FE012103
:40DD00004E4800781AF0ADF901214D4800781AF0A8F999E100BF002000900190029003460322464903900846007819F0ECFD0020009001900290034603224149039008464B
:40DD4000007819F0E0FD03213C4800781AF089F903213B4800781AF084F975E101200021009101910B460A46CDE9021033490846007819F0C8FD01200021009101910B4609
:40DD80000A46CDE902102E490846007819F0BBFD01212A4800781AF064F90121284800781AF05FF950E150E129E100BF002000900190029003460322204903900846007840
:40DDC00019F0A1FD0020009001900290034603221B4903900846007819F095FD0021174800781AF03EF90021154800781AF039F92AE10000FC0300203021002078520020F3
:40DE00000129040800007A43C6DCB53DB8AF833E52B8444114AE4740000096436744293EE5F25F3E52B862416666E6C133331B41000016430080BB440000C8425E070020B3
:40DE400061070020002000900190029003460222F84903900846007819F055FD002000900190029003460322F34903900846007819F049FD00200090019002900346022280
:40DE8000EE4903900846007819F03DFD0221E94800781AF0E6F80221E84800781AF0E1F8002000900190034614220121029004A804E092E072E01EE0A3E0A1E01DF0CAFD8F
:40DEC00004A8DFEDDF0A9FEDDF0A02230022DE490090D84800781DF0A5FC04A8DFEDD80A9FEDD80A02230322D8490090D34800781DF098FCA8E0002000900190029003466D
:40DF00000222CC4903900846007819F0FCFC002000900190029003460322C74903900846007819F0F0FC002000900190029003460222C24903900846007819F0E4FC0621FB
:40DF4000BC4800781AF08DF80621BC4800781AF088F8002000900190034614220121029004A81DF077FD04A8DFEDB50A9FEDB50A02230022B4490090AE4800781DF052FCA9
:40DF800004A8DFEDAF0A9FEDAF0A02230322AF490090AA4800781DF045FC55E0002000900190029003460222A24903900846007819F0A9FC01219F4800781AF052F8A44839
:40DFC000DFED9F0A9FEDA30A052300229E490090984800781DF026FC36E0002000900190029003460322944903900846007819F08AFC0021904800781AF033F824E000BFA6
:40E0000000BF002000900190029003460322894903900846007819F076FC002000900190029003460322844903900846007819F06AFC01217F4800781AF013F801217E4806
:40E0400000781AF00EF800BF00BF834890F8BD01824908700020FFF75DFB00208049087209B000BD7F49097D012900D100E00021084670477B48407D70477A48007D08B979
:40E08000012070470020FCE7774909880143764A11807047F7EE000AB0EE600A7C2202706D4A92F8BD210E2A22D2DFE802F007120809130A0B1721141B211E1800BF00BF4F
:40E0C00000BF00BF01224270DFED680AB0EE600A0FE000BF00BF022242700AE000BF0422427006E00522427003E00622427000E000BF00BF594AD2ED060A60EE800AFCEEB5
:40E10000E00A10EE902A91B281700A0AC270534AD2ED1C0A60EE800AFCEEE00A10EE902A91B201710A0A42714B4AB2F8BE1181710A0AC2717047494890ED010A704701B5DD
:40E1400000BF012269464A48006800F2BD10FDF771FA20B99DF800003F4981F8BD0100BFFFF7B1FC012003F0B9F81E20EFF7F8F908BD01B500BF022269463D48006800F59E
:40E18000E870FDF757FA20B9BDF800003249A1F8D00100BF08BD00202F4991F8BD110E291AD2DFE801F01A0D0A070E0B0810131B1519171100BF012011E000BF01200EE075
:40E1C00000BF01200BE000BF012008E0012006E0012004E0012002E000BF00BF00BF00BF704700201C4991F8BD110E291DD2DFE801F01D0F0B07100C0812151E171C1A1309
:40E2000000BF40F2635013E000BF45F2CC000FE000BFC8200CE000BF322009E0C82007E04FF4FA7004E0642002E000BF00BF00BF00BF70475E0700206107002062070020FA
:40E240000000000000504347000400400000014080EC002000247449302100205429002030290020102A002008040020C0A90646FC0300200020C84991F8381009B91420F9
:40E2800012E0C54991F83810012901D116200BE0C14991F8901009B9152005E0BE4991F89010012900D11720704770B50424BB4880780A2876D2DFE800F0051376C5C5C5F2
:40E2C000C5BFC1C30020B5490870C8808860FFF750FFB2488078B149487001208870B2E0FFF7C8FFAD4908700846007810B10720887056E0A948806820B91BF0C5FDA74946
:40E3000088604EE0A54988684FF47A711BF0C2FD002846D0FFF70FFFBCEEC00A10EE100A85B22846FFF725FF9D48B0F8AC0068B19B48B0F8AC009A49B1F8D011884205DDC2
:40E340009748B0F8AC009549C88021E09448B0F8D001002803DC01209049C88018E0904890F8BD01032804D08D4890F8BD01062805D18B48B0F8D00100F5FA7006E0884810
:40E38000B0F8D0018000032190FBF1F08349C8800220824988701BF077FD804988600020087350E04EE0FFF7C6FE7C48C08800EE900AF8EE600AB4EEE00AF1EE10FA05DBBF
:40E3C0007648007B401C7549087302E0002073490873FFF74FFF714908700846007810B10720887027E06D48007B04280DDB6B48C08800EE900AF8EE600AB0EE600AFFF7DE
:40E4000087FA09206549887015E06449886841F288311BF03FFD70B16048C08800EE900AF8EE600AB0EE600AFFF772FA07205B4988701820087006E0012404E0022402E00A
